:100000000C9415180D943F090D9414090D94E908EA
:100010000D94BE080D9493080D9468080D943D0846
:100020000D9412080C9446180C9446180C9446181B
:100030000C9446180C9446180C9446180D94712193
:100040000C9446180C9446180C9446180C944618B8
:100050000C9446180C9446180C9446180D947D0682
:100060000C9446180D94EF0C0D94C50C0C94461886
:100070000C9446180C9446180C9446180C94461888
:100080000C9446180C9446180C9446180C94461878
:100090000D941B0F0D94910E0D94D30E0D94092306
:1000A0000C9446180C9446180C9446180C94461858
:1000B0000C9446180C9446180C9446180C94461848
:1000C0000C9446180C9446180C9446180D949B0CEE
:1000D0000D94710C0C9446180D94470C0D941D0C46
:1000E0000C94461807634236B79BD8A71A3968564E
:1000F00018AEBAAB558C1D3CB7CC5763BD6DEDFD4A
:10010000753EF6177231BF000000803F0800000006
:10011000BE922449123EABAAAA2ABECDCCCC4C3EFC
:1001200000000080BEABAAAAAA3E00000000BF00EB
:100130000000803F0000000000084178D3BB4387E7
:10014000D1133D190E3CC3BD4282AD2B3E68EC82FB
:1001500076BED98FE1A93E4C80EFFFBE01C4FF7F80
:100160003F00000000000D9430040C9474890D943D
:1001700052150C94F9950C947F230C940B8A0C94D3
:10018000018B0C94BD250C9409200C943B330D94E9
:1001900032040C9486A50C94F6810C947CBF0C94CC
:1001A0006B9A0C9443440C941FDF0C9478350C9498
:1001B0007B270C9410C90C942DE70C94EBE50C9460
:1001C0000BA50C946F2F0C94EFE50C941C430C942E
:1001D000139F0D9490050C94A5190C9403E60C94B0
:1001E000A3430D944B200C94E9580C94B61F0C9427
:1001F0009A340C94E2E50C94C5240C94DD2F0C94F5
:1002000051620C94E0350D9486040C9449C30C940F
:1002100068240D94F5030C944EC70D9480010C9442
:1002200053210C947A440C9423A50C94ED1D0C944A
:10023000DEE50C94D48A0C94B6240C9490B80D94FA
:100240004A030D94E7150D94BC030C94FCDE0C944A
:1002500023E70C9421A50C9411E60C94A7250D948A
:1002600028060D948D2E0C94574E0C94FC1C0C9467
:10027000CEAE0C9412190C94D3250C9442220C94FB
:10028000BC880D94FE020C9402C00D9409190C94C4
:1002900066350C94C1AE0D94F7140C9407E60C94DB
:1002A00074630D94A9040C94D6530C94AF8A0D94E6
:1002B0000F040C9410910C94F7940C94F5E50C94A5
:1002C000BBE60C9438540C94BC550C9434870C94B5
:1002D000B0810C94B98C0C9460190C94D9A50C9431
:1002E00062450C94EB900C9426DF0C94D7610D942E
:1002F0001B030C94801F0C9419930C941BC70D9432
:10030000CB030D94FC030C941F430C94A08A0C9413
:1003100054AF0C94EA210C941C1F0C9469190C9492
:100320009F8F0D94CE110C94A7BA0C942FB40C94FB
:100330003B8B0C94FB8A0C9441E70C94BE550C94B7
:1003400051180C9450A00C94AC440C94AC620C94D6
:10035000CF880C947C190C9400E70C9428ED0C9435
:10036000228B0C94F0880C9421B30C94DB440C94F5
:100370000B450C94E7620C94B8C70D94D5010C940E
:1003800080240C942ACB0C94F9E50C9489B30C943A
:10039000EF430C94B8C10C9466900C94A78C0C9409
:1003A0008F240C9438330C9455E70C94EF1D0D9466
:1003B0007A190C9491340C948F260D94DD040D94CD
:1003C0007E010C94B18C0C94FDE50C944FC70C94F9
:1003D000E6E60C94E2350D9474030C9445220D94DA
:1003E00085040C94C8E60D94782E0C94B2250C94D8
:1003F0001C630C9447B40C940F440C9442450C9429
:1004000025ED0C94A6350C944C230C9403DF0C942E
:10041000542F0C94B62F0D9420110C9482920C94AE
:10042000D4240C940AA40C948B9F0C9466190C94FD
:1004300073B40C941F440C94668C0C94FE180C94AA
:10044000E5E50C94DD1A0C9424540C94612F0C9463
:1004500015E60C94FE8A0C94EF230C9411280C944E
:10046000FEC70D942C180C94A4810C9406410C9496
:10047000B5CD0C94AD8C0D9407040C94441A0C94D7
:10048000B78C0D9495110C94A6190C94EC990C94BE
:100490007D4D0C942ECA0C94802F0D9437110C9422
:1004A000128A0D943A0A0C9488240D94E5030D9455
:1004B000EF020C946B260C9469AE0C941EB40C9451
:1004C000CF960C94A7260C9409ED0C94B3A40C942D
:1004D00035430D94C8150C94AE430D940C050C9443
:1004E00048180C9408450C940AB40C9442870C9458
:1004F000F29D0C947DA00C940BE60C949D810C94C1
:1005000023D90C9437AB0C940E270C949D530C9468
:10051000AB8C0C949F340C9494340D94E9010C949E
:10052000CCD80C94ED430C9476A30C94FC870C94DB
:100530004C890C945E910C9452A40C94B58C0C9440
:10054000E82F0C94D0B30C9452190C9495A40C94ED
:10055000DCE60D940F200C94C2880C9414E70C94E4
:10056000F0530D9457190C94361C0C940A320C94C9
:10057000C9190C9478230C9490210D9437060C948F
:100580001D4E0C94C9780C94D6E50C94DD520C9455
:10059000F8580C949B630C94CE620C94EEE60C9489
:1005A0001A540C946F350D94E2190C94B3190C94F1
:1005B000C2550C9406190C94DA270C94D78A0C9423
:1005C00059440C9423A00C9457300C94A98C0C948F
:1005D000E0190D9422190C94AE4D0C9400C80D94A2
:1005E00098180C9482390D943C030D9422130C94AA
:1005F00077630C949EA50C94A9380C941BA50C94BD
:10060000B9350C9402430C948F190D947D010C9410
:1006100028530C9451220C944DC70C94A6380C947A
:1006200071240C9434220C94AD9F0C944CC70D94FF
:1006300087040C9437E70C9464190C94DC440D94F3
:10064000971C0C94C82F0D9444050C94088A0C94A4
:1006500093350C94BC530C94BD8A0C9481350C9446
:10066000B9260C94BA470D94B0190C94D2E60D94A7
:1006700090020C941B370C94CC250C94AB330C9447
:10068000D0E50D94C6010C94FE210C94C8AA0D94DB
:1006900030180C940F880D9410040D94BF200C9406
:1006A00011220C94F31A0D940F150C94C3E60C94BC
:1006B000AF8C0C9484440C9475CA0C94CC350C9477
:1006C000402F0D9483110C940A190C9411DF0C9493
:1006D000EA1F0C9408ED0C94F5270C94A4330C94A9
:1006E0000CD90C94CB8F0C9467890D9417110C9432
:1006F00097340C94BC240D9496040D940A1D0C940C
:10070000D6350C948B270D9443020C9424620C94E0
:100710003C300C9410E60C94599A0C94C59D0D94A1
:1007200026040C940CAE0C94F2230D94B0040C949B
:10073000FAC80C94D6A40C94F6E60C94BA440C9423
:10074000E8A50C9460CA0C94D6410C94DAE50C949C
:100750009E520C94AF240C9445800C9439940C94C4
:10076000808C0D94240B0C94AC850C94F88A0D9419
:100770008D030C944FA30C9402190C9470A40C9448
:1007800063530C94CB440C94EDD80C942DDF0C9453
:10079000E0430C9441330C944A9A0C9407230C9434
:1007A000258B0C9428190D94F7010C94FAC30C9422
:1007B000F5B30C94FAA40C94F2580C94ABB30C94CB
:1007C000E7420C941FA50C940E190C9436B00C94AF
:1007D00090A50C94308B0C94729F0C9483980C947D
:1007E000DED80C943EA50C94B38C0C9448190C9450
:1007F000B1B90C940AE70D9486030C946B610C94C8
:10080000FFC70C94F0610C94C4430C9472AE0C942A
:100810005B3B0C9410540C941E1A0C949E440C9444
:100820007A630C9428220C94311A0D947F010D9454
:100830002C050D94E1030C94309A0C940ADF0C946F
:100840004BE70C945F410C943DCB0C945A910C9463
:100850007C1D0D9411160C9452920C94C5D80C94D6
:10086000FFC80C9405350C9437220C94C6440D94A3
:1008700006110C946A620C94F8790C948A4E0C94CC
:1008800016190C9462910C942F900C94A1610C9405
:10089000BD230C94A58C4E414E494E495459494EA6
:1008A00046CDCCCC3D0AD7233C17B7D13877CC2BDB
:1008B000329595E6241FB14F0A000020410000C880
:1008C0004200401C4620BCBE4CCA1B0E5AAEC59D01
:1008D000746364696E6F70737578585B00556E6BE6
:1008E0006E6F776E207375666669782000556E6B43
:1008F0006E6F776E20636D642000636C7243747258
:100900003A2000454F46002F00496E3A20003D0036
:10091000494E3A003D004C454741435920494E3A23
:10092000002500C2B04320483D00204448543232E4
:1009300020747970652E20543D00494E3A00204EB7
:100940006F20656D69742064617461210020436FBC
:10095000756E74657220747970652E2076616C3DB9
:1009600000494E3A0020436F756E746572207479A9
:1009700070652E20494E434F525245435420496ED4
:1009800074657272757074206E756D626572212166
:1009900021004952513A002D3E00200023002D3EF7
:1009A00000200050656E6465643A2023005365742E
:1009B000436D643A00737566666978436F64653A9F
:1009C0000020666F7220286D73293A004354524C00
:1009D0003A205363686564756C6520636D6420001C
:1009E000206D73203A0041726D656420666F72203D
:1009F000002044697361726D6564002074696D65DF
:100A00003A004354524C3A205265733A003D00502C
:100A1000696E3A004354524C3A20436F6D6D616EDB
:100A20006420626C6F636B65642062792064726914
:100A3000766572206F72206368616E6E656C2066E9
:100A4000726F7A656E004354524C3A204F4E3A41D1
:100A50006C7265616479204163746976650A00434C
:100A600054524C3A2048414C543A416C726561648E
:100A70007920496E6163746976650A004354524C6B
:100A80003A20584F4E3A2044697361626C65640A9B
:100A9000004354524C3A20584F4E3A416C726561B3
:100AA0006479204163746976650A004354524C3A74
:100AB00020584F464620736B69707065642E205035
:100AC00072657620636D643A004354524C3A205468
:100AD00075726E6564206F66662066726F6D3A008F
:100AE0004354524C3A20526573746F7265642066A9
:100AF000726F6D3A004354524C3A2049676E6F72E0
:100B000065642C206368616E6E656C20636D643D66
:100B10000020457865633A004354524C3A204163C3
:100B2000746976653A004354524C3A2048414C541B
:100B30003A416C726561647920496E6163746976CB
:100B4000650A004354524C3A20584F4E3A204469AB
:100B50007361626C65640A004354524C3A20584FEA
:100B60004E3A416C726561647920416374697665BF
:100B70000A004354524C3A20584F464620736B6942
:100B8000707065642E205072657620636D643A0043
:100B90004354524C3A205475726E6564206F6666F9
:100BA0002066726F6D3A004354524C3A205265737E
:100BB000746F7265642066726F6D3A004354524CD4
:100BC0003A204E6F7420656E6F756768206D656D95
:100BD0006F727920666F722067726F7570206F7008
:100BE00065726174696F6E00496E76616C6964202C
:100BF00061726700496E76616C696420617267009A
:100C00004354524C3A20556E6B6E6F776E2073755D
:100C10006666697800536B697070656420686F6DF3
:100C20006965207374756666002000205375623D07
:100C300000204974656D3D004354524C3A205241A6
:100C40004D3D004354524C3A204F75744F664D65EC
:100C50006D6F72793A2000282D292000282B292039
:100C6000002076616C7565206973200020756E6BBD
:100C70006E6F776E0A005D3D005B0020696E7661E5
:100C80006C6964002000206F6B003A002066616987
:100C90006C6564003A005265747279696E6720561B
:100CA0004354454D5020434D440A005265747279B7
:100CB000696E6720564320434D440A0052657472A2
:100CC00079696E67206D6F6462757320434D440AC5
:100CD000005265747279696E6720434D440A0020A2
:100CE0006572726F723D004D423A20706F6C6C6994
:100CF0006E6720002056616C3A20004D423A200079
:100D00004D423A204E6F7420737570706F72746527
:100D1000642072656720747970650A004D423A203C
:100D2000706F6C6C696E672064696D6D6572200010
:100D30004D423A20496C6C6567616C206172677541
:100D40006D656E74730A00206572726F723D004D9E
:100D5000423A20706F6C6C696E6720504920002DFC
:100D6000004D423A2050492056616C203A004D42D5
:100D70003A20706F6C6C696E6720504920004D42BC
:100D80003A20706F6C6C696E6720464D2066617505
:100D90006C742000206572726F723D004D423A20E3
:100DA000706F6C6C696E6720002D004D423A2046D2
:100DB0004D2056616C203A004D423A20706F6C6CA9
:100DC000696E6720464D20004354524C2F706F6C63
:100DD0006C3A204F75744F664D656D6F72793A208D
:100DE00000207365632072656D61696E696E6700CE
:100DF0005374617475732064656666657265640A10
:100E0000002D3E005075623A20002D3E0050756264
:100E10003A20002D3E005075623A2000000000008C
:100E200000636D640000736574000076616C0000FF
:100E300064656C000048535600005247420000664B
:100E4000616E00006D6F6465006374726C0068759C
:100E5000650000736174000074656D7000726177E5
:100E600000002D3E005075623A20002D3E00507566
:100E7000623A2000556E6B6E6F776E20636D642052
:100E80000A000000000000000000004F4E000000BB
:100E9000000000004F46460000000000005245538D
:100EA000540000000000544F47474C4500000048E4
:100EB000414C540000000000584F4E00000000005C
:100EC00000584F46460000000000494E435245413D
:100ED000534500444543524541534500454E414228
:100EE0004C4500000044495341424C450000554EDA
:100EF000465245455A4500465245455A4500000070
:100F00004155544F000000000046414E5F4F4E4C8B
:100F100059004849474800000000004D45444955E4
:100F20004D0000004C4F57000000000000484541B4
:100F3000540000000000434F4F4C000000000044EC
:100F4000525900000000000053544F5000000000B0
:100F500000524742000000000000485356000000C5
:100F6000000000206661696C65643A004D6F646240
:100F70007573206F7020004D423A206F6B003D006A
:100F80004D423A205643230020636D643D003D00EE
:100F90004D423A2056435F6865617423004D423AE2
:100FA000204E6F7420737570706F72746564207258
:100FB000656720747970650A002056616C3A307854
:100FC0000020543A00205265673A3078004D423A8A
:100FD00020416464723A00444D5800000000000053
:100FE000444D58524742570000444D585247420022
:100FF000000050574D0000000000004D4255534482
:10100000494D0000544845524D4F00000052454C98
:1010100041590000000047524F5550000000005653
:101020004354454D500000004D4255535643000077
:10103000004143484149455200005350494C454402
:101040000000004D4F544F52000000005049440032
:1010500000000000004D42555300000000005541C3
:101060005254425244470052454C415950574D004A
:10107000444D5852474257570056454E545300006E
:101080000000454C455641544F5200434F554E5475
:101090004552000048554D0000000000004D4552EB
:1010A00043555259000020002D3E00436F6E766577
:1010B0007274696E6720002D3E0057726F6E672054
:1010C00041737369676E6D656E7420005247427894
:1010D0003A200020764C6576656C3A0020436F6EAE
:1010E00076563A0020436F6E76533A0020486F746C
:1010F0003A00436F6C643A0020436F6E76657274F9
:10110000656420563A00436F6E766572746564209C
:10111000533A002D3E0057726F6E6720417373691A
:10112000676E6D656E7420002D3E0057726F6E679E
:101130002041737369676E6D656E7420005361762C
:1011400065643A000000000000000000004F4E00FF
:101150000000000000004F46460000000000005262
:101160004553540000000000544F47474C450000D1
:101170000048414C540000000000584F4E00000051
:10118000000000584F46460000000000494E435200
:101190004541534500444543524541534500454E62
:1011A00041424C4500000044495341424C45000037
:1011B000554E465245455A4500465245455A45000A
:1011C00000004155544F000000000046414E5F4F63
:1011D0004E4C59004849474800000000004D454426
:1011E00049554D0000004C4F5700000000000048DA
:1011F0004541540000000000434F4F4C00000000E8
:101200000044525900000000000053544F500000A9
:101210000000005247420000000000004853560002
:10122000000000000020537566663A002041543AE1
:1012300000206973200044656C6574696E672063E3
:101240006F6E662E2052414D207761733A005374C1
:101250006F70706564006E6F7468696E6720746F7C
:101260002073746F700053746F7070696E672063C1
:1012700068616E6E656C73202E2E2E004E6F74208A
:10128000756E6C6F636B656420696E2031307320FE
:101290002D20636F6E74696E7565202E2E2E00559D
:1012A0006E6C6F636B696E6720636F6E6669672033
:1012B0002E2E2E00436F6D706C6574652E20526566
:1012C0006D6F766520746F706963200024636F6DA5
:1012D0006D616E6400536B697070696E672E2E00CD
:1012E000436C65616E55702072657461696E6564EA
:1012F00020746F7069632000220022004F75744FC4
:10130000664D656D6F727921005D20003A5B000AC1
:10131000005D00456D7074793A205B000A003A0068
:101320004D41433A00554450205379736C6F672008
:10133000696E697469616C697A65642E0A00537913
:10134000736C6F6720706172616D733A002E6C6F01
:1013500063616C0053657276696365207265636FC3
:1013600072643A20006D444E5320726573706F6E44
:1013700064657220737461727465642E00457272C4
:101380006F722073657474696E67207570204D44A8
:101390004E5320726573706F6E6465722100476FE3
:1013A0007420495020616464726573733A00276940
:1013B00070205B69705B2C646E735B2C67775B2CB1
:1013C0007375626E65745D5D5D5D27202D207365AC
:1013D00074207374617469632049500A004661691E
:1013E0006C656420746F20636F6E666967757265E3
:1013F0002045746865726E6574207573696E672028
:10140000444843502E20596F752063616E207365E8
:1014100074206970206D616E75616C6C792100209B
:101420004D41534B3A002047573A0020444E533A1F
:10143000004C6F616465642066726F6D20666C613C
:1014400073682049503A000A757365732044484315
:10145000500A005374617274696E67206C616E008B
:10146000546F6F206D616E79204D51545420636F1D
:101470006E6E656374696F6E206572726F72732E23
:101480002052657374617274204C414E0020747256
:101490007920616761696E20696E2035207365630C
:1014A0006F6E6473006661696C65642C2072633DC5
:1014B000004177616974696E6720666F722072659A
:1014C0007461696E656420746F7069637300636F23
:1014D0006E6E65637465642061732000202E2E2E6D
:1014E0000020757365723A003A000A417474656DA4
:1014F0007074696E67204D51545420636F6E6E6531
:101500006374696F6E20746F2000646973636F6E1B
:101510006E6563746564005573696E67204D515440
:10152000542070617373776F72642066726F6D20E0
:10153000636F6E666967002E6C6F63616C006D444B
:101540004E53206E616D6520757064617465643AF8
:101550002000446576696365204E616D653A0041FF
:1015600074206C6561737420646576696365206EB0
:10157000616D6520616E642062726F6B65722049D7
:1015800050206D75737420626520636F6E666967A5
:101590007572656400246E6F646573004F4E2C4F46
:1015A00046462C48414C542C524553542C584F4ECF
:1015B0002C584F46462C544F47474C450024666FE5
:1015C000726D617400656E756D0024646174617480
:1015D0007970650068737600636F6C6F7200302DF0
:1015E00032353500696E746567657200666C6F61CF
:1015F0007400332E302E310024686F6D69650075DC
:101600007074696D652C667265656865617000341B
:101610006439303964645F323032332D31312D32E8
:1016200030004C696768744875622000246E616DF3
:101630006500526562696E642073756363657373D8
:101640002E20495020616464726573733A004572BC
:10165000726F723A20726562696E64206661696CAD
:101660000052656E65776564207375636365737397
:101670002E20495020616464726573733A0045728C
:10168000726F723A2072656E657765642066616973
:101690006C000A4E6F206C696E6B0033307320450E
:1016A0004550524F4D206973206E6F742072656CE7
:1016B0006F616465642E205265626F6F74004163D0
:1016C00063657074696E6720636F6D6D616E6473BE
:1016D0002E2E2E0A004E6F204D51545420636F6EF3
:1016E00066696775726564004C6F6164696E672036
:1016F000636F6E6669672066726F6D20706F7274BB
:10170000616C2064697361626C65642E2075736519
:1017100020676574204F4E20746F20656E61626C87
:101720006500436F6E6669672069732076616C6936
:101730006400436F6E74696E756520776974682004
:1017400070726576696F75736C79206C6F61646512
:101750006420636F6E6669670043757272656E74AC
:10176000204C414E20636F6E6669672869702C6457
:101770006E732C67772C7375626E6574293A000A54
:1017800055736520746865736520636F6D6D616E58
:1017900064733A202768656C7027202D207468696F
:1017A0007320746578740A276D61632064653A61FB
:1017B000643A62653A65663A66653A303027207366
:1017C000657420616E642073746F7265204D4143AF
:1017D0002D6164647265737320696E2045455052B3
:1017E0004F4D0A276970205B69705B2C646E735BD8
:1017F0002C67775B2C7375626E65745D5D5D5D272C
:10180000202D2073657420737461746963204950BE
:101810000A277361766527202D2073617665206322
:10182000757272656E7420636F6E66696720696E8B
:10183000204E5652414D3B204F4E7C4F4646202D68
:1018400020656E61626C652F64697361626C6520EE
:101850006175746F736176650A2767657427205B0D
:10186000636F6E66696720616464725D27202D2056
:1018700067657420636F6E6669672066726F6D209E
:101880007072652D636F6E66696775726564205549
:10189000524C20616E642073746F726520616464C1
:1018A000722C204F4E7C4F4646202D20656E616283
:1018B0006C652F64697361626C6520646F776E6C10
:1018C0006F6164206F6E20737461727475700A2783
:1018D0006C6F616427202D206C6F616420636F6ED4
:1018E0006669672066726F6D204E5652414D0A2719
:1018F00070776427202D20646566696E6520616EAF
:10190000642073746F7265204D515454207061735C
:1019100073776F72640A276F746170776427202D64
:1019200020646566696E6520616E642073746F72F1
:10193000652048545450204150492070617373779A
:101940006F72640A276C6F67205B73657269616CE4
:101950005F6C6F676C6576656C5D205B7564705F4E
:101960006C6F676C6576656C5D27202D20646566FD
:10197000696E65206C6F67206C6576656C20283019
:101980002E2E37290A276B696C6C27202D20746551
:101990007374207761746368646F670A27636C658A
:1019A000617227202D20636C65617220454550527D
:1019B0004F4D0A2773656172636827202D20736578
:1019C0006172636820312D77697265206465760ADB
:1019D000277265626F6F7427202D207265626F6FAA
:1019E0007420636F6E74726F6C6C657200536F66F7
:1019F00074207265626F6F74696E672E2E2E0020E0
:101A00006E65770020697320003157543A003157D2
:101A1000543A20536561726368696E672064657625
:101A20000052414D3D000A5379736C6F6720000AE4
:101A3000312D7769726520000A6D71747420000A77
:101A40006D6F64627573207632000A6D6F64627523
:101A50007320763120282B29000A696E7075747303
:101A600020000A6974656D7320000A436F6E666911
:101A700067757265643A00496E697469616C697A68
:101A8000696E6720496E70757473003157543A203F
:101A90007365747570207265736F6C7574696F6EA1
:101AA00020003157543A204453323438322D3130EB
:101AB00030206E6F742070726573656E74003157DC
:101AC000543A204453323438322D313030204932A8
:101AD0004320726573746F726564003157543A2005
:101AE000427573207265736574206572726F72003F
:101AF0003157543A204275732052657365742064DF
:101B00006F6E65003157543A204453323438322DC9
:101B10003130302070726573656E742C207265737D
:101B20006574004572726F7220312D7720696E697D
:101B300074003157543A204453323438325F3130D4
:101B4000305F4932435F544F5F31575F42524944DF
:101B5000474520696E697400444D584F75742E20B6
:101B6000467265653A00444D58696E204275666656
:101B7000657220616C6C6F632065727200496E69DA
:101B80007420696E2063683A003B003D0050696E26
:101B90003A003B003D4C4F5700546865726D6F3AF8
:101BA000004F6E6520776972652052656164790A1D
:101BB00000467265653A00444D58206F7574207375
:101BC0007461727465642E204368616E6E656C7317
:101BD0003A2000444D5820696E2073746172746518
:101BE000642E204368616E6E656C733A00417070BC
:101BF0006C79696E6720636F6E66696700436F6E0C
:101C0000666967206175746F736176653A000A537F
:101C100079736C6F67206465627567206C657665A3
:101C20006C3A0053657269616C2064656275672067
:101C30006C6576656C3A0053617665640A0053659D
:101C4000742064796E616D69632049500A004545CE
:101C500050524F4D20636C65617265640A004D51AE
:101C600054542050617373776F726420757064618F
:101C70007465640A004F54412050617373776F722A
:101C80006420757064617465640A00636F756C64C8
:101C9000206E6F742070617273653A200055706415
:101CA000617465640A004E6F20495020616472655A
:101CB00073730052656C656173696E6720736F633F
:101CC0006B657420616E64207265747279002053B4
:101CD00061766564004C6F6164696E672048545496
:101CE0005020636F6E666967206F6E207374617237
:101CF0007475703A000000000000000000004F4EB4
:101D0000000000000000004F4646000000000000F8
:101D1000524553540000000000544F47474C4500C3
:101D2000000048414C540000000000584F4E000095
:101D300000000000584F46460000000000494E4396
:101D400052454153450044454352454153450045A2
:101D50004E41424C4500000044495341424C45002D
:101D600000554E465245455A4500465245455A454E
:101D70000000004155544F000000000046414E5FF6
:101D80004F4E4C59004849474800000000004D455F
:101D90004449554D0000004C4F5700000000000022
:101DA000484541540000000000434F4F4C000000E4
:101DB000000044525900000000000053544F5000EE
:101DC0000000000052474200000000000048535647
:101DD0000000000000002B002D00455461673A20F0
:101DE0000047657420455441473A200048545450F8
:101DF0002F312E310025733A2025730D0A0020481B
:101E00005454502F312E310D0A486F73743A2025E7
:101E1000730D0A4163636570743A202A2F2A0D0AF4
:101E2000436F6E6E656374696F6E3A20636C6F7397
:101E3000650D0A0025730020000D0A004745540077
:101E40006661696C656420746F20636F6E6E656394
:101E5000740A004552524F523A20536572766572A9
:101E60002072657475726E65642000436F6E6669DA
:101E700067206E6F74206368616E6765640A004452
:101E80006F6E652E0A00436F6E666967207061721F
:101E900073696E67206661696C65640A00676F74B8
:101EA00020436F6E6669670A0068747470207265FB
:101EB00074636F64652000667265652000436F6E11
:101EC000666967205552493A20687474703A2F2F1A
:101ED000002044656661756C7420636F6E66696787
:101EE0002073657276657220757365643A20006CA4
:101EF000617A79686F6D652E7275000A282D294DFB
:101F0000455243555259000A282B294D554C5449E6
:101F100056454E54000A282B2950574D5F52454CC8
:101F20004159000A282B294D444E53000A282D29D7
:101F300055415254425249444745000A282B2953DF
:101F400059534C4F47000A282B29504944000A286E
:101F50002D294D43503233303137000A282D294185
:101F600052544E4554000A282D294F5441000A2846
:101F70002B29535049204C4544000A282B294D4F0A
:101F8000544F5220435452000A282B2941432048E1
:101F900041494552206F6E2053657269616C330070
:101FA0000A282B2943435338313120262048444303
:101FB00031303830000A282B2952455354415254AD
:101FC0005F4C414E5F4F4E5F4D5154545F455252EE
:101FD0004F5253000A282D29484152445245534537
:101FE000542C207573696E6720736F6674000A281D
:101FF0002B29434F554E544552000A282B2944485B
:1020000054000A282B294453323438322D313030D1
:10201000000A282B294F57495245000A282D2949E3
:10202000504D4F44425553000A282B294D4F4442EE
:1020300055532030783036206174205365726961C1
:102040006C322073706565643A39363030000A2886
:102050002B294144414652554954204C4544000ADD
:10206000282B29444D58000A282B2957697A6E6578
:102070007435313030000A282B294672656552616B
:102080006D207072696E74696E67000A282B29577B
:1020900041544348444F47006C617A79686F6D65DD
:1020A0002E7275000A436F6E6669672073657276DB
:1020B00065723A003230313130334C0020432B2BE3
:1020C0002076657273696F6E3A0034643930396412
:1020D000645F323032332D31312D3230000A4C61A1
:1020E0007A79686F6D652E7275204C6967687448DF
:1020F000756220636F6E74726F6C6C657220002065
:102100004F464600204F4E00204259504153530045
:10211000726561647900247374617465007570740C
:10212000696D650066726565686561700024737429
:10213000617473002054696D65723A00204C6F63BE
:102140006B733A002000204C6F636B733A000A52A5
:10215000414D3D0020457870697265640A00202D6C
:10216000746172676574207A6F6E652D0020416C12
:1021700061726D20457870697265640A0020636D34
:10218000643A00204375723A00205365743A005354
:102190006176656420746F20454550524F4D005361
:1021A0006176696E6720636F6E66696720746F2061
:1021B000454550524F4D2E2E004C6F616465642092
:1021C000455441473A004E6F2073746F7265642026
:1021D000636F6E666967004C6F6164656420667248
:1021E0006F6D20454550524F4D006C6F6164206605
:1021F00061696C6564004A534F4E20646574656381
:10220000746564004C6F6164696E6720436F6E662D
:1022100069672066726F6D20454550524F4D0043EF
:1022200043533831313A20416C72656164792069D9
:102230006E697469616C697A65640043435338312F
:10224000313A20496E6974206572726F72200043C2
:1022500043533831313A20496E6974004844433160
:102260003038303A20416C726561647920696E695A
:102270007469616C697A6564004465766963652098
:1022800053657269616C204E756D6265723D002008
:102290004465766963652049443D3078004D616E40
:1022A0007566616374757265722049443D307800CB
:1022B000484443313038303A20496E69742E20004A
:1022C000432C2052483D00484443313038303A20B6
:1022D0005374617475733D00484443313038303A6B
:1022E000204E6F7420696E697469616C697A6564E7
:1022F000004D7367496E76616C6964005265616474
:10230000526567496E76616C6964004D6561734D15
:102310006F6465496E76616C6964004D61785265E1
:1023200073697374616E63650048656174657246B4
:1023300061756C7400486561746572537570706C7A
:1023400079004343533831313A204572726F72201D
:10235000004343533831313A204661696C6564204B
:10236000746F20676574204552524F525F49442074
:1023700072656769737465722E005D2062617365B2
:102380006C696E655B005D2074564F435B002043B3
:102390004F325B006363733831313A20646174619A
:1023A000206E6F7420617661696C61626C65006398
:1023B0006373383131206E6F7420696E697469619E
:1023C0006C697A656400203C3C0041433A2000413E
:1023D000433A2053657269616C20757365642062AD
:1023E00079204143202D2064697361626C696E67B6
:1023F0002073657269616C206C6F6767696E672016
:10240000616E6420636D640041433A204F7574200F
:102410006F66206D656D6F72790041433A20496E99
:1024200069743A200041433A2044652D496E69742D
:102430003A20004552520041433A204F4B00203E83
:102440003E200041433A200041433A20506F6C6CDB
:10245000696E67000000000000000000004F4E00A1
:102460000000000000004F4646000000000000523F
:102470004553540000000000544F47474C450000AE
:102480000048414C540000000000584F4E0000002E
:10249000000000584F46460000000000494E4352DD
:1024A0004541534500444543524541534500454E3F
:1024B00041424C4500000044495341424C45000014
:1024C000554E465245455A4500465245455A4500E7
:1024D00000004155544F000000000046414E5F4F40
:1024E0004E4C59004849474800000000004D454403
:1024F00049554D0000004C4F5700000000000048B7
:102500004541540000000000434F4F4C00000000C4
:102510000044525900000000000053544F50000086
:1025200000000052474200000000000048535600DF
:1025300000000000007261770071756569740073B6
:1025400077696E67006C6F636B00556E6B6E6F77AB
:102550006E207375666669782000556E6B6E6F77B6
:102560006E20636D642000436F756E7465723A204F
:1025700000444D582D4F757420496E69743A2000FF
:10258000444D582D4F75742073746F703A2000417C
:10259000737369676E65643A00444D5820637472C2
:1025A0006C3A20006931360001693332000275311E
:1025B0003600037533320004693868000569386CE9
:1025C0000006753868000775386C000878313000EF
:1025D00009313030000A44656661756C742073659A
:1025E0007269616C206D6F6465204E38312075739F
:1025F000656400384531002600384E310006003849
:102600004532002E00384E32000E00384F31003671
:1026100000384F32003E0037453100240037453244
:10262000002C00374F31003400374F32003C003768
:102630004E31000400374E32000C004D4255533AE3
:10264000204D6F646275732074656D706C61746584
:10265000206E6F7420666F756E643A20004D42558F
:10266000533A20496E76616C69642074656D706CB4
:102670006174652E002C002C002C002C004D42555E
:10268000533A20636F6E666967206661696C6564A2
:102690003A004D4255533A20636F6E666967206574
:1026A00072726F72004D4255533A20636F6E6669C5
:1026B00067206C6F6164656420004D4255533A2079
:1026C0004F7574206F66206D656D6F7279004D4295
:1026D00055533A20506F6C6C696E67206572726F4B
:1026E0007220004D425553443A2049676E6F72651F
:1026F00064202D20657175616C2077697468207382
:1027000065747465642076616C004D4255533A20BF
:102710004164642040533A20004D425553443A20CE
:102720004D61707065643A004D425553443A204EF5
:1027300065737465644D61707065643A004C6173D3
:10274000744B6E6F776E2076616C75653A2000531E
:102750006561726368696E67207265673A2000720E
:10276000656723206F7574206F662072616E6765E0
:1027700000536561726368696E6720726567230044
:102780003A002066726F6D207479706520004D42AA
:102790005553443A2020676F7420002076616C3ACC
:1027A0000020005265733A200020696E7465726ED5
:1027B000616C2073656E64206572726F72202D20CB
:1027C0006E6F207265672F636F696C0020696E748D
:1027D00065726E616C2073656E64206572726F72D3
:1027E000202D206E6F2074656D706C617465002003
:1027F000696E7465726E616C2073656E64206572BB
:10280000726F72202D206E6F2073746F7265004D91
:10281000425553443A20656E64506F6C6C20004DF5
:10282000425553443A20506F6C6C2000206E6F74F8
:1028300020666F756E64004D4255533A20207061DA
:1028400072616D20002073656E64206572726F7214
:102850002E20004D4255533A202000416464204010
:10286000563A20002056616C3A20004D42555344A0
:102870003A207375666669783A00206F7220737526
:102880006666697820004D4255533A204E6F207499
:10289000656D706C61746520666F7220004D6F7499
:1028A0006F723A2074696D656F757400556E6B6E4A
:1028B0006F776E20636D64004D6F746F723A2046BF
:1028C0006F7263656420657865637574696F6E0007
:1028D0004D756C746956656E7420636F6E666967BA
:1028E000206661696C6564004D756C746956656E2F
:1028F0007420696E6974004D756C746976656E74C8
:102900002044652D496E697400204F75743A00208B
:102910006D33002066726F6D2000204D617820724B
:102920006571756573743A002066616E253A002002
:1029300061637469766520563A00546F74616C2047
:10294000563A005049443A20616C726561647920BE
:10295000696E697469616C697A6564005049443ACA
:1029600020496E76616C696420706172616D2061CE
:10297000727261792E002C002C002C002C00504922
:10298000443A20636F6E666967206661696C6564AE
:102990003A005049443A20636F6E66696720657259
:1029A000726F72005049443A20636F6E6669672007
:1029B0006C6F6164656420005049443A204F75741F
:1029C000206F66206D656D6F7279005049443A2022
:1029D00044652D496E69742000203C414C4D3E00F9
:1029E00020443A0020493A0020503A0020696E3ACB
:1029F00000207365743A005049443A20005049441D
:102A00003A20496E76616C696420706172616D2054
:102A100061727261792E00536574206F7574207431
:102A20006F20002050494420616C61726D2E20009F
:102A30002050494420616C61726D3A20636C6F7361
:102A40006564005049443A20556E6B6E6F776E2076
:102A500073756666697820005049443A20556E6B5C
:102A60006E6F776E20636D64200020536574706F05
:102A7000696E743A005049443A200020496E7075DE
:102A8000742076616C75653A005049443A20002004
:102A9000696E697400200050574D2D4F75742023C6
:102AA000002073746F7000200050574D2D4F7574C7
:102AB0002023003D0050696E3A0020696E69740061
:102AC00052656C61792D4F75742023002073746FEB
:102AD000700052656C61792D4F75742023003D3E66
:102AE000003A0070756220616374696F6E2000693E
:102AF000646C65006F66660068656174696E670086
:102B000066616E00647279696E6700636F6F6C69ED
:102B10006E670020697320004F75742000556E6B3E
:102B20006E6F776E207375666669782000556E6BE0
:102B30006E6F776E20636D642000616374696F6EE1
:102B40000072656C61794374723A200053686F7744
:102B50000020636D643D002D002072656164206576
:102B600072726F7220666F7220003E2000203C005F
:102B70003157543A003157543A206E6F7420696EC1
:102B80006974003157543A20425553592074696D85
:102B9000656F7574003157543A20445332343832DB
:102BA0005F4552524F525F434F4E4649470031579F
:102BB000543A20312D776972652073686F7274659D
:102BC00064005B305D3A2000202D202D202D20EF69
:102BD000BBBF003E003E31202D200000002200251A
:102BE0000028002B002E00310034000201000005F7
:102BF0000108010B0100000A0B02090C0D0E080769
:102C000003040100000000000000000000000000BC
:102C100000000000000000000000000000000000B4
:102C20000012111000000000000000000000000071
:102C3000000000000000000000000000002100244F
:102C40000027002A002D003000330001010000049D
:102C50000107010A0101021020200808102040107D
:102C60002040800201020108040201010204081050
:102C7000204080804020100804020180040201806E
:102C80004020100804020108040201010204081097
:102C9000204080010204081020408005050505073A
:102CA0000508080808020202020A0A0808040404C7
:102CB00004010101010101010103030303030303F3
:102CC00003040707070C0C0C0C0C0C0C0C02020282
:102CD0000206060606060606060B0B0B0B0B0B0B75
:102CE0000B556E7370656369666965642065727201
:102CF0006F722E0047454E455249435F4552524F31
:102D00005200494E5445524E414C5F4552524F522B
:102D1000004932435F4552524F520049445F455289
:102D2000524F520053554343455353004343533886
:102D300031313A200057726F6E67207061796C6193
:102D400064004354524C2F7478743A204F75744F7A
:102D5000664D656D6F72793A2000202D3E204154FA
:102D60003A004368616E20747970653A004E6F20B6
:102D700073746F7265642076616C756573202D20A5
:102D800064656661756C743A2000536176656420F1
:102D9000455441473A0053657420455441473A2011
:102DA000000000000000636D6400007365740000A3
:102DB00076616C000064656C000048535600005258
:102DC0004742000066616E00006D6F6465006374C9
:102DD000726C006875650000736174000074656D45
:102DE0007000726177000020002E00696E00735F32
:102DF0006F7574006D79686F6D65004354524C2F88
:102E0000657865633A204F75744F664D656D6F72D6
:102E1000793A2000202D3E2000456D69743A203C0F
:102E200000202D3E20004974656D436D643A2000FA
:102E3000202D3E20004974656D3A20003157543AE8
:102E400020427573207265736574206572726F72AB
:102E5000003157543A2042757320526573657420CF
:102E6000646F6E65003157543A204453323438321F
:102E70002070726573656E742C20726573657400C2
:102E800049324320526573657400005EBCE2613FC5
:102E9000DD83C29C7E20A3FD1F419DC3217FFCA238
:102EA000401E5F01E3BD3E6082DC237D9FC1421C6A
:102EB000FEA0E1BF5D0380DE3C62BEE0025CDF811C
:102EC000633D7C22C09E1D43A1FF4618FAA42779CA
:102ED0009BC584DA3866E5BB5907DB856739BAE4F8
:102EE00006581947A5FB7826C49A653BD987045A2A
:102EF000B8E6A7F91B45C6987A24F8A6441A99C7DC
:102F0000257B3A6486D85B05E7B98CD2306EEDB389
:102F1000510F4E10F2AC2F7193CD114FADF3702EB7
:102F2000CC92D38D6F31B2EC0E50AFF1134DCE90E9
:102F3000722C6D33D18F0C52B0EE326C8ED0530D9B
:102F4000EFB1F0AE4C1291CF2D73CA947628ABF549
:102F500017490856B4EA6937D58B5709EBB5366877
:102F60008AD495CB2977F4AA4816E9B7550B88D6A9
:102F7000346A2B7597C94A14F6A8742AC896154B5B
:102F8000A9F7B6E80A54D7896B35436F6E6E65634F
:102F90007465642E00436F6E6E2E2061626F7274D2
:102FA0006564003E3E2000496E76616C6964206372
:102FB0006F6D6D616E640000002000230026002903
:102FC000002C002F0032000001000003010601095F
:102FD000013E3E3E004E6F204D414320636F6E66C2
:102FE0006967757265643A20736574206669726DED
:102FF000776172652773204D41430A004545505261
:103000004F4D207369676E6174757265206F6B0038
:10301000496E697469616C697A696E6720454550CB
:10302000524F4D2E00003101F30111241FBECFEF8E
:10303000D1E2DEBFCDBF00E00CBF19E0A0E0B2E0FE
:10304000E0E1FEE802E00BBF02C007900D92A03F56
:10305000B107D9F721E1A0EFB9E001C01D92A03F6F
:10306000B207E1F718E1C4E1D8E100E006C021971A
:103070000109802FFE010F94CC3EC331D10780E0BF
:103080000807A9F70F94A2320D94F6460C9400009D
:103090008FE090E09093E4108093E31088EC90E050
:1030A0000895FC01848195810895DC011696ED91C7
:1030B000FC91309739F080858F70823019F48681C9
:1030C0009781089590E080E00895FC01A481B58186
:1030D000109721F118969C9118979F708EEF890F89
:1030E000823010F091111AC019964D935D936D9333
:1030F0007C931C97A481B58118969C911897907F1A
:10310000926018969C930480F581E02D8085982F1D
:10311000907F903619F48F70806A80870895FC0143
:10312000238130E090E080E0FC01EE0FFF1FE45DC2
:10313000F54FA081B181A217B30761F4880F991FE1
:10314000880F991FFC01E85EF54F4083518362832D
:1031500073830895A081B181AB2B19F42081318153
:10316000EDCF019685309105F9F60895FC01238194
:1031700030E090E080E0FC01EE0FFF1FE45DF54FD2
:10318000408151814217530761F4880F991F880FBE
:10319000991FFC01E85EF54F608171818281938106
:1031A000089540815181452B89F431832083880F14
:1031B000991F880F991FFC01E85EF54F108211825C
:1031C0001282138260E070E0CB0108950196853091
:1031D000910589F6F7CF880F991F880F991FFC0179
:1031E000E050F64F80819181A281B3810196A11DAB
:1031F000B11D80839183A283B383089585E090E01D
:103200000C94EB1884E090E00C94EB1883E090E0D1
:103210000C94EB1882E090E00C94EB1881E090E0C5
:103220000C94EB1890E080E00C94EB18CF93DF93B4
:10323000EC01E881F9810484F585E02D199529894F
:103240003A892F5F3F4F3A8B298BDF91CF910895B9
:10325000CF93DF93EC018E8581110DC081E090E06A
:1032600049895A892C853D854217530708F080E02B
:10327000DF91CF910895E881F9810484F585E02DEF
:10328000CE0119958F3F910549F780E090E0F0CF8E
:10329000FC01848595856817790708F4CB01928B2A
:1032A000818B0895DC011E962C911E97222339F004
:1032B000ED91FC910190F081E02D6FEF199408954C
:1032C000FC0187859089089581E0089590E080E071
:1032D0000895DC011296ED91FC91309761F0019018
:1032E000F081E02D309739F0862F8295807F6085C0
:1032F0006F70682B60870895DC011296ED91FC9148
:10330000309751F00190F081E02D309729F08085C1
:1033100082958F7090E0089590E080E008950F937B
:103320001F93CF93DF9300D000D01F921F92CDB791
:10333000DEB781E028960FB6F894DEBF0FBECDBF92
:10334000DF91CF911F910F910895089590E080E053
:10335000089566ED7DE1811102C068ED7DE186EFA3
:103360009EE00D94CC0B6DEE79E186EF9EE00F941C
:10337000CC0BF0E0E0E0199584EF91E008956CE566
:103380007CE0811102C067E57CE087EA9FE00D9454
:10339000CC0BDC0155962C915597273781F4ED9194
:1033A000FC91008CF18DE02D199563E079E087EABE
:1033B0009FE00F94CC0B87EA9FE00D94160A0895C6
:1033C000CF93DF93EB010297B4F16EEF7CE18A813A
:1033D0009B810F94F836892B29F40E941EDC6F77AD
:1033E0000E9478DC67E07DE18A819B810F94F8364A
:1033F000892B29F40E941EDC60680E9478DC6DEF46
:103400007BE186EF9EE00F94CC0B0E941EDC609562
:10341000661F6627661F70E04AE050E086EF9EE078
:103420000F941D0B86EF9EE00F94160A88EC90E037
:10343000DF91CF9108950E9401C8F8CF892B71F0D8
:10344000FB01828193810E9419DA65E77CE186EFB6
:103450009EE00F94CC0B88EC90E0089590E080E023
:10346000F2CF892B71F0FB01828193810E94B8D940
:103470006EE57CE186EF9EE00F94CC0B88EC90E04B
:10348000089590E080E0F2CFEF92FF920F931F93A8
:10349000CF93DF93CDB7DEB72C970FB6F894DEBF8E
:1034A0000FBECDBF8C017B018AE895E09A838983AA
:1034B0001B821C821D821E8298878F8319861A8622
:1034C0001B861C8605301105ECF0BE01695F7F4F3D
:1034D000F701808591850F946329892B99F0CE019E
:1034E00007960E94E3DABE01695F7F4FF70186818C
:1034F00097810F946329892B61F0CE0107960E9472
:10350000B5DB0EC0CE0101960E94E3DA043011054E
:1035100054F7CE0101960E94B5DB03301105A4F1EA
:10352000BE01695F7F4FF701848195810F94632904
:10353000892B51F1CE0107960E944CDBBE01695FD9
:103540007F4FF701828193810F946329892B19F1B1
:10355000CE0107960E947ADA67E37CE186EF9EE06F
:103560000F94CC0B80E00E94DCDC88EC90E02C9681
:103570000FB6F894DEBF0FBECDBFDF91CF911F9184
:103580000F91FF90EF900895CE0101960E944CDBC1
:10359000023011059CF6CE0101960E947ADA0130C4
:1035A0001105D1F6CE0101960E947ADA6EE37CE134
:1035B00086EF9EE00F94CC0BCFCFCF93C1E068EEA7
:1035C00073E080E090E00E948CE84AE050E06C2FCD
:1035D00086EF9EE00F94330ACF5FC43181F784EF0A
:1035E00091E0CF9108950F931F93CF93DF938C01B8
:1035F000EB010297C4F08A819B810F94AA368093D5
:10360000450299270E94E5DC0230110549F08C81C2
:103610009D810F94AA368093440299270E94EFDC83
:10362000C8ECD0E002C0C0E9D1E063E27CE186EF03
:103630009EE00F94CC0B4AE050E06091450286EF8B
:103640009EE00F94330A6EE07CE186EF9EE00F94DB
:10365000CC0B4AE050E06091440286EF9EE00F946C
:10366000330A86EF9EE00F94160ACE01DF91CF91C8
:103670001F910F910895DC011296ED91FC91309706
:1036800071F090859F70923039F0953041F4CF0100
:103690000E9429D990E0089581E090E0089590E09B
:1036A00080E00895009789F0FC0120852F70253077
:1036B00061F40E9497D8009741F0FC0120852F709B
:1036C000243019F481859285089590E080E0089572
:1036D00065E0FC01808191810E9497D8009749F0B4
:1036E000FC018085982F907F21F082958F7090E06B
:1036F000089590E080E00895CF93C62F63E0FC0129
:10370000808191810E9497D8FC01892B21F19085BD
:10371000892F8D7001F5907F9260908781859285C9
:10372000A385B4858827BB278C2B81879287A387A5
:10373000B4876DEA79E087EA9FE00F94CC0B4AE00A
:1037400050E06C2F87EA9FE00F94330A87EA9FE0EE
:10375000CF910D94160ACF9108958F929F92AF92B8
:10376000BF92CF92DF92EF92FF920F931F93CF936E
:10377000DF93E091E510F091E610309709F467C00F
:10378000812EF02E932EC22EA52ED42EB72EE62EED
:10379000BC01CF010E94E5D7EC01892B19F481E02F
:1037A00090E057C088858F708530C9F760E0CE0102
:1037B0000E9497D88C0161E0CE010E9497D8FC014D
:1037C000C185D285D80119962D913C9121303105C2
:1037D00061F13CF46F2DCE01232B09F70F945A228F
:1037E000DECF2230310531F127303105C1F6892B8A
:1037F000B1F280858F70853091F6C681D781209790
:1038000071F288858F70843061F40F2D182D2C2D66
:10381000392D4D2D5A2D6E2D7B2D89859A850E942F
:10382000AD1B0A80DB81C02DEACF6F2DCE01039640
:103830000F945A226E2DCE010F945A226D2DCE0177
:1038400001960F945A226C2DCE010296C7CF90E0BC
:1038500080E0DF91CF911F910F91FF90EF90DF906B
:10386000CF90BF90AF909F908F9008952F923F92EE
:103870004F925F926F927F928F929F92AF92BF9280
:10388000CF92DF92EF92FF920F931F93CF93DF932C
:103890008091A70A9091A80A892B09F49AC02090D8
:1038A000A60A312C3594279435942794EE24E3947A
:1038B000F12CD0E0C0E088248394912C2C163D0696
:1038C00009F487C0C090A70AD090A80A24010C2E42
:1038D00002C0440C551C0A94E2F7052C000C660843
:1038E0007708F7013197EC0DFD1D5701A4E0AA0EF2
:1038F000B11CC70160E02091420230914302AC014B
:103900002817390720F44091420250914302209138
:10391000DD103091DE10240F351FD9012C9131912B
:103920003217C1F04091F7095091F8096091F909F7
:103930007091FA0944295529662977294093F70996
:103940005093F8096093F9097093FA09DF01119710
:103950002C9361E001968A159B0569F66623B1F107
:103960008091A90A9091AA0A009729F1FC0120856B
:103970002F70253001F56C2F0E9497D8FC0190859F
:103980009F709430C1F4818592850097A1F0FE016B
:10399000EE0FFF1FEE0FFF1FEC0DFD1D038110E06A
:1039A000228130E0EC0CFD1CD7014C9150E060818D
:1039B00070E00E94AD1B80E00F945B286093FB09D0
:1039C0007093FC098093FD099093FE09219675017F
:1039D00075CFDF91CF911F910F91FF90EF90DF9006
:1039E000CF90BF90AF909F908F907F906F905F909F
:1039F0004F903F902F9008950F931F93CF93DF9395
:103A0000CDB7DEB769970FB6F894DEBF0FBECDBF56
:103A1000E091CA10F091CB10309709F460C080910A
:103A2000E7109091E810892B09F459C08FEF838734
:103A300014861382148215821682178210861186CC
:103A400012866EE07AE186EF9EE00F94CC0B86EF53
:103A50009EE00F94160ABE016E5E7F4F8091CA10E1
:103A60009091CB100F94B4261816CCF5A895AE0102
:103A70004F5F5F4F68E0CE0142960F94B827198AD6
:103A8000BE016F5F7F4F8091E7109091E8100E9418
:103A9000E5D78C0169E07AE186EF9EE00F94CC0BCC
:103AA000BE016F5F7F4F86EF9EE00F94660B01159E
:103AB000110591F0C8010E94D7C48C01892B59F2DD
:103AC00064E07AE186EF9EE00F94CC0BB80186EFBC
:103AD0009EE00F94660BBBCF6FEF79E1B4CF88EC1B
:103AE00090E069960FB6F894DEBF0FBECDBFDF91B0
:103AF000CF911F910F9108950F931F93CF93DF9351
:103B000000D000D0CDB7DEB70E94E7CC69E577E101
:103B100086EF9EE00F94CC0BCE0101960E94D7E376
:103B2000CE0101960F940D290AE815E01A83098346
:103B30008091F60C9091F70CA091F80CB091F90CD3
:103B40008B839C83AD83BE83CE0101960F940D2998
:103B50001A8309831B821C821D821E8280E590E0ED
:103B60000E94D4E344E050E0BE016D5F7F4F81E0EE
:103B700090E00F94D8130F94CF14CE0101960F94B8
:103B80000D291A8309831B821C821D821E8280E5F7
:103B900090E00E94D4E344E050E0BE016D5F7F4FAF
:103BA00085E090E00F94D8130F94CF14CE010196C6
:103BB0000F940D296FE777E186EF9EE00F94CC0B11
:103BC00088EC90E026960FB6F894DEBF0FBECDBF0E
:103BD000DF91CF911F910F9108950D9479350D9438
:103BE0007935CF92DF92EF92FF920F931F93CF938D
:103BF000DF9300D000D0CDB7DEB78091BA0A811133
:103C00009CC08091E3109091E41002970CF495C051
:103C10008091B10A9091B20A009709F48EC06FEBBF
:103C200075E00E94E5D78C01009709F486C00E94D8
:103C300029D9E82EF12CE114F10409F47EC070E0DA
:103C400060E0C8010E94521B6C01EA94EF2809F45D
:103C500083C061E0C8010E9497D8FC0101851285EC
:103C6000CE0101960E94D7E3CE0101960E94F5E3B2
:103C70006EE373E186EF9EE00F94CC0BB60186EF06
:103C80009EE00F94660B61E179E086EF9EE00F9471
:103C9000660B4AE050E0B80186EF9EE00F941D0BE2
:103CA00061E179E086EF9EE00F94660B67E47BE0CC
:103CB00086EF9EE00F94660B86EF9EE00F94160A47
:103CC00062E072E085EC9FE00F942219D092BB0F66
:103CD000C092BA0F1093BD0F0093BC0F87E49BE016
:103CE000892BE9F58DEB95E09093BF0F8093BE0F84
:103CF0008091AB0A9091AC0A009741F070E060E0CF
:103D00000E94521B9093C6108093C5108091C510DD
:103D10009091C610009731F19093C10F8093C00F1E
:103D20001092C30F1092C20F81E08093BA0A65E22D
:103D300073E186EF9EE00F94CC0B26960FB6F894B5
:103D4000DEBF0FBECDBFDF91CF911F910F91FF90CE
:103D5000EF90DF90CF90089502E012E081CF87E4EA
:103D60009BE0C2CF87E594E0D7CFEF92FF920F930D
:103D70001F93CF93DF930097C1F0FC012081222392
:103D8000A1F08C0181E2E82E8EE0F82EC1E0D0E0B7
:103D9000B701C8010F941637892B49F02196F5E039
:103DA000EF0EF11CCE30D10599F7D0E0C0E0CE0186
:103DB000DF91CF911F910F91FF90EF900895CF92D7
:103DC000DF92EF92FF920F931F93CF93DF93CDB7C4
:103DD000DEB7C154D1090FB6F894DEBF0FBECDBF18
:103DE0006C01AB0130E020E060E4CE0101967C0183
:103DF0000F947928F70101900020E9F731978F019E
:103E00000E191F09A801B701C6010F945943892B48
:103E100011F010E000E0C801CF5BDF4F0FB6F8945F
:103E2000DEBF0FBECDBFDF91CF911F910F91FF90ED
:103E3000EF90DF90CF900895CF92DF92EF92FF92B4
:103E40000F931F93CF93DF93CDB7DEB7C054D10943
:103E50000FB6F894DEBF0FBECDBF8091E3109091F6
:103E6000E410059709F449C06115710509F445C0CE
:103E700069017A018B0140E450E0CE0101960F9474
:103E800067436FE270E0CE0101960F942E43892BB9
:103E900041F4980143E050E060E4CE0101960F94B4
:103EA00079284FE350E0B601CE0101960F944943C3
:103EB0000E9403D8882309F18091E3109091E410C7
:103EC0000697D9F48091C910811117C0B701CE01AE
:103ED00001960E941BEB81E090E0C05CDF4F0FB6C3
:103EE000F894DEBF0FBECDBFDF91CF911F910F9130
:103EF000FF90EF90DF90CF90089590E080E0EDCFBD
:103F0000CF92DF92EF92FF920F931F93CF93DF93A5
:103F1000CDB7DEB760970FB6F894DEBF0FBECDBF4A
:103F20007C016B01CA01B9012AE0AE014F5F5F4F0E
:103F30000F94BA37D701ED91FC910288F389E02DF7
:103F40009801AE014F5F5F4FB601C70119956096AA
:103F50000FB6F894DEBF0FBECDBFDF91CF911F919A
:103F60000F91FF90EF90DF90CF900895CF92DF9266
:103F7000EF92FF920F931F93CF93DF93CDB7DEB7EE
:103F800060970FB6F894DEBF0FBECDBF7C016B010A
:103F9000BA01A901CE0101960F94A129D701ED9193
:103FA000FC910288F389E02D9801AE014F5F5F4FCD
:103FB000B601C701199560960FB6F894DEBF0FBE23
:103FC000CDBFDF91CF911F910F91FF90EF90DF90C8
:103FD000CF9008951F93CF93DF93FC01162FC389D1
:103FE000D489818992899C012F5F3F4F328B218B2D
:103FF000C80FD91FCE010F942F3E181721F0612F43
:10400000CE010F94373E81E090E0DF91CF911F9178
:104010000895FC018189928924853585821793074B
:1040200040F423893489820F931F0F942F3E90E030
:1040300008958FEF9FEF0895CF93DF9300D000D0C6
:104040001F921F92CDB7DEB7FC01862F8F70618162
:10405000607F682B618388E0DE01119601900D92EC
:104060008A95E1F729813A814B815C816D817E815E
:104070008F81988528960FB6F894DEBF0FBECDBF0E
:10408000DF91CF910895CF93DF9300D000D01F929E
:104090001F92CDB7DEB7FC01608398E0DE01119678
:1040A00001900D929A95E1F729813A814B815C81CB
:1040B0006D817E818F81988528960FB6F894DEBF3A
:1040C0000FBECDBFDF91CF9108956F927F928F92F7
:1040D0009F92AF92BF92CF92DF92EF92FF920F9397
:1040E0001F93CF93DF93CDB7DEB7A0970FB6F894A9
:1040F000DEBF0FBECDBF8C01862E7A01DC018D9113
:104100009C911197892B09F466C01496ED91FC914E
:10411000309709F460C080818071BFEF6B135DC080
:10412000B1F481E0A0960FB6F894DEBF0FBECDBF0C
:10413000DF91CF911F910F91FF90EF90DF90CF9083
:10414000BF90AF909F908F907F906F900895433075
:10415000510539F3818082942FE0822263EA79E06D
:1041600087EA9FE00F94CC0B4AE050E0D801139609
:104170006C9187EA9FE00F94330A61EA79E087EA5D
:104180009FE00F94CC0BD8011496ED91FC916181C6
:104190006F704AE050E087EA9FE00F94330A6EE9BF
:1041A00079E087EA9FE00F94CC0B4AE050E0682D5D
:1041B00087EA9FE00F94330A87EA9FE00F94160A7C
:1041C000D8011496ED91FC9181818F70881207C0FF
:1041D00080818F7E808380E0A5CF8111FCCF198EF6
:1041E0001A8E1B8E1C8E1D8E1E8E1F8E18A28A8DFF
:1041F0008F708A8FD8011496ED91FC9181818F7018
:104200008815A9F1B3E0EB16F10489F16CE979E0C6
:1042100087EA9FE00F94CC0B4AE050E0F8016381FD
:1042200087EA9FE00F94330A6AE979E087EA9FE022
:104230000F94CC0BD8011496ED91FC9161816F70B5
:104240004AE050E087EA9FE00F94330A67E979E09B
:1042500087EA9FE00F94CC0B4AE050E0682D87EA94
:104260009FE00F94330A87EA9FE00F94160AF80143
:1042700020813181FCE0F81508F416C1E82DF0E04A
:104280008827EA5BFE4D8F4F0D94CC3E5321902141
:104290001122282234221122EA211122372242221D
:1042A000FE2145225122D8011496CD90DC90F601D2
:1042B00081818F70853009F4F7C050F48230C1F0ED
:1042C00064ED75E0C9010E94E5D73C01912C4BC01B
:1042D0008730D1F08A30A1F76DEC75E0C9010E94FA
:1042E000E5D73C01D6019C9092FA992490F83BC006
:1042F00067EC75E0C9010E94E5D73C01D6019C90AE
:1043000090FA992490F82FC066EC75E0C9010E94DC
:10431000E5D73C01F601908091FA992490F823C0EA
:1043200069ED75E0C9010E94E5D73C01D8011496FA
:10433000ED91FC91808180FB992490F8982F9E7FCD
:1043400080FF916090836114710469F461E0CE0193
:1043500049960E944320298B3A8B4B8B5C8B6D8B4B
:104360007E8B8F8B988FF801A080B1806FE076E014
:10437000C5010E94E5D76C0164E176E0C5010E94A9
:10438000E5D75C01892B81F4C114D10469F460E0A4
:10439000CE0149960E94432029833A834B835C8354
:1043A0006D837E838F839887D8011496ED91FC915D
:1043B0006114710409F07CC0898D811179C0B82D18
:1043C000BF708B2E8181807F882A818280818F7E41
:1043D0008083A7CE6EED75E0C9010E94E5D73C0150
:1043E000D8011496ED91FC91808181FB992490F87D
:1043F000982F9D7F81FF92609083B5CF64EE75E02A
:10440000C9010E94E5D73C01D8011496ED91FC91B9
:10441000808182FB992490F8982F9B7F82FF946083
:10442000EBCF64ED75E0C9010E94E5D73C01892B13
:1044300009F04CCF62E0CE0149960E9443202987C3
:104440003A874B875C876D877E878F87988B3ECFB7
:104450006AEE75E0C9010E94E5D73C01D8011496C7
:10446000ED91FC9190804CCF6FEE75E0F3CF65EF4E
:1044700075E0C9010E94E5D73C01D8011496ED9181
:10448000FC9149CF6BEF75E0F4CF62E076E0C901B3
:104490000E94E5D73C01D8011496ED91FC919080E3
:1044A00023CF68E076E0F3CF912C712C612C5BCFA9
:1044B00083E0E816F104B9F0982D9F70892E818170
:1044C000807F882A818280818F7E8083E98CFA8C2C
:1044D0000B8D1C8D2D8D3E8D4F8D58A1692DC301E7
:1044E0000F94C02B1ECE81818F70881509F419CED0
:1044F000829490EF8922882A81828081806168CFAE
:10450000CF93DF9300D000D01F921F92CDB7DEB7BC
:10451000FC0191819F70906B9183448355836683E6
:10452000778388E0DE01119601900D928A95E1F77C
:1045300029813A814B815C816D817E818F81988553
:1045400028960FB6F894DEBF0FBECDBFDF91CF9196
:104550000895CF93DF9300D000D01F921F92CDB764
:10456000DEB7FC0191819F70906A918344835583EB
:104570006683778388E0DE01119601900D928A951B
:10458000E1F729813A814B815C816D817E818F8148
:10459000988528960FB6F894DEBF0FBECDBFDF9189
:1045A000CF910895CF93DF9300D000D01F921F9238
:1045B000CDB7DEB7FC016F3F710519F014F06FEF56
:1045C00070E077FD60E09181892F82958F70815036
:1045D0008230C8F4648388E0DE01119601900D9268
:1045E0008A95E1F729813A814B815C816D817E81D9
:1045F0008F81988528960FB6F894DEBF0FBECDBF89
:10460000DF91CF9108959F7090619183E3CFCF9315
:10461000DF93CDB7DEB760970FB6F894DEBF0FBE5D
:10462000CDBF19821A821B821C821D821E821F82AC
:1046300018868A818F708A836FEF70E0CE010196B1
:104640000E94D22260960FB6F894DEBF0FBECDBF97
:10465000DF91CF910895CF92DF92EF92FF92DC012C
:10466000362F1196EC911197E295EF70EC3008F02F
:10467000B6C0F0E08827E05CFC4D8F4F0D94CC3E37
:10468000F22378237823EF23EF23EF23BD237F2327
:10469000EF23EF234C234C2314968D919D910D9085
:1046A000BC91A02D662399F0B7FD9FC08F3F910567
:1046B000A105B10529F024F08FEF90E0A0E0B0E073
:1046C0002FEF30E0A901481B590BCA010CC0B7FD00
:1046D00089C08F3F9105A105B10529F024F08FEF26
:1046E00090E0A0E0B0E0FF90EF90DF90CF900895D1
:1046F00014962C91822F90E06623A9F3E1CF1496B3
:10470000CD90DD90ED90FC901797662301F120E0AD
:1047100030E0A901C701B6010F940B3D87FD65C0CC
:1047200020E030E04FE753E4C701B6010F94134097
:1047300018160CF457C0A701960160E070E08FE7EF
:1047400093E40F94FE3E0F94DD3FCB01CCCF20E0ED
:1047500030E0A901C701B6010F940B3D87FD42C0AF
:1047600020E030E04FE753E4C701B6010F94134057
:104770001816DCF1C701B601E6CF14966D917D9154
:104780008D919C9117973323B1F06D395FEF7507C9
:104790008507950754F1611524E672078105910597
:1047A0000CF52CE93FEF4FEF5FEF0F94773EC90117
:1047B00081509F4F98CF6D394FEF7407840794074E
:1047C0008CF0611554E675078105910574F424E6B3
:1047D00030E040E050E00F94773EC90184CF8FEF86
:1047E0009FEF81CF90E080E07ECF8FEF90E07BCF96
:1047F000CF93DF93EC01DB01898182958F70863046
:10480000E1F128F481508230C8F080E014C0873094
:1048100009F18A508230C8F72FEF30E00F94E33E61
:1048200024E630E040E050E00F94773E2C833D8357
:104830004E835F8381E0DF91CF9108952FEF30E0C9
:104840000F94E33E24E630E040E050E00F94773EE2
:104850002C83F0CF2FEF30E00F94E33E24E630E0DE
:1048600040E050E00F94773ECA01B9010F94123D29
:104870006C837D838E839F83DDCF2CE933E60F9499
:10488000E33E24E630E040E050E00F94773E2C8396
:104890003D834E835F83B9CFDC011196EC91119774
:1048A000E295EF70E150EB3008F039C0F0E0882776
:1048B000E35AFB4D8F4F0D94CC3E802480248F24EF
:1048C000682468247124882488248824682468241F
:1048D00014966D917D918D919C9117970F94123D37
:1048E000089514966D917D918D919C91179724E672
:1048F00030E040E050E00F94773ECA01B901EECFBE
:1049000014966C9170E090E080E00F94103D089553
:1049100014966D917D918D919C911797089560E00B
:1049200070E0CB010895DC011196EC911197E295AE
:10493000EF70E150EB3008F037C0F0E08827EC551D
:10494000FB4D8F4F0D94CC3EB624B624D424AF2417
:10495000AF24C524BC24BC24BC24AF24AF241496AB
:104960006D917D918D919C911797089514966C91FE
:1049700070E090E080E0089514966D917D918D91A6
:104980009C9117970F94DD3F089514966D917D913A
:104990008D919C91179724E630E040E050E00F9411
:1049A000773ECA01B901089560E070E0CB01089537
:1049B0008F929F92AF92BF92CF92DF92EF920F931E
:1049C0001F93CF93DF9300D000D01F921F92CDB7DB
:1049D000DEB7FC0109831A832B833C834D835E83FE
:1049E0006F837887808191810097A1F490E080E0C7
:1049F00028960FB6F894DEBF0FBECDBFDF91CF91E2
:104A00001F910F91EF90DF90CF90BF90AF909F904C
:104A10008F9008958F010E9429D9C82ED12C86E04D
:104A2000C816D10464F40E94E0DDBC01F801808165
:104A300091810E94EDDDFFEFCF1ADF0AF0CF65E034
:104A4000F801808191810E9497D88C01892B71F2A5
:104A50008981803158F6CE0101960E949324161662
:104A600017061806190644F4F8018085982F9D70E2
:104A7000A1F08F70873089F0F80180858F70808772
:104A800061EF79E087EA9FE00F94CC0B87EA9FE023
:104A90000F94160A81E090E0ABCF0E947EEA4B01B2
:104AA0005C01CE0101960E949324860E971EA81EDB
:104AB000B91EF80181869286A386B48682E0E11051
:104AC00087E099819295907F892BF801808766EE27
:104AD00079E087EA9FE00F94CC0BCE0101960E940B
:104AE0009324AB01BC012AE030E087EA9FE00F94F9
:104AF000D50A60EE79E087EA9FE00F94CC0BF801CD
:104B000041855285638574852AE030E087EA9FE01D
:104B10000F94D50ABBCFDC011196EC911197E29569
:104B2000EF70E150EB3008F03EC0F0E08827E4562B
:104B3000FA4D8F4F0D94CC3EB225B225D325A72533
:104B4000A725CC25BD25BD25BD25A725A7251496C0
:104B50002D913D914D915C911797A4E6B0E00F9493
:104B6000963E089514966C9184E6689FB0011124D6
:104B7000072E000C880B990B089520E030E048ECDC
:104B800052E414966D917D918D919C9117970F949D
:104B9000713D0F94DD3F089514966D917D918D9137
:104BA0009C911797089560E070E0CB010895FC0197
:104BB000A7812A2F2E7FD1F0818182958F7081501D
:104BC0008330A0F4A695A150BB0B2BE531E00F94E8
:104BD000E33E24E630E040E050E00F94773EDA0117
:104BE000C90187569F4FAF4FBF4F08958FEF9FEF7B
:104BF00008952F923F924F925F926F927F928F9281
:104C00009F92AF92BF92CF92DF92EF92FF920F935B
:104C1000CF93DF9300D01F92CDB7DEB77C017A83AC
:104C200069835C834B83DB011C92FC0160816623FA
:104C300009F44EC030FF4CC0F9E06F9FB001112461
:104C40006C5B7E4ECD010F944D37D70111968C9140
:104C5000807F41F04B815C816BE678E089819A81AD
:104C60000F944943E981FA8101900020E9F73197D7
:104C700029813A81E21BF30B19012E0E3F1E4B8155
:104C80005C814E1B5F0B415051095C834B83D70104
:104C90001196EC9111978E2F807F09F4F7C0E29561
:104CA000EF70E150EC3008F0F1C0F0E08827E45AF2
:104CB000F94D8F4F0D94CC3E6B260E277B27DA27BC
:104CC000F527B9268B278B278B27A7268F26112818
:104CD00029803A80DCCFF7018481282F30E050E032
:104CE00040E0002359F030E0A4E6B0E00F94A93E84
:104CF0002FEF30E040E050E00F94773E5F934F930A
:104D00003F932F9389E196E09F938F93FC81FF93CC
:104D10002B812F933F922F920F948143B2C017960D
:104D20008C9117978F9316968C9116978F93159653
:104D30008C9115978F9314968C918F938CE196E0BC
:104D40009F938F93BC81BF93EB81EF93E3CF179633
:104D50008C9117978F9316968C9116978F93159623
:104D60008C9115978F9314968C918F9380E296E097
:104D7000E7CF1496CD90DD90ED90FC901797F7FE5D
:104D800034C084E6882E912CA12CB12CC701B60129
:104D9000A50194010F94773E9B01AC0188279927C8
:104DA000DC01821B930BA40BB50BBF93AF939F93B6
:104DB0008F9366277727CB016C197D098E099F0990
:104DC000A50194010F94773E5F934F933F932F93E8
:104DD00084E296E09F938F933C813F934B814F9366
:104DE0003F922F920F9481434CC0C701B60124E635
:104DF00030E040E050E00F94773E9F938F937F9395
:104E00006F935F934F933F932F9385E296E09F9329
:104E10008F939C819F93AB81AF93E2CFC7010E9498
:104E2000D725BC01D7011696CC9016971796DC9023
:104E30001797D0FADD24D0F814969C911497159604
:104E4000FC90EB80BC80292F30E050E040E077FD03
:104E500035C0011135C07F936F931F921F921F922F
:104E60009F931F92FF92DF92CF928EE296E09F93E4
:104E70008F93FC81FF932B812F933F922F920F945E
:104E800081430FB6F894DEBF0FBECDBF89819A81F2
:104E90000F900F900F900F90DF91CF910F91FF9097
:104EA000EF90DF90CF90BF90AF909F908F907F90CA
:104EB0006F905F904F903F902F900895002361F086
:104EC000292F30E0A4E6B0E00F94A93E2FEF30E0A8
:104ED00040E050E00F94773E5F934F933F932F93C2
:104EE0001F92FF92DF92CF9281E396E09F938F9380
:104EF000BF92EF9275CF15968C9115971F928F9355
:104F000016969C91169717968C9181708F939F930C
:104F100084E396E015CF14968D909D90AD90BC9053
:104F2000179720E030E0A901C501B4010F940B3DB3
:104F30002401350187FF04C077FA709477F87094E4
:104F4000C301B2010F94DD3F6B01072E000C880BEB
:104F5000990B0F94123D9B01AC01C301B2010F9458
:104F6000FE3E20E030E04AE754E40F94713D0F9498
:104F700068400F94DD3F062F772E20E030E0A90136
:104F8000C501B4010F940B3D87FF07C07F920F93BB
:104F9000DF92CF928AE396E0D3CE7F920F93DF9297
:104FA000CF928BE396E09F938F933C813F934B810D
:104FB0004F93B0CE14968C9114971F928F931596A1
:104FC0008C9115971F928F9316968C911F928F93A9
:104FD00081E396E09F938F93BC81BF93EB81EF9326
:104FE0003F922F920F9481434CCF17968C91179735
:104FF0001F928F9314968C9114971F928F931596EE
:105000008C9115971F928F9316968C911F928F9368
:105010008EE296E09F938F93BC81BF93EB81EF93D9
:10502000DFCE14966D917C914B815C81C1010F9410
:1050300067432CCFEF92FF920F93CF93DF93CDB7BF
:10504000DEB7A0970FB6F894DEBF0FBECDBF7C01D0
:1050500000E020E033E040E250E0BE016F5F7F4FB0
:105060000E94F925BE016F5F7F4F87EA9FE00F9492
:10507000660B6CE272E187EA9FE00F94CC0BF701BC
:10508000618162956F704AE050E087EA9FE00F947B
:10509000330A65E272E187EA9FE00F94CC0BF701D7
:1050A00061816F704AE050E087EA9FE00F94330A15
:1050B00087EA9FE00F94160AA0960FB6F894DEBF19
:1050C0000FBECDBFDF91CF910F91FF90EF9008956C
:1050D000CF93DF93EC016115710539F48F818170F5
:1050E0008F8381E0DF91CF9108958981982F9295E8
:1050F0009F7029F180E09430A8F79B01770F440B53
:10510000550B2959310941095109A4E6B0E00F9422
:10511000963E2BE531E040E050E00F94773E37FFBC
:1051200002C030E020E02536310514F024E630E0FE
:105130002F5F220F8F818170282B2F83D2CF8F700A
:1051400080628983DACFFC019181892F82958F70EB
:1051500021F0823029F080E008959F709062918361
:105160009B0177FF02C030E020E02E3681E0380757
:1051700014F02DE631E02683878130FB80F98783A8
:1051800081E00895EF92FF920F931F93CF93DF93E7
:10519000FC01892B69F19081992351F19D3291F1A4
:1051A00080ED890F8A3070F1C8E0D0E0953211F1BE
:1051B000CEEFDFEF9B37F1F0C7E1D0E09332D1F0D3
:1051C0008F018DE4E82E81E1F82EC1E0D0E0C70127
:1051D0000F942637AC01B701C8010F943F37892BD4
:1051E00049F0219689E0E80EF11CC931D10579F723
:1051F000CFEFDFEFCE01DF91CF911F910F91FF90A5
:10520000EF900895D0E0C0E0F5CFEF92FF920F93BA
:105210001F93CF93DF93EC01892B51F188858F7019
:10522000843009F5E984FA84C7010E94C2288C0100
:1052300018161906ECF4C7010F946D10C801012E61
:10524000000CAA0BBB0B89879A87AB87BC87888524
:10525000807F82608887C801DF91CF911F910F9175
:10526000FF90EF900895823019F409851A85F3CFE5
:1052700010E000E0F0CF2F923F924F925F926F923A
:105280007F928F929F92AF92BF92CF92DF92EF92D6
:10529000FF920F931F93CF93DF93CDB7DEB76C9739
:1052A0000FB6F894DEBF0FBECDBF6115710549F58D
:1052B00028E0FC01DE01119601900D922A95E1F79C
:1052C00029813A814B815C816D817E818F819885B6
:1052D0006C960FB6F894DEBF0FBECDBFDF91CF91B5
:1052E0001F910F91FF90EF90DF90CF90BF90AF9004
:1052F0009F908F907F906F905F904F903F902F90F6
:1053000008956B018C016AEB78E0C6010E94E5D735
:10531000FC01892B09F40EC180858F70843009F45B
:1053200052C0853009F006C1E680F780E114F1042F
:1053300009F400C1F70180858F70823011F4E2809A
:10534000F380E114F10409F4F5C0F70180858F7052
:10535000853011F0F701F3CFC7010E9429D98230BF
:10536000C9F760E0C7010E9497D85C010E94052937
:1053700061E0C7010E9497D84C01FC0180858F70C5
:10538000823041F7C8010E949324F4014184528481
:10539000638474846415750586059705D9F6A11490
:1053A000B10409F4C7C019821A821B821C821D82B3
:1053B0001E821F8218868A818F708A83F50161851B
:1053C000CE0101964EC06EEC77E0818592850F94F8
:1053D0003943892B09F0AEC0C8010E94932461159E
:1053E00071058105910509F48BC0660F771F881F31
:1053F000991F2FEF30E040E050E00F94773E57FDCB
:1054000015C023303105410551050CF05FC0DA01AC
:10541000C9010196A11DB11D82309105A105B105FB
:10542000D9F10397A105B10509F450C019821A8278
:105430001B821C821D821E821F8218868A818F70A9
:105440008A8367E0CE0101960E941C2029873A8753
:105450004B875C876D877E878F87988B62E1CE0153
:1054600009960E944320298B3A8B4B8B5C8B6D8B6A
:105470007E8B8F8B988F49895A896B897C898D891E
:105480009E89AF89B88D49835A836B837C838D83D2
:105490009E83AF83B88714CF19821A821B821C8225
:1054A0001D821E821F8218868A818F708A8367E020
:1054B000CE0101960E941C2029873A874B875C8782
:1054C0006D877E878F87988B61E1C9CF19821A8299
:1054D0001B821C821D821E821F8218868A818F7009
:1054E0008A8367E0CE0101960E941C2029873A87B3
:1054F0004B875C876D877E878F87988B60E1AFCF06
:1055000019821A821B821C821D821E821F821886AB
:105510008A818F708A8367E0CE0101960E941C20E9
:1055200029873A874B875C876D877E878F87988B23
:1055300062E095CF63E476E0C6010E94E5D75C01A6
:10554000009709F4C5C0FC0180858F70853009F093
:10555000AEC0C5010E9429D9843009F0B9C060E00D
:10556000C5010E9497D84C0161E0C5010E9497D8FF
:105570003C0162E0C5010E9497D8FC01C184D2843D
:10558000E384F48463E0C5010E9497D85C01C801FC
:105590000E9493246C157D058E059F059CF419824D
:1055A0001A821B821C821D821E821F8218868A819B
:1055B0008F708A8340E050E0BA01CE0101960E94CC
:1055C000802251CFF4010184F285E02DFA8FE98F1A
:1055D000F30121843284F5010184F285E02DFC8FF2
:1055E000EB8F19821A821B821C821D821E821F82EF
:1055F00018868A818F708A83298D3A8D4901330FED
:10560000AA08BB0826010D2C000C66087708C80103
:105610000E9493249B01AC012419350946095709BE
:10562000B101032C000C880B990B681979098A09C0
:105630009B090F94453EEB8DFC8D9F01FF0F440BA2
:10564000550B24193509460957090F94773E820EE8
:10565000931EA41EB51EC101298D3A8D821B930B8A
:105660006B8D7C8D6C197D090F94B83E77FF02C05D
:105670006F5F7F4F75956795CB01770FAA0BBB0BBB
:10568000880E991EAA1EBB1EB7FC0CC0A401B50152
:105690003FEF83169104A104B10409F00CF48DCFFF
:1056A0004FEF01C040E050E060E070E086CF811134
:1056B0000FC019821A821B821C828A818F708A8392
:1056C00049815A816B817C8180E090E0DC01DBCEF6
:1056D000F801408151816281738184819581A68125
:1056E000B781D1CE4F925F926F927F928F929F92AD
:1056F000AF92BF92CF92DF92EF92FF920F931F93E0
:10570000CF93DF93CDB7DEB760970FB6F894DEBFC7
:105710000FBECDBF6115710539F528E0FC01DE0132
:10572000119601900D922A95E1F729813A814B81DA
:105730005C816D817E818F81988560960FB6F8942B
:10574000DEBF0FBECDBFDF91CF911F910F91FF90B4
:10575000EF90DF90CF90BF90AF909F908F907F9011
:105760006F905F904F9008956B018C016AEB78E029
:10577000C6010E94E5D75C01F801F080FF2009F422
:105780004EC0009709F44BC0FC0180858F708430B7
:1057900009F4BFC0853009F042C067E476E087EACB
:1057A0009FE00F94660B87EA9FE00F94160AF501BD
:1057B000E680F780E114F10491F1F70180858F70A4
:1057C0005701823061F0B12CA12CE114F10409F4ED
:1057D0001DC1F70180858F70853021F0F701E280CF
:1057E000F380F3CFC7010E9429D98230B9F760E076
:1057F000C7010E9497D80E9405294C0161E0C701AA
:105800000E9497D8F80120812815190439F7FC0166
:1058100020852F70223011F7009709F001C163E451
:1058200076E0C6010E94E5D77C01F8018181807F86
:1058300009F407C1E114F10409F47DC0F701808582
:105840008F70853009F001C1C7010E9429D98430C9
:1058500009F0FBC0C8010E9493244B015C0160E089
:10586000C7010E9497D8FC0181859285A385B485E4
:1058700019821A821B821C821D821E821F82188638
:1058800088169906AA06BB060CF499C08A818F7007
:105890008A8363E0C7010E9497D85C0162E0C70178
:1058A0000E9497D8FC01418452846384748461E02F
:1058B000C7010E9497D84C0160E0C7010E9497D8A9
:1058C000FC01C184D284E384F484C8010E9493243F
:1058D000F50121853285438554852419350946090A
:1058E00057096C197D098E099F090F94453EF401F3
:1058F00021853285438554852C193D094E095F0960
:105900000F94773EBA01A901440D551D661D771D00
:1059100031C06EEC77E0818592850F943943892BF5
:1059200009F07DCFF0E1FF1609F460C0FF1568F0C3
:1059300082E0F816E1F1F8014081518162817381C2
:1059400084819581A681B78129C0E1E1FE16F1F13C
:10595000F2E1FF12F0CF19821A821B821C821D8293
:105960001E821F8218868A818F708A8344E150E0EC
:1059700060E070E0CE0101960E94802229873A877C
:105980004B875C876D877E878F87988B49855A8583
:105990006B857C858D859E85AF85B88949835A83C3
:1059A0006B837C838D839E83AF83B887BECE198241
:1059B0001A821B821C821D821E821F8218868A8187
:1059C0008F708A8340E050E0BA01D4CF19821A82E6
:1059D0001B821C821D821E821F8218868A818F7004
:1059E0008A8340E850E060E070E0C4CF19821A82F8
:1059F0001B821C821D821E821F8218868A818F70E4
:105A00008A834FEF50E060E070E0B4CFA114B1049E
:105A100009F405CFF50180858F7009F400CFC50129
:105A200019821A821B821C821D821E821F82188686
:105A30002A812F702A83FC014185528563857485F4
:105A400099CFE114F10409F476CFF70180858F70C6
:105A500009F071CF19821A821B821C828A818F7091
:105A60008A8349815A816B817C8180E090E0DC01EE
:105A700095CF0F931F93CF93DF938C01FC01C081CF
:105A8000D1816FE270E0CE010F9476430097E9F088
:105A9000FC011192CF010E94B51EEC0165EB79E08B
:105AA00087EA9FE00F94CC0B4AE050E0BE0187EA02
:105AB0009FE00F941D0B87EA9FE00F94160ACE011A
:105AC000DF91CF911F910F910895CE010E94B51ED5
:105AD000EC01892BA1F3F80111821082F0CFDC01D7
:105AE000ED91FC91309729F090859F7081E0953081
:105AF00009F080E00895EF92FF920F931F93CF93E8
:105B0000DF93EC017B018E819F81892BA9F4888131
:105B100099810E9429D9082F10E00530110564F4FD
:105B20000E94E0DD9F838E83BC01888199810E9461
:105B3000EDDD0F5F1F4FF1CFEE81FF813097D9F080
:105B40008085982F9F70A9F4807F82608087EE8186
:105B5000FF811186128613861486EE81FF81F782FB
:105B6000E682C701DF91CF911F910F91FF90EF90D7
:105B70000895923061F3F12CE12CF3CFCF92DF92B4
:105B8000EF92FF920F931F93CF93DF93EC016A0183
:105B90007B018E819F81892BA9F4888199810E9444
:105BA00029D9082F10E00530110564F40E94E0DDCA
:105BB0009F838E83BC01888199810E94EDDD0F5FF8
:105BC0001F4FF1CFEE81FF81309781F08085982FB4
:105BD0009F7051F4807F82608087EE81FF81C18653
:105BE000D286E386F48602C09230B9F3DF91CF917A
:105BF0001F910F91FF90EF90DF90CF900895FC01DF
:105C000086819781009799F0FC0120852F702230C2
:105C100029F461857285838594850895253039F44A
:105C200060E00E9497D8009711F0FC01F2CF60E08D
:105C300070E0CB0108950F931F93CF93DF93FC0186
:105C4000C281D3812097C9F18B0188858F708530FF
:105C500021F5CE010E9429D98017110671F16CF14E
:105C6000602FCE010E9497D8FC01892B31F18085ED
:105C70008F70823039F461857285838594850F94A5
:105C8000123D06C08330C9F4618572858385948591
:105C9000DF91CF911F910F910895672B71F482309E
:105CA00029F469857A858B859C85E9CF833029F431
:105CB00069857A858B859C85EBCF60E070E0CB01B0
:105CC000E7CF0F931F93CF93DF93FC01C281D38162
:105CD0002097F9F088858F70823049F4672BC9F4DA
:105CE00089859A85DF91CF911F910F910895853015
:105CF00081F48B01CE010E9429D98017110649F049
:105D000044F0602FCE010E9497D8FC0181859285D6
:105D1000E9CF90E080E0E6CF0F931F93CF93DF931E
:105D2000EC018B017B836A8387EC92E09983888303
:105D300070E060E0C8010E94612E97FD0CC09D8359
:105D40008C83C8010E943B1B9F838E83DF91CF9180
:105D50001F910F910895919581959109F0CF8F92A0
:105D60009F92AF92BF92CF92DF92EF92FF920F93EA
:105D70001F93CF93DF93EC01888199810E9429D9E9
:105D8000082F10E00430110554F40E94E0DDBC013E
:105D9000888199810E94EDDD0F5F1F4FF3CF60E096
:105DA000888199810E9497D87C01009769F1DC0174
:105DB00018968C9118978F70843041F51996CD9074
:105DC000DC90C114D10401F1F60180818823E1F057
:105DD00087ED882E8FE0982EB12CA12C1A2DC401AE
:105DE0000F942637AC01B401C6010F943F37892BBD
:105DF00009F46BC1FFEFAF1ABF0A89E0880E911C4E
:105E0000A7E1AA16B10451F71FEF04C08230E1F7F1
:105E1000F70111851887C880D98061E0C6010E940A
:105E200097D87C019B838A8362E0C6010E9497D841
:105E30009D838C8364E0C6010E9497D89F838E83E4
:105E4000153108F031C0E12FF0E08827E55DF04D15
:105E50008F4F0D94CC3E612F612F612F402F542F17
:105E6000542F542F542F542F542F802F6F2FB62F71
:105E7000DD2FC82F542FE82F612F3C30542F57307F
:105E80008AE090E00F94DD348C01BE010E948C2EDC
:105E90008FEA93E0D80111969C938E9319961C92E9
:105EA0001E9218971A870987DF91CF911F910F9142
:105EB000FF90EF90DF90CF90BF90AF909F908F902A
:105EC000089588E090E00F94DD348C01BE010E94BB
:105ED0008C2E8BE893E0F80191838083E3CF8DE0F3
:105EE00090E00F94DD348C01BE010E948C2E87E679
:105EF00093E0D8018D939C93C8010E941CC7D2CF18
:105F000089E090E00F94DD348C01FC01D383C283DF
:105F100085E493E091838083CE010E945518D801D7
:105F200015969C938E9314978EEA9BE018969C93FB
:105F30008E931797CE010E943B1B892B09F4B2CF99
:105F400070E060E0CE010E94612EF8018683882314
:105F500041F0823009F0A6CF8BE49CE090878783E4
:105F6000A1CF8AE09FE0908787839CCF8EE090E06E
:105F70000F94DD348C01DC011396DC93CE931297E1
:105F800089E394E08D939C93C8010E9450C78ACF07
:105F900086E090E00F94DD348C01FC01D383C28352
:105FA00083E293E091838083CE010E945518D8014B
:105FB00015969C938E93149775CF86E090E00F947E
:105FC000DD348C01FC01D383C28381E093E0EACF0E
:105FD0008BE090E00F94DD348C01FC01D383C2830D
:105FE00087E194E091838083168270E060E0CE01C7
:105FF0000E94612E97FD2DC0D80115969C938E931B
:106000001497D80114968D919C91009719F08634BD
:1060100091052CF080E290E0F8019583848361E0A3
:1060200070E0CE010E941B2E20E030E04AE754E4ED
:106030000F94713D0F94E43F611571058105910541
:1060400089F0D80117966D937D938D939C931A9741
:1060500029CF919581959109F8019583848381E0F9
:106060008683CFCF88E893E1A0E0B0E0F801878392
:106070009087A187B28716CF86E090E00F94DD3439
:10608000FC01D383C28385EF93E0918380831582E3
:106090001482E114F10441F0D70118968C918F70AD
:1060A000863011F4F582E482FA87E987FDCE84E038
:1060B00090E00F94DD34FC01D383C28323ED33E001
:1060C000318320839A878987EFCEC6010F946D10A4
:1060D0008A2D90E0B0E0A0E0F70181879287A38746
:1060E000B4878085807F8260808794CECF92DF9254
:1060F000EF92FF926A017B0163E0FC018081918154
:106100000E9497D8FC01892BA9F080858D7091F4AD
:10611000C094D094E094F094CC24CA948185928564
:10612000A385B4858C219D21AE21BF2181879287D3
:10613000A387B487FF90EF90DF90CF900895CF9220
:10614000DF92EF92FF926A017B0163E0FC018081A4
:1061500091810E9497D8FC01892BA9F09085892F05
:106160008D7089F4907F92609087CC24FF244185C4
:106170005285638574854C295D296E297F29418765
:10618000528763877487FF90EF90DF90CF900895D8
:10619000CF92DF92FF920F931F93CF93DF93F12C57
:1061A0006115710509F499C06A01EB018C01CB01FD
:1061B0000E946F2DF82E882309F48FC0D2FE09C0EB
:1061C000D8018C918B3009F44BC0E8F58A3009F482
:1061D0004CC0D0FE09C0F801608186EF860F843084
:1061E00018F0CE010E947C1BD1FE6EC0D80114961F
:1061F0004D915D916D917C91179711968C9182953F
:106200008F70873038F0893008F43EC08A50823071
:1062100008F46CC0CE010E946518EC81FD813097B6
:1062200009F452C080858F709EEF980F923010F065
:1062300081114AC0D80111969C91907F80858F7002
:10624000892B808741C08C30B9F040E050E062E09B
:1062500070E08D3009F0BDCFCE010E949F30B9CFE4
:1062600040E050E061E070E0F7CF40E050E061E0F6
:1062700070E0CE010E94763040E050E062E070E0D5
:10628000CE010E947630A5CFEC81FD813097E1F000
:1062900080858F709EEF980F923010F0811114C09E
:1062A0004187528763877487EC81FD818085807F79
:1062B00083608087EC81FD818085982F907F8F702F
:1062C0008067903609F4BDCF6DE371E187EA9FE006
:1062D0000F94CC0BC8010E941A288F2DDF91CF910B
:1062E0001F910F91FF90DF90CF900895CE010E94F3
:1062F0006518EACFCF92DF92EF92FF926A017B019D
:1063000063E0FC01808191810E9497D8009791F011
:10631000FC0120852F70223069F4618572858385A8
:1063200094856C217D218E219F21FF90EF90DF903D
:10633000CF90089560E070E0CB01F7CFAF92BF92AD
:10634000CF92DF92EF92FF920F931F93CF93DF9341
:10635000CDB7DEB7CD56D1090FB6F894DEBF0FBE6C
:10636000CDBF5C01A7960FAFA797A8961FAFA897C0
:10637000A9962FAFA997AA963FAFAA97AB964FAF12
:10638000AB97AC965FAFAC97AD966FAFAD97AE964F
:106390007FAFAE9723961FAE1EAE2397FE01ED5B37
:1063A000FF4F82E1DF011D928A95E9F77296119203
:1063B000119287E0DF011D928A95E9F7CE018A5993
:1063C0009F4F0E941A28F0FE2CC0A796EFADA7970A
:1063D000E83108F050C1F0E08827EE50FE4C8F4FB6
:1063E0000D94CC3E41330A3238333B333B333833A0
:1063F0000A323B333B333B333B333B333B333B335F
:106400000A320A323B333B333B330A320A320A3216
:106410003B3341336BE87EE0CE018B5A9F4F0F94A4
:106420001F370E9403D8882309F407C18091C9103F
:10643000811103C1C114D10409F05EC030E020E035
:1064400043E050E060E4CE0101960F947928D50135
:10645000ED91FC91608171814FE350E0CE01019696
:106460000F944943F1FE10C1A7968FADA7978230D4
:1064700009F40AC1853009F407C1A8968FADA89721
:1064800082958F709FE0980F9F70923018F088303F
:1064900009F0FAC001E020E032E044E150E0BE0142
:1064A0006F5B7F4FCE018A599F4F0E94F925BE0135
:1064B0006F5B7F4FCE0101960E941BEB6EE67EE084
:1064C00087EA9FE00F94CC0BBE016F5F7F4F87EA96
:1064D0009FE00F94660B6BE67EE087EA9FE00F94E7
:1064E000CC0BBE016F5B7F4F87EA9FE00F94660B7A
:1064F00087EA9FE00F94160AA8968FADA897807F31
:10650000870100271072882311F0F1FC04C00115E7
:10651000110509F4F5C030E020E043E050E060E40C
:10652000CE0101960F947928D501ED91FC916081FF
:1065300071814FE350E0CE0101960F944943C1149D
:10654000D10469F066E877E0CE0101960F94234309
:106550004FE350E0B601CE0101960F94494366E83F
:1065600077E0CE0101960F9423434FE350E060E3C0
:106570007EE00115110511F466E27EE0CE01019680
:106580000F942F37A8968FADA89782958F7084505F
:10659000823008F09FC067E1CE018A599F4F0E9468
:1065A00043206F962FAF6F97A0963FAFA097A1960D
:1065B0004FAFA197A2965FAFA297A3966FAFA39795
:1065C000A4967FAFA497A5968FAFA597A6969FAFE9
:1065D000A69700E020E033E044E150E0BE016F5BAD
:1065E0007F4FCE018A599F4F0E94F92566E17EE0D8
:1065F00087EA9FE00F94CC0BBE016F5F7F4F87EA65
:106600009FE00F94660B63E17EE087EA9FE00F94C2
:10661000CC0BBE016F5B7F4F87EA9FE00F94660B48
:1066200087EA9FE00F94160A0E9403D8882329F076
:106630008091C910882309F455C0A701FF0C660B8F
:10664000770BC5010E949F3090E080E0C359DF4F77
:106650000FB6F894DEBF0FBECDBFDF91CF911F9173
:106660000F91FF90EF90DF90CF90BF90AF90089583
:1066700064E97EE0D1CE64E77EE087EA9FE00F9494
:10668000CC0BE894F0F8CDCEF0FE36CF66968FAD09
:106690006697882309F430CFBE016B5A7F4FCE0135
:1066A00001960E941BEB65E67EE087EA9FE00F946F
:1066B000CC0BBE016F5F7F4F87EA9FE00F94660BA4
:1066C00062E67EE087EA9FE00F94CC0BBE016B5A36
:1066D0007F4F0ACF20E032E0012B11F020E033E0C1
:1066E00000E07ACFBE016F5B7F4FCE0101960E9422
:1066F0001BEB40E052E060E070E0C5010E947630A4
:10670000F0FE90C0A796EFADA797E150E53118F5E0
:10671000F0E08827E157FC4C8F4F0D94CC3E9A3423
:10672000AB33AB33AB33AB339A34AB33AB33AB3389
:10673000AB33AB33AB33AB339F349734AB33AB3387
:10674000AB33A433913494346DE27FE0CE018B5AA5
:106750009F4F0F941F3730E020E043E050E060E4AB
:10676000CE0101960F947928D501ED91FC916081BD
:1067700071814FE350E0CE0101960F944943C1145B
:10678000D10469F066E877E0CE0101960F942343C7
:106790004FE350E0B601CE0101960F94494366E8FD
:1067A00077E0CE0101960F9423434FE350E061E27E
:1067B0007EE0CE0101960F942F376DE07EE087EAF0
:1067C0009FE00F94CC0BBE016F5F7F4F87EA9FE085
:1067D0000F94660B6AE07EE087EA9FE00F94CC0B93
:1067E000BE016B5A7F4F87EA9FE00F94660B87EAE2
:1067F0009FE00F94160A0E9403D8882309F41DCF46
:106800008091C910811119CFBE016B5A7F4FCE0103
:1068100001960E941BEB40E051E060E070E0C50192
:106820000E947630F2FE7AC040E050E061E070E015
:10683000C5010E947A31672B682B692B09F482C04D
:1068400065EE7EE0CE018B5A9F4F0F941F3730E0EC
:1068500020E043E050E060E4CE0101960F947928F7
:10686000D501ED91FC91608171814FE350E0CE0143
:1068700001960F944943C114D10469F066E877E0AA
:10688000CE0101960F9423434FE350E0B601CE01B1
:1068900001960F94494366E877E0CE0101960F9484
:1068A00023434FE350E069E47EE0CE0101960F946C
:1068B0002F3764E07EE087EA9FE00F94CC0BBE01A7
:1068C0006F5F7F4F87EA9FE00F94660B61E07EE089
:1068D00087EA9FE00F94CC0BBE016B5A7F4F87EA8B
:1068E0009FE00F94660B87EA9FE00F94160A0E94C0
:1068F00003D8882309F4A1CE8091C91081119DCEBF
:10690000BE016B5A7F4FCE0101960E941BEB40E007
:1069100054E060E070E0C5010E94763081E090E0D4
:1069200095CE66E37FE012CF6FE37FE00FCF69E0A3
:106930007FE00CCFF5018085853009F00CCF60E059
:106940007FE004CF40E050E062E070E0C5010E94CB
:106950007A31672B682B692B19F067EF7EE072CFD5
:106960006CED7EE06FCFAF92BF92CF92EF920F931C
:106970001F93CF93DF93CDB7DEB7C856D1090FB6BB
:10698000F894DEBF0FBECDBF5C01A2960FAFA297F9
:10699000A3961FAFA397A4962FAFA497A5963FAF3A
:1069A000A597A6964FAFA697A7965FAFA797A8966D
:1069B0006FAFA897A9967FAFA9979E2D28E0FE01FB
:1069C000EF59FF4FDE01A75ABF4F01900D922A9554
:1069D000E1F7A296EFADA297E150ED3008F0F2C0DA
:1069E000EC2CF0E08827E850FB4C8F4F0D94CC3E08
:1069F0006F357835D635E035CC3505356635E23539
:106A0000E23581359335B935A635992331F0C50185
:106A10000E94681B009709F449C067E0CE01875ABD
:106A20009F4F0E9443206CEC79E087EA9FE00F942F
:106A3000CC0B4AE050E06A966FAD6A9787EA9FE018
:106A40000F94330A61EC79E087EA9FE00F94CC0B56
:106A5000CE01875A9F4F0E949324AB01BC012AE0CC
:106A600030E087EA9FE00F94D50A87EA9FE00F9411
:106A7000160A6A960FAD6A976B961FAD6B976C9668
:106A80002FAD6C976D963FAD6D976E964FAD6E972F
:106A90006F965FAD6F97A0966FADA097A1967FADF3
:106AA000A197C5010E94D82481E090E0C859DF4F2A
:106AB0000FB6F894DEBF0FBECDBFDF91CF911F910F
:106AC0000F91EF90CF90BF90AF900895911105C0B6
:106AD000C5010E94681B009749F366E09FCF992388
:106AE00029F0C5010E94681B009701F362E096CF70
:106AF000911105C0C5010E94681B0097B9F261E0C1
:106B00008DCF40E050E061E070E0C5010E947A3135
:106B1000672B682B692B29F4C5010E94681B00971D
:106B200029F26BE07BCF40E050E061E070E0C5010E
:106B30000E947A31672B682B692B31F0C5010E94C6
:106B4000681B009709F4B2CF6AE068CF40E050E0DC
:106B500062E070E0C5010E947A31672B682B692BD7
:106B600031F0C5010E94681B009709F49FCF6CE0CB
:106B700055CF40E050E062E070E0C5010E947A31FC
:106B8000672B682B692B31F4C5010E94681B0097A5
:106B900009F48CCF6DE042CF911106C0C5010E946F
:106BA000681B009709F482CF63E038CF992331F056
:106BB000C5010E94681B009709F478CF65E02ECFCD
:106BC00064E02CCF90E080E071CF63E0FC01808135
:106BD00091810E9497D8009719F0FC018185089552
:106BE0008FEF0895AF92BF92CF92DF92EF92FF9214
:106BF0000F931F93CF93DF9300D000D01F921F926B
:106C0000CDB7DEB76115710509F461C05A016B019A
:106C10007C01CB010E946F2D082F882379F1D601CA
:106C200014968D919C91009709F445C0FC01108544
:106C3000212F2F703EEF320F323010F0211130C073
:106C400012951F70B0FE5BC0C6010E94E535F701CA
:106C50008083112391F11295107F81818F70182B01
:106C60001183D6011496ED91FC9181859285A385BF
:106C7000B485F70184839583A683B783802F2896F4
:106C80000FB6F894DEBF0FBECDBFDF91CF911F913D
:106C90000F91FF90EF90DF90CF90BF90AF9008954D
:106CA000253049F460E00E9497D8009721F0DC017C
:106CB00018961C91C5CF10E0C5CFD6011496ED9162
:106CC000FC9180858F70823021F0833051F000E09C
:106CD000D5CF4185528563857485C7010E94A9225D
:106CE000CDCF4185528563857485F70181818F7091
:106CF000806781834483558366837783BFCF112365
:106D0000E1F21295107FF701A8CFAF92BF92CF9218
:106D1000DF92EF92FF920F931F93CF93DF9300D0F8
:106D200000D01F921F92CDB7DEB75C017B0160FFE0
:106D300003C0E894E0F8F4F8F4FC0DC00F94FA29CD
:106D4000663971058105910530F08091E3109091CD
:106D5000E410059719F5A70144275770052E000C7C
:106D6000660B770BC5010E949F3060EF7DE087EADC
:106D70009FE00F94CC0B8FEF9FEF28960FB6F894FF
:106D8000DEBF0FBECDBFDF91CF911F910F91FF905E
:106D9000EF90DF90CF90BF90AF90089519821A8244
:106DA0001B821C821D821E821F8218868A818F7020
:106DB0008A8340E053E0B501CE0101960E94F2358E
:106DC00040E057E060E070E0C5010E947A31E62AB9
:106DD000F72AD12CC12C09811A812B813C814D814C
:106DE0005E816F817885C5010E949E31C6CFCF93A9
:106DF000DF93EC0140E053E060E070E00E947A3104
:106E0000611571058105910599F02091E31030918C
:106E1000E4102630310561F4CE010E94853640E051
:106E200053E060E070E0CE01DF91CF910C947630BA
:106E3000DF91CF9108958F929F92AF92CF92EF9270
:106E4000FF920F931F93CF93DF9300D000D01F9238
:106E50001F92CDB7DEB74C0109831A832B833C8385
:106E60004D835E836F8378876AEF78E087EA9FE0DF
:106E70000F94CC0BCE0101960E941A2889818111B2
:106E800030C00A810F70013089F140F1023019F0F1
:106E900010E00530F1F5D401ED91FC91068CF78DF1
:106EA000E02D09811A812B813C814D815E816F81AA
:106EB0007885C401199581E090E028960FB6F89482
:106EC000DEBF0FBECDBFDF91CF911F910F91FF901D
:106ED000EF90CF90AF909F908F900895CC24C39463
:106EE000DACF813071F1823009F451C06DEE78E073
:106EF00087EA9FE00F94CC0B4AE050E0698187EA73
:106F00009FE00F94330A87EA9FE00F94160A01E08E
:106F100010E06DED78E087EA9FE00F94CC0B4AE03B
:106F200050E0B80187EA9FE00F941D0B87EA9FE0CD
:106F30000F94160ACE0101960E941A2890E080E074
:106F4000BCCFCE0101960E94A6D84497B8F46EE15A
:106F500070E0CE0101960E94F823F40162817381F2
:106F600040E052E0CE0101960E94C83060E072E13C
:106F7000D40112968D919C910E948536D401ED9199
:106F8000FC91068CF78DE02DCC24C3948ACF1D8212
:106F90001E821F821886D401ED91FC91068CF78D1C
:106FA000E02DCC24C39402E01A812B813C8140E087
:106FB0007DCF8F929F92AF92BF92CF92DF92EF924E
:106FC000FF920F931F93CF93DF93CDB7DEB76097F8
:106FD0000FB6F894DEBF0FBECDBF8C017B0140E041
:106FE00058E060E070E00E947A31672B682B692BD3
:106FF00009F0A9C062E070E0C8010E94612E6C0136
:1070000019861A861B861C861D861E861F86188A70
:107010008A858F708A87D7FC96C040E052E0B8011D
:10702000CE0109960E94F23563E070E0C8010E942B
:10703000612EAC011816190614F04FE350E081E000
:10704000C816D10429F4EF2CFF0CFF08FF2404C05C
:1070500082E0C816D104D4F32FEF30E0D7010F94AB
:10706000E33E9A01550F440B550B0F94773E4901AF
:107070006901C8010E94E535E82EF12C60E0CE01DF
:1070800009960E942B2388169906F9F4CD2841F021
:1070900082E0E816F10419F185E0E816F104F9F050
:1070A00081E090E060960FB6F894DEBF0FBECDBFD2
:1070B000DF91CF911F910F91FF90EF90DF90CF90D4
:1070C000BF90AF909F908F900895CD2859F186E0A2
:1070D000E816F10441F081E0E816F10421F061E0E6
:1070E000C8010E947C1BB401CE0109960E94D222E5
:1070F00040E052E0B801CE0109960E94C83082E01B
:10710000E816F10421F085E0E816F10429F460E0C6
:1071100071E0C8010E94853660E072E0C8010E94FB
:107120008536BECF85E0E816F10409F4B9CF82E0D8
:10713000E816F10409F4B4CF62E0C8010E947C1B98
:1071400060E071E0EBCF90E080E0ACCF81E090E0D8
:1071500008950F931F93CF93DF9300D000D01F9219
:107160001F92CDB7DEB719821A821B821C821D8244
:107170001E821F8218862A812F702A83FC010281B9
:107180001381C8010E94E535813041F020F0823042
:1071900011F0853081F490E080E002C081E090E061
:1071A00028960FB6F894DEBF0FBECDBFDF91CF910A
:1071B0001F910F91089540E052E0B801CE01019671
:1071C0000E94F23560E0CE0101960E942B23E8CFA9
:1071D0008F929F92AF92BF92CF92DF92EF92FF92E7
:1071E0000F931F93CF93DF93CDB7DEB767970FB69B
:1071F000F894DEBF0FBECDBF8C017B014C018BE04C
:10720000880E911C9F8A8E8AF80112861186138639
:10721000148E138E672B09F463C0A090E510B09014
:10722000E610A114B10409F45BC06FE270E0C7017D
:107230000F942E436C01892B09F44AC0F701DE013B
:10724000119690E080E0BD012191222341F02F3280
:1072500031F08431910519F02D930196F5CF860F09
:10726000971FFC011082C5010E94E5D7F8019183A8
:107270008083B6016F5F7F4F4FE050E0C4010F94F1
:107280006743CE0146960E94392DF801948F838F73
:107290008E899F89892B09F41386C8010E946F2D5E
:1072A000882319F0C8010E94AF2E67960FB6F89494
:1072B000DEBF0FBECDBFDF91CF911F910F91FF9029
:1072C000EF90DF90CF90BF90AF909F908F900895F8
:1072D000B701C5010E94E5D7F80191838083DDCF16
:1072E000F80111821082D9CFDC0119968D919C9101
:1072F000009739F0DC01ED91FC910280F381E02DE3
:10730000199408958F929F92AF92BF92CF92DF927D
:10731000EF92FF920F931F93CF93DF93CDB7DEB71A
:10732000CD55D1090FB6F894DEBF0FBECDBF8C018D
:107330006B016115710519F041155105D1F46CE12E
:1073400073E187EA9FE00F94CC0B63E173E187EA76
:107350009FE00F94CC0BB80187EA9FE00F94660B77
:1073600061E173E187EA9FE00F94CC0B87EA9FE02D
:1073700032C0460F571FDA011C920F94FA294B01B5
:107380006FE073E187EA9FE00F94CC0B4AE050E096
:10739000B40187EA9FE00F941D0B6CE073E187EA6C
:1073A0009FE00F94CC0BB80187EA9FE00F94660B27
:1073B00069E073E187EA9FE00F94CC0BBAE38B1688
:1073C000B1E09B06F4F46CEF72E180E09FE00F9473
:1073D000CC0B80E09FE00F94160AC35ADF4F0FB624
:1073E000F894DEBF0FBECDBFDF91CF911F910F91FB
:1073F000FF90EF90DF90CF90BF90AF909F908F90D5
:1074000008956AEF72E187EA9FE00F94CC0BB60112
:1074100087EA9FE00F94660B68EF72E187EA9FE0CE
:107420000F94CC0B87EA9FE00F94160A1A821982F8
:10743000FE0133968EE3DF011D928A95E9F7809174
:10744000E3109091E410059791F563E070E0C801B6
:107450000E94DF1E7C01892BE9F5E091260DF09159
:10746000270D808180FFB9CF61E070E0C8010E94E4
:10747000DF1E892B09F4B1CF64E270E0C8010F94DC
:107480007643892B09F0A9CF60EE72E187EA9FE08D
:107490000F94CC0BB80187EA9FE00F94660B87EA44
:1074A0009FE00F94160AC8010E9469E596CF61E03B
:1074B00070E0C8010E94DF1E7C01892B49F562E063
:1074C00070E0C8010E94DF1E7C0165ED72E1892B2E
:1074D00009F448CFE00EF11E6CEC72E1C7010F9485
:1074E0001637892BE9F4F60101900020E9F731976E
:1074F000EC19FD093297A0F0C8010E9469E5F60178
:107500008081882309F469CFC6010F94A90F65CF44
:107510004FE350E0B801CE0101960F946743DACFF4
:1075200064E270E0C8010F947643892B09F055CFCF
:10753000B701CE018F5B9F4F0E94E838CE018F5B71
:107540009F4F0E946F2D882339F1B601CE018F5BCA
:107550009F4F0E9434DF18161906F4F4898188239E
:10756000D9F08091E3109091E4100597A9F064EBB5
:1075700072E187EA9FE00F94CC0BBE016F5F7F4FF3
:1075800087EA9FE00F94660B87EA9FE00F94160A44
:10759000CE0101960E9469E5CE018F5B9F4F0E944C
:1075A00074391BCFCF93DF93EC01798368831A86FC
:1075B00019861B861C8E1B8E0E946F2D882329F036
:1075C000CE01DF91CF910C94AF2EDF91CF91089532
:1075D000CF93DF93EC01FB01248135814081518100
:1075E000628173810F94D50ACE01DF91CF91089506
:1075F000CF92DF92EF92FF921F93CF93DF9300D051
:1076000000D0CDB7DEB760E273E186EF9EE00F9465
:10761000CC0B8AEDE82E8EE0F82E10E090E1C92E1A
:10762000D12CF70181917F01803130F465E576E05E
:1076300086EF9EE00F94660B153041F1F70131970C
:10764000808190E0B0E0A0E089839A83AB83BC8323
:10765000DE82CD82BE016F5F7F4F86EF9EE00E948B
:10766000E83A6EE173E10F94CC0B1F5F1630C9F658
:1076700026960FB6F894DEBF0FBECDBFDF91CF9137
:107680001F91FF90EF90DF90CF9008958091DF0ED3
:1076900090E0B0E0A0E089839A83AB83BC83DE8274
:1076A000CD82BE016F5F7F4F86EF9EE00E94E83A79
:1076B0000F94160ADACFEF92FF920F931F93CF9396
:1076C000DF9300D000D01F92CDB7DEB77B01CE0193
:1076D00007969F938F9301979F938F9301979F9303
:1076E0008F9301979F938F9301979F938F93019708
:1076F0009F938F938E010F5F1F4F1F930F9387E50B
:1077000096E09F938F93DB0113968C9113978F9341
:1077100012968C918F930F94EE430FB6F894DEBFC0
:107720000FBECDBF0697ECF46BE87CE180E09FE0F4
:107730000F94CC0BD70112966D917C9180E09FE065
:107740000F94660B80E991E027960FB6F894DEBFA0
:107750000FBECDBFDF91CF911F910F91FF90EF90A2
:1077600008958091D20E9091D30E892B09F449C0CF
:107770000E9439D9882309F444C0A091D20EB09157
:10778000D30E52961C921E92519754961C921E92A2
:10779000539784E890E01D969C938E931C971E96B9
:1077A0001C921E9782E755968C935597ED91FC910C
:1077B00011970088F189E02D64E070E0CD01199502
:1077C0008091D20E9091D30EDC01ED91FC9102805C
:1077D000F381E02D46E050E0B801199586E0F8010C
:1077E000AAEDBEE001900D928A95E1F78091D20E4C
:1077F0009091D30EDC01ED91FC910488F589E02D88
:1078000019950E94F83A6DE97CE186EF9EE00F94AD
:10781000CC0B88EC90E098CFEF92FF920F931F93E0
:10782000CF93DF9300D000D0CDB7DEB77C018B01C2
:107830006CE67FE087EA9FE00F94CC0BD701ED91D7
:10784000FC916081718187EA9FE00F94660B63E68B
:107850007FE087EA9FE00F94CC0B012E000C220BF7
:10786000330B09831A832B833C8380E190E09E8352
:107870008D83BE016F5F7F4F87EA9FE00E94E83AE9
:107880000F94160A40E058E060E070E0C7010E94E3
:107890009F3026960FB6F894DEBF0FBECDBFDF91A6
:1078A000CF911F910F91FF90EF9008953F924F92CB
:1078B0005F926F927F928F929F92AF92BF92CF9280
:1078C000DF92EF92FF920F931F93CF93DF93CDB789
:1078D000DEB72C970FB6F894DEBF0FBECDBF5C01AC
:1078E000362E972E3A0169016DEC7FE087EA9FE022
:1078F0000F94CC0B4AE050E0632D792D87EA9FE08E
:107900000F941D0B65EC7FE087EA9FE00F94CC0B92
:10791000C301B0E0A0E08F839887A987BA8730E1E0
:10792000432E512C5C864B86BE01695F7F4F87EAF0
:107930009FE00E94E83A4C0161EC7FE00F94CC0B91
:107940004AE050E0B601C4010F941D0B69EB7FE0E3
:10795000C4010F94CC0BC701B0E0A0E089839A83E7
:10796000AB83BC835E824D82BE016F5F7F4FC401DB
:107970000E94E83A0F94160A8091B60A9091B70ACD
:1079800070E060E0892B09F047C081E090E09093BF
:10799000B70A8093B60A26E040E855E260E070E05E
:1079A0008BE49CE00F94190D30924B0D8BE49CE01E
:1079B00090934A0D8093490D1092560E1092580ED6
:1079C0001092570E0130110509F44EC00CF041C061
:1079D000012B09F44EC0C114D10409F457C082E050
:1079E000C816D10409F062C07092D10D6092D00D1A
:1079F0001092D30D1092D20DF092D50DE092D40DCD
:107A000086E00E94A4EB1092B70A1092B60A88236F
:107A100009F456C0682F70E0C5010E940C3C90E04C
:107A200080E02C960FB6F894DEBF0FBECDBFDF917D
:107A3000CF911F910F91FF90EF90DF90CF90BF906B
:107A4000AF909F908F907F906F905F904F903F90FE
:107A500008950330110581F00430110509F0BBCF02
:107A6000FE24EF24FE24B7CFFE2CEE24EE24EA946D
:107A7000B2CFFF24FA94AFCFEF2821F492E0E92EA1
:107A8000F12CEECFEE24E394F12CEACF7092D10DDD
:107A90006092D00D90E080E0EE2011F080E09FEF4A
:107AA0009093D30D8093D20D85E0ABCF6DE97FE04D
:107AB00087EA9FE00F94CC0B1092B70A1092B60A97
:107AC00081E090E0AECF2F923F924F925F926F9203
:107AD0007F928F929F92AF92BF92CF92DF92EF925E
:107AE000FF920F931F93CF93DF93CDB7DEB72C9701
:107AF0000FB6F894DEBF0FBECDBF5C0109831A83B9
:107B00002B833C834D835E836F837887CE01019600
:107B10000E94A6D81C01023011F0053011F4312C5E
:107B2000212CF50102811381F80180858F70853049
:107B300009F07FC0C8010E9429D9E82EF12CF2E09B
:107B4000EF16F1040CF475C060E0C8010E9497D8EC
:107B5000FC01818592859C878B8761E0C8010E942A
:107B600097D8FC01418452846384748488248A9465
:107B7000982CF2E0EF16F10459F062E0C8010E947F
:107B800097D8FC0181849284F3E0EF16F104A1F40C
:107B90008FE390E09A87898792E0C92ED12C2985BE
:107BA0003A85D1010F94DB3E24E630E040E050E01E
:107BB0000F94773E79011CC063E0C8010E9497D8FA
:107BC000FC01818592859A87898782E0C82ED12C15
:107BD000F4E0EF16F10439F064E0C8010E9497D890
:107BE000FC01C184D28489859A857101892BB9F6FB
:107BF00084019601A2016B857C85C5010E94563CDB
:107C00002C960FB6F894DEBF0FBECDBFDF91CF919B
:107C10001F910F91FF90EF90DF90CF90BF90AF90AA
:107C20009F908F907F906F905F904F903F902F909C
:107C3000089590E080E0E4CF8F929F92AF92BF9240
:107C4000DF92EF92FF920F931F93CF93DF93CDB705
:107C5000DEB7A5970FB6F894DEBF0FBECDBF7C018F
:107C60000E8F1F8F28A339A34AA35BA36CA37DA308
:107C7000CE014E960E944C244B015C01D701129616
:107C8000ED91FC9180858F70843009F0E9C0102F50
:107C900061857285CE0101960E94E838CE01019679
:107CA0000E946F2D882309F44AC08985893009F024
:107CB00046C070E060E0CE0101960E94612E082F60
:107CC000D92E60E97FE087EA9FE00F94CC0B4AE071
:107CD00050E0602F7D2D87EA9FE00F941D0B6EE82A
:107CE0007FE087EA9FE00F94CC0BB501A40187EAFF
:107CF0009FE00E940FDD68E87FE087EA9FE00F9435
:107D0000CC0B612F70E04AE050E087EA9FE00F94CF
:107D10001D0B87EA9FE00F94160A8091B60A909196
:107D2000B70A892B29F140E053E0B701CE014E9606
:107D30000E94C83070E060E0C7010E940C3C10E077
:107D400000E0CE0101960E947439C801A5960FB6D5
:107D5000F894DEBF0FBECDBFDF91CF911F910F9181
:107D6000FF90EF90DF90BF90AF909F908F9008951D
:107D700081E090E09093B70A8093B60A26E040E84D
:107D800055E260E070E08BE49CE00F94190D0093E5
:107D90004B0D8BE49CE090934A0D8093490D10921B
:107DA000560E1092580E1092570EE981FA81153036
:107DB00021F01F3011F0123011F580858F7080870F
:107DC00070E060E083ED97E09093D10D8093D00D4B
:107DD0001092D30D1092D20D7093D50D6093D40DE7
:107DE00086E00E94A4EB1092B70A1092B60A01E056
:107DF00010E0882309F4A5CF682F70E09DCF80851F
:107E00008F708061808722E538EB42E152E4C50142
:107E1000B4010F94FF3E20E030E040E251E40F94C3
:107E2000713D2DEE3EE94CE35EE30F946B3F4B0159
:107E30005C0120E030E0A9010F94134020E030E025
:107E400040E05FE387FD07C0C501B4010F94FF3E2A
:107E50000F94DD3FB7CFC501B4010F94FE3EF8CFBC
:107E600010E000E072CFCF92DF92EF92FF920F937B
:107E70001F93CF93DF9300D000D01F921F92CDB7F6
:107E8000DEB77C0109831A832B833C834D835E8399
:107E90006F837887CE0101960E94A6D88C018981D4
:107EA000882359F09A819F70923008F0BAC08230CE
:107EB00011F0853011F410E000E070E060E0C701DF
:107EC0000E94612ED82EC92E60E87FE087EA9FE0ED
:107ED0000F94CC0B4AE050E06D2D7C2D87EA9FE09B
:107EE0000F941D0B6EE77FE087EA9FE00F94CC0BA9
:107EF0004AE050E0B80187EA9FE00F941D0B87EA43
:107F00009FE00F94160A8091B60A9091B70A892BC8
:107F1000E9F040E053E0B701CE0101960E94C8307D
:107F200070E060E0C7010E940C3C90E080E0289681
:107F30000FB6F894DEBF0FBECDBFDF91CF911F917A
:107F40000F91FF90EF90DF90CF90089581E090E047
:107F50009093B70A8093B60A26E040E855E260E0C5
:107F600070E08BE49CE00F94190DD0924B0D8BE4E4
:107F70009CE090934A0D8093490D1092560E1092FA
:107F8000580E1092570E80ED97E09093D10D80938C
:107F9000D00D1092D30D1092D20D01151105E1F103
:107FA00085E090E09093D50D8093D40D86E00E94FB
:107FB000A4EBD82E64E670E080E090E00E948CE8AC
:107FC000D1100AC067E77FE087EA9FE00F94CC0BEF
:107FD00087EA9FE00F94160A82ED97E09093D10D07
:107FE0008093D00D1092D30D1092D20D24E6209FD5
:107FF000C001219F900D11249093D50D8093D40D35
:1080000086E00E94A4EB1092B70A1092B60A882369
:1080100059F0682F70E086CF1092D50D1092D40DD4
:10802000C5CF8FEF9FEF83CF81E090E080CFEF92BD
:10803000FF920F931F93CF93DF93EC018B011D826F
:108040001C821A821B82E880F980E114F10409F491
:108050005DC08091B10A9091B20A892B09F456C093
:10806000672B09F48701F80180858F708630A9F4A9
:1080700061EE78E0C8010E94E5D7009719F0FC0195
:1080800081858A8360E877E0C8010E94E5D7009780
:1080900009F443C0FC0181858B836BE676E0C70160
:1080A0000E94E5D7009779F569E079E087EA9FE0DB
:1080B0000F94CC0B4AE050E06B8187EA9FE00F946D
:1080C000330A67E079E087EA9FE00F94CC0B4AE03F
:1080D00050E06A8187EA9FE00F94330A87EA9FE0C5
:1080E0000F94160A20E030E0A9016BE676E0888163
:1080F00099810E94A2DE6BE676E0888199810E94D8
:10810000E5D7009719F009969D838C83DF91CF9175
:108110001F910F91FF90EF900895F8018081918158
:108120000F94AA36B9CFFC016115710519F4848149
:108130009581089586819781681779072CF084814D
:108140009581860F971F0895828193810C94612EEB
:10815000EF92FF920F931F93CF93DF93DC01129660
:10816000ED91FC91309709F17A018B01EC0164E10A
:1081700076E0808191810E94E5D70097B1F0FC0103
:1081800020852F70243089F461857285E881F9811A
:108190000288F389E02D9701A801CE01DF91CF91EC
:1081A0001F910F91FF90EF90199490E080E0DF9184
:1081B000CF911F910F91FF90EF900895EF92FF9252
:1081C0000F931F93CF93DF93CDB7DEB760970FB6B2
:1081D000F894DEBF0FBECDBF8C017901CE010196B0
:1081E0000F94A129A701BE016F5F7F4FC8010E94B4
:1081F000A84060960FB6F894DEBF0FBECDBFDF91EA
:10820000CF911F910F91FF90EF900895FF920F93E0
:108210001F93CF93DF9300D000D0CDB7DEB78C0192
:10822000BC01CE0101960F94A307BE016F5F7F4F83
:1082300087EA9FE00F94BE0B87EA9FE00F94160A2F
:10824000CE0101960F949B071A8219821C821B8211
:108250001E821D826AED7DE1CE0101960F943E07DC
:10826000F801248135818D819E81F12C28173907F1
:1082700038F0BE016F5F7F4FC8010E9454E5F82EB1
:10828000CE0101960F949B07FF2069F0B801CE0143
:1082900001960F94A307CE0101960E9479F2CE01B8
:1082A00001960F949B0726960FB6F894DEBF0FBE7B
:1082B000CDBFDF91CF911F910F91FF900895AF92A5
:1082C000BF92DF92EF92FF920F931F93CF93DF93B2
:1082D00000D000D0CDB7DEB78C017B01D42EFB01DE
:1082E00084819581892BF9F0A080B1806FE370E0E3
:1082F000C5010F942E430097B1F09C012A193B0948
:1083000037FD11C050E040E0B701CE0101960F9457
:10831000BD07BE016F5F7F4FC7010F94F306CE010B
:1083200001960F949B07F70184819581892BD9F1E0
:10833000E080F1806EE676E0C7010F943943892B27
:1083400001F5F801128A118A80E090E1958784870F
:1083500084E890E0948B838B81E08687D58A81E0E6
:1083600090E026960FB6F894DEBF0FBECDBFDF912A
:10837000CF911F910F91FF90EF90DF90BF90AF9042
:1083800008956BE776E0C7010F943943892B59F4C0
:10839000F801128A118A148A138A84E890E095877A
:1083A00084871686DBCF90E080E0DBCF0F931F93AE
:1083B000CF93DF9300D000D0CDB7DEB7A091D20E1F
:1083C000B091D30E109709F478C052961C921E9269
:1083D000519754961C921E92539784E890E01D96F4
:1083E0009C938E931C971E961C921E9787E755961A
:1083F0008C935597ED91FC9111970088F189E02DB0
:1084000070E060E0CD01199510E000E08091D20E9F
:108410009091D30EDC01ED91FC9111971C962D915A
:108420003C910217130740F40190F081E02D60E0C9
:1084300019950F5F1F4FEACF0088F189E02D70E09A
:1084400060E0199509ED14E08091D20E9091D30E61
:10845000F80161918F01DC01ED91FC910190F081B7
:10846000E02D1995B4E00D3D1B0771F78091D20EF8
:108470009091D30EDC01ED91FC910488F589E02DFB
:1084800019956AE879E0CE0101960F94AC07CE0108
:1084900001960E9479F2CE0101960F949B0787E026
:1084A00090E00E94E5DC87E090E00E94EFDC6EE463
:1084B0007CE186EF9EE00F94CC0B1092F20E1092AE
:1084C000F10E80E090E19093ED0E8093EC0E84E845
:1084D00090E09093F40E8093F30E81E08093EE0E83
:1084E00082E78093F50E80EE9EE00E94521980EEA6
:1084F0009EE00E94C91988EC90E026960FB6F89489
:10850000DEBF0FBECDBFDF91CF911F910F910895B8
:108510002F923F924F925F926F927F928F929F9293
:10852000AF92BF92CF92DF92EF92FF920F931F9381
:10853000CF93DF93CDB7DEB7A6970FB6F894DEBF23
:108540000FBECDBF1C010F8B188F298F3A8F4B8F19
:108550005C8F6D8F7E8F22E1E216F10408F035C04A
:10856000F701E953FB4F30813F8FCE0147960E94C0
:10857000D72597FD04C0BC01C1010E946828988DD1
:10858000892F8F70D1011196EC911197E07FE82B24
:108590001196EC9311978F898C93E295EF70EC30E4
:1085A00008F063C0F0E08827E752FD4B8F4F0D9431
:1085B000CC3EDC44024302437A44E742084543444C
:1085C000844484448444434443441F8ECECFB12C1E
:1085D00092959F709D3008F0CDC4E92FF0E0882778
:1085E000EB50FD4B8F4F0D94CC3E354342456245D9
:1085F00042450B450B4542454245BA47BA474245BD
:1086000042450F4492959F709D3008F018C1E92FA4
:10861000F0E08827E15FFC4B8F4F0D94CC3E354353
:10862000ED43E043A3431F431C43C443EF431F44B4
:108630001F44AE43AE430F448E8DF10187838D8D71
:10864000D10116968C9316978C8D15968C93159751
:108650008B8D14968C9314979295907F11968C9194
:1086600011978F70982B11969C93BF8DBB2309F4A3
:1086700067C0F101818182958F702B2F30E08217C6
:10868000130609F45DC06BEA70E187EA9FE00F947E
:10869000CC0BD10111966C9162956F704AE050E05D
:1086A00087EA9FE00F94330A68EA70E187EA9FE067
:1086B0000F94CC0B4AE050E06F8D87EA9FE00F9457
:1086C000330A66EA70E187EA9FE00F94CC0BF10170
:1086D000008119821A821B821C821D821E821F82C7
:1086E00018868F8D8295807F9A819F70892B8A83CF
:1086F0000983EE24EA94FE2C118122813381448186
:10870000558166817781CE0101960E948842D10110
:108710002C9311963C93119712964C9312971396A3
:108720005C93139714966C93149715967C931597F6
:1087300016968C93169717969C93C1010E941A283F
:1087400088E0F10178C18D8D9E8DF101868387814E
:1087500090FB80F987838C8D858387CF8B8D9C8D53
:10876000AD8DBE8DB7FD0EC08F3F9105A105B10542
:1087700029F024F08FEF90E0A0E0B0E0D101149652
:108780008C9373CF80E0FACF6B8D7C8D8D8D9E8D19
:1087900020E06D39BFEF7B078B079B076CF02FEF55
:1087A0006115E4E67E078105910534F424E630E0A6
:1087B00040E050E00F94773ED10114962C9355CFB2
:1087C0008D8D9E8DF1018683878190FB80F9878353
:1087D0008C8D85838B8D848348CF8B8DCFCFCB8C35
:1087E000DC8CED8CFE8C20E030E0A901C701B601E5
:1087F0000F940B3D60E087FD0FC020E030E04FE7B5
:1088000053E4C701B6010F9413406FEF181624F01C
:10881000C701B6010F94E43FF101648326CFD10173
:1088200011968C9111978F70806C11968C93119783
:108830008B8D9C8D15969C938E93149716CF6BE21F
:1088400071E187EA9FE00F94CC0B688D62956F70A1
:108850004AE050E087EA9FE00F94330A68E271E152
:1088600087EA9FE00F94CC0BF101618162956F70F4
:108870004AE050E087EA9FE00F94330A87EA9FE0DE
:108880000F94160AF2CE92959F70933091F09C301F
:1088900031F24B8D5C8D6D8D7E8DF101448355835E
:1088A000668377839295907F81818F70982B9183D7
:1088B000DCCE60E0C1010E942B23D10114968C9381
:1088C00014978D8D9E8D16968C93169717968C9176
:1088D000179790FB80F917968C9317978C8D1596A8
:1088E0008C93159711968C9111978F7080621196C9
:1088F0008C93BBCE60E0CE0147960E942B23D10122
:1089000014968C931497EECF92959F709D3008F03B
:1089100066C0E92FF0E08827EF56FB4B8F4F0D9490
:10892000CC3E3543AC44DB445944DB44DB449E44F9
:10893000CB44CB44CB44BA44C6440F448B8D9C8D6E
:10894000AD8DBE8DF10184839583A683B78381812C
:108950008F708066818389CE6B8D70E090E080E0BF
:108960000F94103DD10114966D937D938D939C933C
:1089700017977BCE6B8D7C8D8D8D9E8D0F94123DC8
:10898000F10164837583868397836FCE6B8D7C8DB5
:108990008D8D9E8DE5CF9295907FF10181818F70B5
:1089A000982B91838B8D9C8DAD8DBE8D848395830B
:1089B000A683B7835ACE9295907FD10111968C9160
:1089C00011978F70982B11969C938B8D9C8DAD8DEC
:1089D000BE8DF10184839583A683B78346CE66E17D
:1089E00071E187EA9FE00F94CC0B688D62956F7000
:1089F0004AE050E087EA9FE00F94330A63E171E1B7
:108A000087EA9FE00F94CC0BD10111966C912ECF89
:108A1000BB24B394DDCD4B8D5C8D6D8D7E8DF101CE
:108A200044835583668377839295907F81818F708D
:108A3000982B918388E0DE01119601900D928A9522
:108A4000E1F729813A814B815C816D817E818F8143
:108A50009885A6960FB6F894DEBF0FBECDBFDF9106
:108A6000CF911F910F91FF90EF90DF90CF90BF902B
:108A7000AF909F908F907F906F905F904F903F90BE
:108A80002F900895963009F442C148F46B8D9130CF
:108A900071F06FEF70E0933051F060E008C09730F4
:108AA00009F441C19A506B8D7C8D9230B0F784E609
:108AB0008D8F8E8D8E7F8E8F1C8E888D8F708062B5
:108AC000888F6B8F2C8D30E0AFEFB0E00F94A93E14
:108AD000C12CD12C7601CA946115F4E67F0781057B
:108AE000910544F424E630E040E050E00F94773EF6
:108AF00069017A0186012B8D28A3622E712CBB207F
:108B000009F475C08E8D8695A82FA150BB0B2D0141
:108B1000BFEF4B165B0609F027C1003811050CF0BA
:108B200009C18FE790E08C199D09869DD001879D32
:108B3000B00D969DB00D11242FEF30E00F94E33E61
:108B400021E83EE740E050E00F94773EF1012783B3
:108B5000ABE9B0E0A70196010F94963EEFE78E2EA9
:108B6000912CA12CB12CA50194010F94773E890181
:108B70009A010C591F4F2F4F3F4FAEEFB1E0A701A5
:108B800096010F94963EA50194010F94773ED30170
:108B90000F94963E2FEF30E040E050E00F94773E88
:108BA00039012FEF6216710421F01CF066246A94DB
:108BB000712C66E071E187EA9FE00F94CC0B4AE0EC
:108BC00050E0B80187EA9FE00F941D0B68EF70E159
:108BD00087EA9FE00F94CC0B4AE050E0B30187EAAC
:108BE0009FE00F941D0B87EA9FE00F94160A30E078
:108BF00020E050E040E070E060E0CE0101960F948C
:108C0000D70DF02E2D8D3E8D3170AFEFBFEF0F944D
:108C1000A93E2DE631E040E050E00F94773E442736
:108C20005527AAEFB5E00F94963EDC01CB01905892
:108C3000AF4FBF4FCD01BB2797FDB095AB2F8E3FF8
:108C4000E1E09E0708F06FC1382F8F3F910508F4CF
:108C50008CC14EEF481B50E03FEFF30131961127D6
:108C60000F5F1F4FF094EF2CF12C309FC001319F0C
:108C7000900D1124292F33272E0D3F1DDF010F9456
:108C8000E33E4B015C018824AA24BB24509F900141
:108C9000519F300D1124232F33272E0D3F1D0F948C
:108CA000E33EBB27A92F982F872F882A992AAA2A23
:108CB000409F9001419F300D1124232F33272E0D0B
:108CC0003F1DDF010F94E33EB82FA72F962F882773
:108CD00088279927BB2788299929AA29F101A683E2
:108CE000958384836CEC70E187EA9FE00F94CC0B52
:108CF000C1010E941A288A859B850F9479358F813E
:108D0000988597FDB2CC60E00E9447E6AECC6B8DB3
:108D10007C8D8D8D9E8D24E630E040E050E00F94F8
:108D2000773EB901C4CE6B8D7C8D8D8D9E8D0F9459
:108D3000DD3FBDCEA70196012058310941095109F7
:108D4000ABE9B0E00F94963E2FE730E040E050E012
:108D50000F94773E89019A010C591F4F2F4F3F4FB7
:108D6000D10117961C9225CF9201AAEBBFEF0F9469
:108D7000DB3E44E6842E912CA12CB12CA50194015C
:108D80000F94773EDA01C9018C599F4FAF4FBF4F07
:108D900089A39AA3ABA3BCA326E430E0D2010F942D
:108DA000E33EA50194010F94773E49015A019EE1EB
:108DB000890E911CA11CB11C003811050CF099C042
:108DC0008FE790E08C199D09869DD001879DB00D9D
:108DD000969DB00D1124A50194010F94A13E9B0115
:108DE000AC01AFEFB0E00F94963E24E63AE640E0E7
:108DF00050E00F94773ED10117962C9329A13AA108
:108E00004BA15CA12C0D3D1D4E1D5F1DAEEFB1E0D1
:108E10000F94963E23EE30E040E050E00F94773E12
:108E200029013A013EA32DA3AFEFB0E0A7019601BF
:108E30000F94963E2FE730E040E050E00F94773EED
:108E40008901E8A1AE2FB0E0A30192010F94963EF4
:108E50002FEF30E040E050E00F94773E39012F3F94
:108E6000310521F01CF066246A94712C62EF70E1E8
:108E700087EA9FE00F94CC0B2AE030E049A15AA189
:108E80006BA17CA187EA9FE00F94D50A6CEE70E19C
:108E900087EA9FE00F94CC0B2AE030E0B501A401F3
:108EA00087EA9FE00F94D50A64EE70E187EA9FE0BD
:108EB0000F94CC0B4AE050E0B80187EA9FE00F9492
:108EC0001D0B6CED70E187EA9FE00F94CC0B4AE03C
:108ED00050E0B30187EA9FE00F941D0B63ED70E152
:108EE00087EA9FE00F94CC0B4AE050E06DA17EA191
:108EF00076CEA70196012058310941095109ABE905
:108F0000B0E00F94963E2FE730E040E050E00F9441
:108F1000773E89019A010C591F4F2F4F3F4FD101C6
:108F200017961C92A3CF8C3FF3E09F0768F48D3F08
:108F300022E0920728F452E0580F3FEF40E08DCE38
:108F40003CEF381B5FEFFACF8A3F35E0930781F0A3
:108F50008B3FE4E09E0728F444E0480F5FEF30E0E9
:108F60007CCE5AEF581B30E001C050E04FEF75CE79
:108F700050E0F9CF6AEB70E187EA9FE00F94CC0BE9
:108F8000688D62956F704AE050E087EA9FE00F9429
:108F9000330A67EB70E134CD2F923F924F925F928C
:108FA0006F927F928F929F92AF92BF92CF92DF92F9
:108FB000EF92FF920F931F93CF93DF93CDB7DEB75E
:108FC000C75CD1090FB6F894DEBF0FBECDBF1C0140
:108FD000CF54DF4F0883C15BD040CE54DF4F18839E
:108FE000C25BD040CD54DF4F2883C35BD040CC540C
:108FF000DF4F3883C45BD040CB54DF4F4883C55B21
:10900000D040CA54DF4F5883C65BD040C954DF4FAD
:109010006883C75BD040C854DF4F7883C85BD040BB
:10902000C754DF4FF982E882C95BD040C254DF4F9A
:10903000C882CE5BD040C154DF4FA882CF5BD04006
:109040000F94FA296B01C054DF4F79836883C05CA9
:10905000D040683C7105B4F463E47CE080E09FE0BC
:109060000F94CC0B4AE050E0B60180E09FE00F94F3
:109070001D0B80E09FE00F94160AAA24AA94BA2C34
:109080000C94ED510E947EEACC53DF4F68837983C4
:109090008A839B83C45CD040CE54DF4F8881C25BFF
:1090A000D0408F70282F30E0C454DF4F398328839D
:1090B000CC5BD0408091E3109091E410CE53DF4F11
:1090C00099838883C25CD040C754DF4FE881F9811F
:1090D000C95BD040309721F0808181110C94E95612
:1090E000D1011B968C91882341F0C1010B96C75486
:1090F000DF4F99838883C95BD040C454DF4FE88138
:10910000F981CC5BD040EF2B11F00C944557C7543C
:10911000DF4FE881F981C95BD040309711F00C94A2
:10912000F256D1015B960D90BC91A02DC454DF4F37
:10913000B983A883CC5BD040AB2B11F40C9445577A
:10914000CE54DF4F8881C25BD0408F7011F00C94F9
:109150004557C454DF4F6881CC5BD040CE018F545B
:109160009F4F0E941C20C756DF4F2883C959D0400B
:10917000C656DF4F3883CA59D040C556DF4F4883A3
:10918000CB59D040C456DF4F5883CC59D040C3563A
:10919000DF4F6883CD59D040C256DF4F7883CE5918
:1091A000D040C156DF4F8883CF59D040C056DF4FE3
:1091B0009883C05AD0400C944557D1012D913C91D1
:1091C000232B09F45ACFC454DF4FE881F981CC5BDB
:1091D000D040349799F5C154DF4FE880CF5BD04041
:1091E000CF54DF4F0881C15BD040CE54DF4F188190
:1091F000C25BD040CD54DF4F2881C35BD040CC54FC
:10920000DF4F3881C45BD040CB54DF4F4881C55B12
:10921000D040CA54DF4F5881C65BD040C954DF4F9D
:109220006881C75BD040C854DF4F7881C85BD040AD
:10923000C1010E94D8245C010C94ED5128E0FE018C
:10924000EF54FF4FDE01A755BF4F01900D922A95B5
:10925000E1F7CF54DF4F1881C15BD040143009F4DF
:1092600012C348F4112309F469C0912C812CAA245B
:10927000AA94BA2C8CC388EF810F8230B0F788E0B3
:10928000FE01EF54FF4FDE01119601900D928A9579
:10929000E1F7CE54DF4F8881C25BD040807F09F474
:1092A00085C3CE018F549F4F0E948B254B015C01DB
:1092B00081149104A104B10409F478C3193041F474
:1092C000B094A09490948094811C911CA11CB11C1A
:1092D000B101CE018F549F4F0E940BDE60E0CE01A2
:1092E0008F549F4F0E9443206A962FAF6A976B96C8
:1092F0003FAF6B976C964FAF6C976D965FAF6D9766
:109300006E966FAF6E976F967FAF6F97A0968FAF89
:10931000A097A1969FAFA197C454DF4FA881B981B0
:10932000CC5BD040A230B10509F49AC30CF044C321
:10933000AB2B09F4D3C3912C812C58C519821A8206
:109340001B821C821D821E821F8218862A812F701A
:109350002A83CE54DF4F2881C25BD040207F09F49E
:1093600084CFC454DF4F08811981CC5BD0400A30D0
:10937000110509F440C254F40115110571F10230D0
:10938000110509F4E1C0912C812C2CC2C454DF4F8B
:1093900028813981CC5BD0402B30310509F4D3C111
:1093A0002C30310581F7B101CE0101960E940BDE10
:1093B000CE018F549F4F0E94D725BC01CE0101964C
:1093C0000E94682888E0FE013196DE01AF54BF4F4D
:1093D00001900D928A95E1F702C2892B59F060E065
:1093E0007CE087EA9FE00F94CC0B87EA9FE00F9424
:1093F000160AC9CFC1010E9462588C0161E070E079
:109400001816190614F070E060E04AE050E087EAB0
:109410009FE00F941D0B6BE678E087EA9FE00F94C6
:10942000660BCE018F549F4F0E949324AB01BC0169
:109430002AE030E087EA9FE00F94D50A87EA9FE0B0
:109440000F94160ACE018F549F4F1016110614F078
:109450000C94D7560E949324672B682B692B09F034
:1094600069C162E0CE018F549F4F0E944320CF56C6
:10947000DF4F2883C159D040CE56DF4F3883C259C1
:10948000D040CD56DF4F4883C359D040CC56DF4F34
:109490005883C459D040CB56DF4F6883C559D0405C
:1094A000CA56DF4F7883C659D040C956DF4F8883EC
:1094B000C759D040C856DF4F9883C859D040882438
:1094C0008394982C31E0C554DF4F3883CB5BD04078
:1094D0005524539442C061E0CE018F549F4F0E94A7
:1094E0004320C757DF4F2883C958D040C657DF4FA6
:1094F0003883CA58D040C557DF4F4883CB58D04037
:10950000C457DF4F5883CC58D040C357DF4F6883D0
:10951000CD58D040C257DF4F7883CE58D040C15786
:10952000DF4F8883CF58D040C057DF4F9883C05952
:10953000D04088248394982C81E0C554DF4F8883E1
:10954000CB5BD040512C09C0912C812CC554DF4FEE
:109550001882CB5BD04055245A94B101CE010196BC
:109560000E940BDE8A81982F92959F70945F9F7066
:10957000923060F4CE54DF4F9881C25BD040929518
:109580009F70923019F48F7080628A83D10118968F
:109590009C91973071F4CE54DF4F8881C25BD040EC
:1095A000807E803211F0803421F48A818F70806255
:1095B0008A83F101A185B285892F90E0109741F04F
:1095C000ED91FC911197048CF58DE02DCD0119954D
:1095D0007C01CF54DF4F0881C15BD040CE54DF4FB8
:1095E0001881C25BD040CD54DF4F2881C35BD0408F
:1095F000CC54DF4F3881C45BD040CB54DF4F48811F
:10960000C55BD040CA54DF4F5881C65BD040C954B7
:10961000DF4F6881C75BD040C854DF4F7881C85B9B
:10962000D040CE0101960E948842CF57DF4F288359
:10963000C158D040CE57DF4F3883C258D040CD57A5
:10964000DF4F4883C358D040CC57DF4F5883C458AE
:10965000D040CB57DF4F6883C558D040CA57DF4F43
:109660007883C658D040C957DF4F8883C758D04049
:10967000C857DF4F9883C858D040CE0101960E944A
:109680001A28C554DF4FF881CB5BD040FF2351F13E
:10969000CE54DF4F8881C25BD04082958F709FE0AF
:1096A000980F9F70923020F08A5F8F708230D0F4D4
:1096B0008A8182958F7081508230A0F42D8130E0B4
:1096C000AFEFB0E00F94A93E2FEF611504E67007ED
:1096D0008105910534F424E630E040E050E00F9439
:1096E000773E2D8388E0FE013196DE01AF54BF4FF7
:1096F00001900D928A95E1F712E1912AF12CAA24AA
:10970000AA94BA2CD10118968C911897873009F039
:109710008DC5C054DF4FE881F981C05CD040EE3583
:10972000F1400CF090C36CEB7BE080E09FE00F9485
:10973000CC0B9FCC912C812C91E0C554DF4F9883AA
:10974000CB5BD040C5CEB101CE0101960E940BDEAD
:10975000CA54DF4F8881C65BD0409A8192959F7032
:1097600039F0923049F0912C812CFF24F3943BC0C6
:109770009A819F7090629A8390E08536910514F0EB
:1097800084E690E08E8388E0FE013196DE01AF54DE
:10979000BF4F01900D928A95E1F762E0CE018F54A0
:1097A0009F4F0E941C20EA962FAFEA97EB963FAF9F
:1097B000EB97EC964FAFEC97ED965FAFED97EE968B
:1097C0006FAFEE97EF967FAFEF97C158DF4F88836B
:1097D000CF57D040C058DF4F9883C058D040812C1D
:1097E000F2E19F2EF12CC554DF4F1882CB5BD040A5
:1097F00055245A9484CFB101CE0101960E940BDE0C
:10980000C954DF4F6881C75BD040C854DF4F7881AF
:10981000C85BD0407170CE0101960E94A328C55448
:10982000DF4F8883CB5BD040912C812CFF24F394B5
:109830008823F1F288E0FE013196DE01AF54BF4F7C
:1098400001900D928A95E1F762E0CE018F549F4F0F
:109850000E941C20E2962FAFE297E3963FAFE3977A
:10986000E4964FAFE497E5965FAFE597E6966FAF66
:10987000E697E7967FAFE797E8968FAFE897E99688
:109880009FAFE997ACCFC454DF4F28813981CC5BBF
:10989000D0402930310509F461C0C1010E946258ED
:1098A0001816190674F562E0CE018F549F4F0E947E
:1098B0004320AA962FAFAA97AB963FAFAB97AC9633
:1098C0004FAFAC97AD965FAFAD97AE966FAFAE971B
:1098D000AF967FAFAF97E0968FAFE097E1969FAFDF
:1098E000E19788248394982CAA24AA94BA2CF12C6A
:1098F00031E0C554DF4F3883CB5BD04055245394BF
:1099000001CF61E0CE018F549F4F0E944320A29669
:109910002FAFA297A3963FAFA397A4964FAFA4975C
:10992000A5965FAFA597A6966FAFA697A7967FAFB0
:10993000A797A8968FAFA897A9969FAFA9978824B5
:109940008394982CAA24AA94BA2CF12C81E0C554B3
:10995000DF4F8883CB5BD040512CD4CE40E050E029
:1099600061E070E0C1010E947A31672B682B692B9E
:10997000A9F040E050E061E070E0C1010E94763063
:109980008824839424E0922EAA24A394B12CF12C51
:10999000C554DF4F1882CB5BD040DDC040E050E0C3
:1099A00061E070E0C1010E949F30EACF95E0892E0E
:1099B000912CA12CB12C82CCC454DF4FE881F981C9
:1099C000CC5BD040EA30F10509F4B3C13B9709F014
:1099D000B2CCCE54DF4F8881C25BD04082958F706D
:1099E000823009F023C2C501B40124E630E040E032
:1099F00050E00F94773ECA54DF4F8881C65BD04059
:109A000090E0280F391F37FF02C030E020E02536F4
:109A1000310514F024E630E0CA54DF4F2883C65BDA
:109A2000D04062E0CE018F549F4F0E941C202A96A6
:109A30002FAF2A972B963FAF2B972C964FAF2C9793
:109A40002D965FAF2D972E966FAF2E972F967FAFE7
:109A50002F9760968FAF609761969FAF6197C3C154
:109A6000C554DF4F1882CB5BD040D10119968D9140
:109A70009C911A97009709F038C018968C9190E045
:109A800000E5402E512C612C712C8530910549F058
:109A9000412C512C3201449721F0412C512C3201A0
:109AA0004A94CE54DF4FE881C25BD040E295EF701C
:109AB000E150EB3008F02EC1F0E08827ED59F24B71
:109AC0008F4F0D94CC3E7D4D7D4D8A4E8A4E8A4EF1
:109AD000574E1D4E1D4E1D4EAE4DAE4DF1E0C554C0
:109AE000DF4FF883CB5BD040C0CFDC01ED91FC9120
:109AF000048CF58DE02D1995C3CFCB54DF4F188121
:109B0000C55BD040C501B40124E630E040E050E040
:109B10000F94773EDA01C901810F911DA11DB11D7E
:109B2000B7FF03C080E090E0DC018F3F9105A10505
:109B3000B10529F024F08FEF90E0A0E0B0E0CB5425
:109B4000DF4F8883C55BD040812C12E1912EF12C30
:109B5000AA24AA94BA2C55245A94D4CDCB54DF4FBE
:109B6000C880D980EA80FB80C55BD040B4E68B1604
:109B70009104A104B104DCF5A4E6B0E0A7019601CC
:109B80000F94963E860E971EA81EB91E41145104CE
:109B900061047104B9F0A30192010F94963E362F2F
:109BA000272FB501A40177FF03C040E050E0BA01C0
:109BB000832E922E5C01481559056A057B0514F425
:109BC0004A015B01CB54DF4F88829982AA82BB8213
:109BD000C55BD040CE54DF4F8881C25BD0408F70D0
:109BE0008066CE54DF4F8883C25BD040ADCFC501C5
:109BF000B40124E630E040E050E00F94773EC20E1E
:109C0000D31EE41EF51E411451046104710461F079
:109C1000F7FE03C0C12CD12C76014C145D046E04F8
:109C20007F0414F473016201CB54DF4FC882D982E0
:109C3000EA82FB82C55BD04087CFCB54DF4F68817F
:109C400079818A819B81C55BD0400F94DD3F6B0198
:109C50007C01C501B40124E630E040E050E00F94FF
:109C6000773ECA01B9016C0D7D1D8E1D9F1D4114EB
:109C700051046104710481F06B017C01F7FE03C0A3
:109C8000C12CD12C7601C701B601461657066806CD
:109C9000790614F4C301B2010F94123DCB54DF4F87
:109CA000688379838A839B83C55BD0404DCFCB5437
:109CB000DF4F88819981AA81BB81C55BD040880E26
:109CC000991EAA1EBB1E4114510461047104C9F0FF
:109CD000A4E6B0E0A30192010F94963E362F272F01
:109CE000B501A40177FF03C040E050E0BA01832E24
:109CF000922E5C01481559056A057B0514F44A014A
:109D00005B01CB54DF4F88829982AA82BB82C55BFC
:109D1000D0401ACF88E0FE013196DE01AF54BF4F2C
:109D200001900D928A95E1F7912C812CFF24F394F8
:109D30000FCFCE54DF4F8881C25BD04082958F70A9
:109D4000823009F055C0C501B40124E630E040E09E
:109D500050E00F94773EC954DF4F8881C75BD040F5
:109D6000C854DF4F6881C85BD040962F9170280F90
:109D7000391F2E36E1E03E072CF437FF05C02DE6F3
:109D800031E002C030E020E0C954DF4F2883C75BD8
:109D9000D040C854DF4F8881C85BD04030FB80F989
:109DA000C854DF4F8883C85BD04062E0CE018F5437
:109DB0009F4F0E941C2062962FAF629763963FAF21
:109DC000639764964FAF649765965FAF65976696A5
:109DD0006FAF669767967FAF679768968FAF689704
:109DE00069969FAF6997812CB2E19B2EF12C18C028
:109DF00088E0FE013196DE01AF54BF4F01900D9215
:109E00008A95E1F764EF7BE080E09FE00F94CC0B54
:109E100080E09FE00F94160A912C812CFF24F3948C
:109E2000C554DF4F1882CB5BD04092CE88E0FE0154
:109E30003196DE01AF54BF4F01900D928A95E1F744
:109E400068EE7BE0E1CFC254DF4F1881CE5BD0409B
:109E5000112309F46FC01296ED91FC9180858F70EB
:109E6000853009F074C0CE53DF4FE881F981C25CC0
:109E7000D040359709F46BC0C1010E94625821E0BF
:109E8000181619060CF020E0522EC754DF4F4881F7
:109E90005981C95BD040C154DF4F2881CF5BD0408E
:109EA000BE016F547F4FD10112968D919C910E94FB
:109EB0009B57C454DF4FE881F981CC5BD040319788
:109EC00009F045C0CE54DF4F8881C25BD040807F0F
:109ED000F1F1C154DF4FC880CF5BD040E52CC755AE
:109EE000DF4F0881C95AD040C655DF4F1881CA5A82
:109EF000D040C555DF4F2881CB5AD040C455DF4FE5
:109F00003881CC5AD040C355DF4F4881CD5AD0401C
:109F1000C255DF4F5881CE5AD040C155DF4F6881BE
:109F2000CF5AD040C055DF4F7881C05BD040C101CF
:109F30000E94B334CF54DF4F8881C15BD04085305D
:109F400009F445C150F48330B9F1D12CC3C0C254D7
:109F5000DF4F1882CE5BD040EDCF863009F482C04F
:109F6000873099F7C1010E94E535182F863009F036
:109F700066C060E97BE087EA9FE00F94CC0B4AE083
:109F800050E066E070E087EA9FE00F941D0B87EADF
:109F90009FE00F94160A62E0CE018F549F4F0E94FB
:109FA000432029AF3AAF4BAF5CAF6DAF7EAF8FAF01
:109FB00021969FAF21973FC0C1010E94E5358530B2
:109FC00021F093E0A92EB12C08C267EA7BE087EA72
:109FD0009FE00F94CC0B4AE050E065E070E087EA28
:109FE0009FE00F941D0B87EA9FE00F94160AB101C2
:109FF000CE018F549F4F0E940BDE61E0CE018F5443
:10A000009F4F0E94432022962FAF229723963FAF67
:10A01000239724964FAF249725965FAF25972696D2
:10A020006FAF269727967FAF279728968FAF2897F1
:10A0300029969FAF2997689480F890F886CF62E7B9
:10A040007BE087EA9FE00F94CC0B612F70E04AE041
:10A0500050E087EA9FE00F941D0B87EA9FE00F9482
:10A06000160AAFCF40E050E061E070E0C1010E940D
:10A070007A31672B682B692B09F0A6C0FFEF5F12BE
:10A080000EC0C1010E946258512C181619064CF4DA
:10A0900068E57BE087EA9FE00F94CC0B92CF5110EC
:10A0A000F7CFB101CE018F549F4F0E940BDE61E0CC
:10A0B000CE018F549F4F0E94432029AB3AAB4BAB4C
:10A0C0005CAB6DAB7EAB8FAB98AF689480F890F8CB
:10A0D000E6E0DE2E84010160CE54DF4F8881C25B52
:10A0E000D040982F9F70923050F4CF54DF4F98811A
:10A0F000C15BD040992319F0840101601160807F19
:10A1000009F489C01260C254DF4F2881CE5BD04071
:10A1100021111D7FA801B101CE018F549F4F0E94D4
:10A12000C8304801AA24A394B12CF110FFC6D10174
:10A1300019968D919C91009709F0A7C340E050E0DB
:10A1400062E070E0C1010E947A31672B682B692BB5
:10A1500009F4CDC364E17AE080E09FE00F94CC0B7A
:10A1600080E09FE00F94160A92FC0CC662E07AE051
:10A1700087EA9FE00F94CC0B4AE050E0B50187EAF4
:10A180009FE00F941D0B6BEF79E087EA9FE00F943F
:10A19000CC0B0E947EEAAB01BC01CC53DF4F08819F
:10A1A00019812A813B81C45CD040401B510B620B5A
:10A1B000730B2AE030E087EA9FE00F94310A87EAC8
:10A1C0009FE00F94160A09C163E47BE063CF0FEFB1
:10A1D00050120BC0C1010E946258552453941816A6
:10A1E00019062CF066E27BE055CF5520D9F362E0EA
:10A1F000CE018F549F4F0E94432029A73AA74BA717
:10A200005CA76DA77EA78FA798AB689480F890F89D
:10A2100075E0D72E5FCF40E052E0B101CE018F5400
:10A220009F4F0E94F23581116DCF6DCF3FEF5312DA
:10A230009DC0C1010E9462585524539418161906F6
:10A240000CF497C0512C68E17BE087EA9FE00F9403
:10A25000CC0B052D052C000C110BC054DF4F1983BE
:10A260000883C05CD0404AE050E0B80187EA9FE034
:10A270000F941D0B61E17BE087EA9FE00F94CC0B0C
:10A28000C554DF4F1881CB5BD040612F70E04AE0AE
:10A2900050E087EA9FE00F941D0B87EA9FE00F9440
:10A2A000160AC754DF4F08811981C95BD0400115D8
:10A2B000110509F4B7C06BE87EE0C8010F941637AA
:10A2C000CC24C394D12C892B09F45DC064E97EE0D1
:10A2D000C8010F94163742E0C42ED12C892B09F403
:10A2E00052C06FEA7EE0C8010F94163735E0C32EE6
:10A2F000D12C892B09F447C068EB7EE0C8010F948C
:10A30000163726E0C22ED12C892BE9F16DE27FE0D1
:10A31000C8010F941637892B99F166E37FE0C801D5
:10A320000F941637892B09F473C060E07FE0C801F1
:10A330000F941637BEE0CB2ED12C892B21F169E08A
:10A340007FE0C8010F941637AFE0CA2ED12C892BBD
:10A35000D1F06FE37FE0C8010F941637D12CC12CE8
:10A36000892B89F4F5E1CF2ED12C0DC0552009F4AD
:10A370006ACF81E0C554DF4F8883CB5BD04063CF89
:10A3800093E1C92ED12CC1010E94E535682E712CB4
:10A390006114710431F4C054DF4F68807980C05C6F
:10A3A000D040C114D10409F486C06C147D04A1F11D
:10A3B00065EF7AE087EA9FE00F94CC0B4AE050E02B
:10A3C000B30187EA9FE00F941D0B87EA9FE00F948B
:10A3D000160AEDEFAE2EBB24BA94C501C953DF4F68
:10A3E0000FB6F894DEBF0FBECDBFDF91CF911F91A6
:10A3F0000F91FF90EF90DF90CF90BF90AF909F9024
:10A400008F907F906F905F904F903F902F90089526
:10A4100084E1C82ED12CB7CFC754DF4F19821882E0
:10A42000C95BD040C454DF4FE881F981CC5BD04098
:10A430003197A9F4C254DF4FF881CE5BD040FF239F
:10A4400099F0CE54DF4F8881C25BD040807F01E01D
:10A45000C254DF4F0883CE5BD040811105C0C25487
:10A46000DF4F1882CE5BD040CF54DF4FD880C15B26
:10A47000D04015E11D1508F4E7C1ED2DF0E0882767
:10A48000EB5BFD4A8F4F0D94CC3E9E52D653BC538E
:10A49000DD529E529D53635328539E529E52105438
:10A4A0001A5438543854F053F05324542454245438
:10A4B000F053F053F053D10119968D919C91009770
:10A4C00009F4B0CFDC01ED91FC910488F589E02D11
:10A4D000C154DF4FA880CF5BD040C554DF4FC88048
:10A4E000CB5BD0407801CF54DF4F0881C15BD040B7
:10A4F000CE54DF4F1881C25BD040CD54DF4F28814E
:10A50000C35BD040CC54DF4F3881C45BD040CB54C8
:10A51000DF4F4881C55BD040CA54DF4F5881C65BCE
:10A52000D040C954DF4F6881C75BD040C854DF4F6B
:10A530007881C85BD04019950C941B49D12CC2542A
:10A54000DF4F8881CE5BD040882309F4EECDC15423
:10A55000DF4FC880CF5BD040952D9170E92EC75555
:10A56000DF4F0881C95AD040C655DF4F1881CA5AFB
:10A57000D040C555DF4F2881CB5AD040C455DF4F5E
:10A580003881CC5AD040C355DF4F4881CD5AD04096
:10A59000C255DF4F5881CE5AD040C155DF4F688138
:10A5A000CF5AD040C055DF4F7881C05BD040C10149
:10A5B0000E94B334E89491F8B8CDC1010E94E5350A
:10A5C000853009F0FECC60EE7AE087EA9FE00F94D8
:10A5D000CC0B4AE050E065E070E087EA9FE00F9422
:10A5E0001D0B87EA9FE00F94160AB101CE018F542C
:10A5F0009F4F0E940BDED10118968C918530C9F4D3
:10A600006EE0CE018F549F4F0E94432029A33AA3AE
:10A610004BA35CA36DA37EA38FA398A7689480F837
:10A6200090F8D12CB1E0C554DF4FB883CB5BD0405C
:10A6300086CF61E0CE018F549F4F0E944320298F27
:10A640003A8F4B8F5C8F6D8F7E8F8F8F98A3E6CF65
:10A65000C1010E94E535182F863091F569EC7AE04A
:10A6600087EA9FE00F94CC0B4AE050E066E070E090
:10A6700087EA9FE00F941D0B87EA9FE00F94160A6C
:10A6800062E0CE018F549F4F0E944320298B3A8B6A
:10A690004B8B5C8B6D8B7E8B8F8B988F40E050E06B
:10A6A00068E070E0C1010E947630689480F890F80C
:10A6B000D12CE1E0C554DF4FE883CB5BD0403FCFE6
:10A6C0006BEA7AE0BECC40E050E061E070E0C101AE
:10A6D0000E947A31672B682B692B61F5511027C0D6
:10A6E000B101CE018F549F4F0E940BDE61E0CE017D
:10A6F0008F549F4F0E94432029873A874B875C875E
:10A700006D877E878F87988B40E050E068E070E02F
:10A71000C1010E949F30689480F890F876E0D72EAF
:10A72000F1E0C554DF4FF883CB5BD04008CF61E93F
:10A730007AE0B0CC6CE77AE0ADCC5520D1F062E0A5
:10A74000CE018F549F4F0E94432029833A834B832D
:10A750005C836D837E838F839887689480F890F8FC
:10A7600065E0D62E01E0C554DF4F0883CB5BD040B7
:10A77000E6CE6FE57AE08ECCCE54DF4F8881C25BA7
:10A78000D0408F70D12C823068F7C1010E94E5352E
:10A79000689480F890F8853009F413CCD12C11E03E
:10A7A000C554DF4F1883CB5BD040C9CECE54DF4FAA
:10A7B0008881C25BD0408F70823080F7552081F055
:10A7C00066E47AE087EA9FE00F94CC0B61E0C10178
:10A7D0000E947C1B60E071E1C1010E948536F1CBD3
:10A7E000CE54DF4F8881C25BD040982F9F7092304B
:10A7F00008F043C0DD2069F0807F31F4B101CE0163
:10A800008F549F4F0E940BDE689480F823E0922AB9
:10A81000D12C31E0C554DF4F3883CB5BD0408FCE95
:10A82000689492F8D12C81E0C554DF4F8883CB5BCC
:10A83000D04085CE689492F8D12C91E0C554DF4F7A
:10A840009883CB5BD0407BCECE54DF4F8881C25BF8
:10A85000D040807F51F4689490F8D12CA1E0C55489
:10A86000DF4FA883CB5BD0406ACEB3E09B2A20CFDA
:10A87000D12C812C54E0952E53CFD12C21E0C554FE
:10A88000DF4F2883CB5BD0405ACEDC01ED91FC91A9
:10A89000008CF18DE02DCF54DF4F0881C15BD0409B
:10A8A000CE54DF4F1881C25BD040CD54DF4F28819A
:10A8B000C35BD040CC54DF4F3881C45BD040CB5415
:10A8C000DF4F4881C55BD040CA54DF4F5881C65B1B
:10A8D000D040C954DF4F6881C75BD040C854DF4FB8
:10A8E0007881C85BD0401995811128CC33CCF10117
:10A8F00081859285892B09F473C08114910439F004
:10A90000A401B101CE018F549F4F0E94C830D101E4
:10A9100019968D919C91C754DF4FE880F980C95BEF
:10A92000D040DC01ED91FC910488F589E02DC15403
:10A93000DF4FA880CF5BD040C554DF4FC880CB5BD2
:10A94000D040CF54DF4F0881C15BD040CE54DF4FA1
:10A950001881C25BD040CD54DF4F2881C35BD0400B
:10A96000CC54DF4F3881C45BD040CB54DF4F48819B
:10A97000C55BD040CA54DF4F5881C65BD040C95434
:10A98000DF4F6881C75BD040C854DF4F7881C85B18
:10A99000D04019955C01F10181859285DC01ED9132
:10A9A000FC91048CF58DE02D1995059711F46894B0
:10A9B00080F892FC2CC1DD2021F06D2DC1010E9498
:10A9C0007C1BCE53DF4F08811981C25CD040B4019B
:10A9D0000530110509F4CACBC1010E948536C6CBEA
:10A9E0008085863009F477C008F5843009F417C1F2
:10A9F000853009F78114910439F0A401B101CE0129
:10AA00008F549F4F0E94C830C454DF4F0881198172
:10AA1000CC5BD0400230110509F4FDC003301105B4
:10AA200009F4D2C00130110531F6CAC0883009F4EA
:10AA30005AC1893009F0BFCF8114910439F0A401C3
:10AA4000B101CE018F549F4F0E94C830C554DF4FD3
:10AA5000E881CB5BD040EE2309F4ADCF552079F0EF
:10AA6000CF54DF4F8881C15BD040813041F4CE5458
:10AA7000DF4F8881C25BD040807F09F49CCFCF54E8
:10AA8000DF4F0881C15BD040CE54DF4F1881C25BDD
:10AA9000D040CD54DF4F2881C35BD040CC54DF4F32
:10AAA0003881C45BD040CB54DF4F4881C55BD04078
:10AAB000CA54DF4F5881C65BD040C954DF4F68810C
:10AAC000C75BD040C854DF4F7881C85BD040C1011C
:10AAD0000E94333FF2C0CF54DF4FF880C15BD040BB
:10AAE000FF2009F487CF70E060E0C1010E94612E71
:10AAF0008C018114910439F0A401B101CE018F546D
:10AB00009F4F0E94C8300115110509F454CF712CD4
:10AB1000612C17FF06C011950195110966246394F5
:10AB2000712CC80101978634910508F044CFE02EBE
:10AB300061E0802F0E9447E6EFEFEF0DE53110F561
:10AB4000F0E08827E955FA4A8F4F0D94CC3EBC556A
:10AB5000BE55C255C255BE55BC55BE55C255C2554F
:10AB6000C255C255C255C255BC55BC55C255C25539
:10AB7000C255C255BC55BC55F1E06F26662D8E2DD1
:10AB80000E9419E66FE07AE087EA9FE00F94CC0B11
:10AB90004AE050E0B80187EA9FE00F941D0B6DE09A
:10ABA0007AE087EA9FE00F94CC0B4AE050E0B301D3
:10ABB00087EA9FE00F941D0B87EA9FE00F94160A27
:10ABC000689480F890F823C0C1010E94FF2D892B62
:10ABD00049F4D101ED91FC916081718187E896E0A3
:10ABE0000E9436EBCE018F549F4F0E944C2420E0F0
:10ABF00030E048EC52E40F94713D0F94DD3F2B019F
:10AC000088E00F945B28A201C1010E94BE2DAA24F6
:10AC1000A394B12CD0CE689480F891F8F8CF811429
:10AC2000910439F0A401B101CE018F549F4F0E94CD
:10AC3000C830C554DF4FB881CB5BD040BB2309F48B
:10AC4000BACECF54DF4F8881C15BD0405520B9F1D7
:10AC5000813041F4CE54DF4F8881C25BD040807F89
:10AC600009F4A9CECF54DF4F0881C15BD040CE5448
:10AC7000DF4F1881C25BD040CD54DF4F2881C35BCA
:10AC8000D040CC54DF4F3881C45BD040CB54DF4F31
:10AC90004881C55BD040CA54DF4F5881C65BD04065
:10ACA000C954DF4F6881C75BD040C854DF4F7881FB
:10ACB000C85BD040C1010E94633D5C017CCE813005
:10ACC00089F6CE018F549F4F0E94A6D8449750F624
:10ACD0006EE170E0CE018F549F4F0E94F82368947C
:10ACE00080F891F8BFCF8114910439F0A401B1012B
:10ACF000CE018F549F4F0E94C830C554DF4FF8815A
:10AD0000CB5BD040FF2309F456CE552079F0CF54C9
:10AD1000DF4F8881C15BD040813041F4CE54DF4F9A
:10AD20008881C25BD040807F09F445CECF54DF4F8D
:10AD30000881C15BD040CE54DF4F1881C25BD04048
:10AD4000CD54DF4F2881C35BD040CC54DF4F3881D6
:10AD5000C45BD040CB54DF4F4881C55BD040CA5460
:10AD6000DF4F5881C65BD040C954DF4F6881C75B55
:10AD7000D040C854DF4F7881C85BD040C1010E94E9
:10AD80001C3E9BCFCE53DF4F28813981C25CD0401F
:10AD90002530310509F4EAC940E054E0B101CE01A3
:10ADA0008F549F4F0E94C83060E074E015CE0E941F
:10ADB0009324672B682B692B11F00C946B4A912C10
:10ADC000812C11E0C554DF4F1883CB5BD0400C942D
:10ADD000A24AC454DF4F28813981CC5BD040232B59
:10ADE00009F053C08081882311F40C949148CE015E
:10ADF00087549F4F0E94392DC454DF4F9983888315
:10AE0000CC5BD040CE54DF4F8881C25BD0408F7086
:10AE100091F5C454DF4F6881CC5BD040CE018F5494
:10AE20009F4F0E941C20CF55DF4F2883C15AD0402E
:10AE3000CE55DF4F3883C25AD040CD55DF4F4883BF
:10AE4000C35AD040CC55DF4F5883C45AD040CB555D
:10AE5000DF4F6883C55AD040CA55DF4F7883C65A42
:10AE6000D040C955DF4F8883C75AD040C855DF4FFF
:10AE70009883C85AD040C454DF4FE881F981CC5B35
:10AE8000D040EF2B11F40C94914868E37CE087EA02
:10AE90009FE00F94CC0B4AE050E0B60187EA9FE0B8
:10AEA0000F941D0B61E37CE087EA9FE00F94CC0BCD
:10AEB000D101ED91FC916081718187EA9FE00F944F
:10AEC000660B6BE27CE087EA9FE00F94CC0BC754E3
:10AED000DF4F68817981C95BD04087EA9FE00F949A
:10AEE000660B69E27CE087EA9FE00F94CC0BCE0111
:10AEF0008F549F4F0E941A28C754DF4F8881998131
:10AF0000C95BD040009711F40C94DD48FC0120810E
:10AF1000243211F00C94DD4865E17CE087EA9FE083
:10AF20000F94CC0B87EA9FE00F94160A8CEFA82EA3
:10AF3000BB24BA9452CA2F923F924F925F926F9263
:10AF40007F928F929F92AF92CF92DF92EF92FF9279
:10AF50000F931F93CF93DF93CDB7DEB76D970FB6E7
:10AF6000F894DEBF0FBECDBF009709F4A9C0FC0165
:10AF700030853F70353009F0A3C0D22E1A014B0145
:10AF8000668077808091DF108F5F8093DF1061147F
:10AF9000710409F490C0F30180858F70843009F04A
:10AFA00086C0618572858091E5109091E6100E94BF
:10AFB000E5D72C01009709F47AC0FC0180858F70D9
:10AFC000853009F074C0B201CE0101960E94D23AD8
:10AFD00081149104B1F0CE0101960E946F2D882357
:10AFE00081F0AD2CC12C7101F4010081118122810D
:10AFF00033814481558166817781CE0101960E941B
:10B00000CC4760E0C2010E9497D80097E9F1FC01AB
:10B0100020852F702230C1F581859285A385B48566
:10B020000797A105B10581F561E0C2010E9497D89B
:10B030002D2DA101B4010E949B578114910499F513
:10B04000882389F18091DF1081508093DF10CE0139
:10B0500001960E94743981E06D960FB6F894DEBFB8
:10B060000FBECDBFDF91CF911F910F91FF90EF9059
:10B07000DF90CF90AF909F908F907F906F905F9078
:10B080004F903F902F9008958114910461F4CE0168
:10B0900001960E946F2D882331F0CE0101960E9407
:10B0A0006258892B79F6CE0101960E947439F3011A
:10B0B000628073806CCF8091DF1081508093DF10AD
:10B0C00080E0CACFDF92EF92FF920F931F93CF934E
:10B0D000DF9300D000D01F921F92CDB7DEB77C0166
:10B0E00019821A821B821C821D821E821F82188670
:10B0F0008A818F708A83D701ED91FC916081718183
:10B1000087EA9FE00F94660B64E87CE087EA9FE0A3
:10B110000F94CC0BC7010E946F2D81111BC06BE7F0
:10B120007CE087EA9FE00F94CC0B87EA9FE00F94C6
:10B13000160A0FEF1FEFC80128960FB6F894DEBF6E
:10B140000FBECDBFDF91CF911F910F91FF90EF9078
:10B15000DF900895C7010E94E535D82EF70181855B
:10B160009285009791F0DC01ED91FC910688F789BA
:10B17000E02D19958C0197FD08C081E0011511059E
:10B1800009F480E00E94BF19D6CFF701808587308F
:10B1900009F42EC0EFEFED0DE43150F5F0E0882713
:10B1A000EB52F74A8F4F0D94CC3EE958F258F858BD
:10B1B000F858F258E958F858F858F858F858F85824
:10B1C000F858F858E958F858F858F858F858E9581D
:10B1D000E9586CE57CE087EA9FE00F94CC0B01E036
:10B1E00010E0A9CF80E00E94BF1910E000E0A3CFDB
:10B1F00040E052E0B701CE0101960E94F235D7013E
:10B2000018968C911897873089F160F4833009F48F
:10B2100057C0843061F06CE67CE087EA9FE00F94D1
:10B22000CC0BE3CF883009F44BC08930A1F760E044
:10B23000CE0101960E942B238C0161E67CE087EA17
:10B240009FE00F94CC0B4AE050E0B80187EA9FE002
:10B250000F941D0B87EA9FE00F94160A91E080E09F
:10B26000012B09F490E0092F182F65CF1296ED916C
:10B27000FC9180858F7010E000E08530F1F669E781
:10B280007CE087EA9FE00F94CC0B20E050E040E0A8
:10B2900070E060E0F701828193810E949B57F82E55
:10B2A000082F10E066E77CE087EA9FE00F94CC0B64
:10B2B0008F2D0E94BF1987EA9FE00F94160A3BCF9B
:10B2C000CE0101960E9493248B01B7CFAF92CF920B
:10B2D000EF92FF920F931F93CF93DF9300D000D094
:10B2E0001F921F92CDB7DEB719821A821B821C8271
:10B2F0001D821E821F8218861A811F70A12CCC24E9
:10B30000C394F12CE12C02E02B813C8140E05E8172
:10B310006F8178850E94CC4728960FB6F894DEBFDF
:10B320000FBECDBFDF91CF911F910F91FF90EF9096
:10B33000CF90AF9008952F923F924F925F926F926D
:10B340007F928F929F92AF92BF92CF92DF92EF92B5
:10B35000FF920F931F93CF93DF93CDB7DEB7CA55FC
:10B36000D1090FB6F894DEBF0FBECDBF4C013B0133
:10B3700040E058E060E070E00E947A31672B682B73
:10B38000692B09F45CC019821A821B821C821D82FF
:10B390001E821F8218868A818F708A8340E053E064
:10B3A000B401CE0101960E94F235D40119968D9117
:10B3B0009C91892B09F41AC140E058E060E070E0EC
:10B3C000C4010E94763061ED7CE087EA9FE00F9433
:10B3D000CC0BF40181859285DC01ED91FC91048810
:10B3E000F589E02DA12CCC24C394F12CE12C09810A
:10B3F0001A812B813C814D815E816F817885199501
:10B40000D401ED91FC918F3F9807C9F06081718163
:10B41000892B09F055C187EA9FE00F94660B64E918
:10B420007CE087EA9FE00F94CC0B6CE87CE087EA35
:10B430009FE00F94CC0B87EA9FE00F94160A65E01B
:10B44000F401808191810E9497D85C01009709F4F2
:10B450006FC1DC011896BC916996BFAF6997B29530
:10B46000BF706896BFAF6897FC0121843284438423
:10B4700054840E947EEA6896FFAD6897FF2309F422
:10B4800057C1261A370A480A590A19A21AA21BA23A
:10B490001CA21DA21EA21FA218A68AA18F70806BDB
:10B4A0008AA3F9A3B201A101CE0181960E94A9222B
:10B4B0002F962FAF2F9760963FAF609761964FAF53
:10B4C000619762965FAF629763966FAF639764967A
:10B4D0007FAF649765968FAF659766969FAF6697C7
:10B4E00024E06216710451F5D12CC12CE12C50E2FC
:10B4F000F52E09A11AA12BA13CA14DA15EA16FA11E
:10B5000078A5C4010E949E31C201B10128EE33E04A
:10B5100040E050E00F94773EBA01A9012AE030E004
:10B5200087EA9FE00F94D50A61EE7DE087EA9FE00D
:10B530000F94CC0B87EA9FE00F94160A57FEF8C0D1
:10B5400082E028163104410480E858060CF4F0C06B
:10B550000F94FA291B016B967FAF6EAF6B97D12CBE
:10B56000C12CE12C40E2F42E09A11AA12BA13CA18F
:10B570004DA15EA16FA178A5C4010E949E316B967A
:10B58000AEADBFAD6B97A83CB1050CF0A6C068ECA2
:10B590007DE080E09FE00F94CC0B4AE050E0B101E9
:10B5A00080E09FE00F941D0B80E09FE00F94160A4F
:10B5B00066246A94762CC301C65ADF4F0FB6F894FE
:10B5C000DEBF0FBECDBFDF91CF911F910F91FF90D6
:10B5D000EF90DF90CF90BF90AF909F908F907F9033
:10B5E0006F905F904F903F902F900895F401808569
:10B5F000883009F445C0893019F1843009F01FCF33
:10B600008091B60A9091B70A892B09F018CF40E0D3
:10B6100058E060E070E0C4010E9476306CEB7CE0A2
:10B6200087EA9FE00F94CC0B09811A812B813C8122
:10B630004D815E816F817885C4010E94633DE0CEBB
:10B640008091B60A9091B70A892B09F0F8CE40E0B4
:10B6500058E060E070E0C4010E9476306BEA7CE064
:10B6600087EA9FE00F94CC0B09811A812B813C81E2
:10B670004D815E816F817885C4010E94333FC0CEC9
:10B680008091B60A9091B70A892B09F0D8CE40E094
:10B6900058E060E070E0C4010E94763066E97CE02A
:10B6A00087EA9FE00F94CC0B09811A812B813C81A2
:10B6B0004D815E816F817885C4010E941C3EA0CEC1
:10B6C00087EA9FE00F94660B6AE87CE087EA9FE0D8
:10B6D0000F94CC0B66E87CE0AACEF50180858F70D4
:10B6E000808719821A821B821C821D821E821F8201
:10B6F00018868A818F708A836896FFAD6897F98370
:10B7000069968FAD69978F70AA24A394873009F04A
:10B71000A12CCC24C394F12CE12C09811A812B811A
:10B720003C814D815E816F817885C4010E94CC4748
:10B7300021E06216710459F4D40118968C9184307A
:10B7400079F0893009F470C1C4010E94F736F40120
:10B7500081859285009709F0A0C4712C612C2BCFB4
:10B760008091B60A9091B70A892BB9F4F40142800E
:10B770005380D20118968C918F70853041F4C201AC
:10B780000E9429D9082F10E00230110554F460E31B
:10B790007DE087EA9FE00F94CC0BC4010E94F7364E
:10B7A0000ACF7092B70A6092B60A70E060E0C401F6
:10B7B0000E94612E1C0161E070E0C4010E94612EB4
:10B7C0005C01053011050CF440C064E0C2010E9428
:10B7D00097D8FC010185128526E040E855E260E03B
:10B7E00070E08BE49CE00F94190D20924B0D8BE4DC
:10B7F0009CE090934A0D8093490D1092560E109242
:10B80000580E1092570E6CE17DE087EA9FE00F948E
:10B81000CC0BD401ED91FC916081718187EA9FE0AE
:10B820000F94660B87EA9FE00F94160A013011050A
:10B8300009F4C2C06CF4012B09F4B3C060E07DE0F0
:10B8400087EA9FE00F94CC0B25C002E010E0C4CF44
:10B850000230110579F00330110581F7B0924D0DDA
:10B86000A0924C0D81E090E090934F0D80934E0D8F
:10B8700084E00BC0B0924D0DA0924C0D81E090E0A1
:10B8800090934F0D80934E0D83E00E94A4EB67963A
:10B890008FAF67976796BFAD6797B11197C000915B
:10B8A000500D1091510D6BEF7CE087EA9FE00F94F3
:10B8B000CC0BD401ED91FC916081718187EA9FE00E
:10B8C0000F94660B64EF7CE087EA9FE00F94CC0B4B
:10B8D000C801012E000CAA0BBB0B89839A83AB8392
:10B8E000BC8380E190E09E838D83BE016F5F7F4FBC
:10B8F00087EA9FE00E94E83A0F94160AB801C40153
:10B900000E94D937E091AF0AF091B00A6281738149
:10B91000CE0101960E94D23A8091AF0A9091B00A6E
:10B92000892BB1F1CE0101960E946F2D882381F100
:10B930008985843069F570E060E0CE0101960E944F
:10B94000612E2816390621F561E070E0CE010196DE
:10B950000E94612EA816B906D9F4B801CE0101964D
:10B960000E94D937E091AF0AF091B00A82819381A9
:10B970009093B00A8093AF0A892B51F4E091E510BF
:10B98000F091E610868197819093B00A8093AF0A78
:10B99000CE0101960E9474391092B70A1092B60A2D
:10B9A000FCCEB0924D0DA0924C0D81E090E09093B2
:10B9B0004F0D80934E0D69CFB0924D0DA0924C0D5E
:10B9C00010934F0D00934E0D82E05FCF67EE7CE049
:10B9D00087EA9FE00F94CC0BD401ED91FC9160813C
:10B9E000718187EA9FE00F94660B6FED7CE087EA38
:10B9F0009FE00F94CC0B6796EFAD67978E2F90E08A
:10BA0000B0E0A0E089839A83AB83BC8380E190E0BF
:10BA10009E838D83BE016F5F7F4F87EA9FE00E9408
:10BA2000E83A0F94160AB8CF8091B60A9091B70AF7
:10BA3000892B09F0B2CE7092B70A6092B60A0F94C1
:10BA4000EF122C01009741F0DC0118968C911897A9
:10BA5000807F866018968C93F20180858F70808736
:10BA600030E020E043E050E060E2CE0101960F9428
:10BA70007928D401ED91FC91608171814FE150E012
:10BA8000CE0101960F94494366E976E0CE01019616
:10BA90000F94234326E040E855E260E070E08BE439
:10BAA0009CE00F94190D70E060E0C4010E94612ECB
:10BAB00080934B0D8BE49CE090934A0D8093490D4D
:10BAC0001092560E1092580E1092570E68EB7DE0B1
:10BAD00087EA9FE00F94CC0BD401ED91FC9160813B
:10BAE000718187EA9FE00F94660B87EA9FE00F94CD
:10BAF000160A62E370E080E090E00E948CE884E344
:10BB000098E090934D0D80934C0D8AE090E09093D7
:10BB10004F0D80934E0D83E00E94A4EB182F8111EE
:10BB200054C26BEA7DE087EA9FE00F94CC0B00E5FE
:10BB30001DE094E6292E9DE0392E20E1A22EB12CA5
:10BB4000F801819191918F01092E000CAA0BBB0B7A
:10BB500089A39AA3ABA3BCA3BEA2ADA2BE016F5D95
:10BB60007F4F87EA9FE00E94E83A69EA7DE00F9400
:10BB7000CC0B2016310621F787EA9FE00F94160AB6
:10BB80006091540D7091550D90E080E00F94123D3E
:10BB900020E030E048EC52E40F946B3F9B01AC0195
:10BBA00062E178E0C2010E9479E3C090580DD09024
:10BBB000590DF12CE12CA70196016CE976E0C20148
:10BBC0000E94A2DE60915A0D70915B0D90E080E0C2
:10BBD0000F94123D20E030E048EC52E40F946B3FAC
:10BBE0009B01AC0160EA76E0C2010E9479E36091BA
:10BBF0005C0D70915D0D90E080E00F94123D20E0AF
:10BC000030E040E251E40F946B3F9B01AC016EE9E0
:10BC100076E0C2010E9479E32091500D3091510DE0
:10BC200050E040E062EA76E0C2010E94A2DECD2848
:10BC3000CE28CF2809F47AC0D4011296ED91FC9158
:10BC400090859F70953009F071C061E0CF010E942E
:10BC500097D8009709F46AC0FC0120852F70243022
:10BC600009F064C061857285CE0181960E94E83832
:10BC7000CE0181960E946F2D882309F453C022962D
:10BC80001CAE1DAE1EAE1FAE229726961CAE1DAE7C
:10BC90001EAE1FAE26978FAD8F7080618FAF8FEF76
:10BCA00023968FAF239724965FAD249725963FADBB
:10BCB000259726962FAD26979EAD7FAD21966FAD29
:10BCC000219722964FAD2297092F27969FAF27974E
:10BCD00028967FAF289729966FAF29972A964FAF5E
:10BCE0002A97482F2B968FAF2B972C965FAF2C97C8
:10BCF0002D963FAF2D972E962FAF2E97A12CCC24AB
:10BD0000C394F12CE12C172F262F2A963FAD2A97AA
:10BD10002D966FAD2D972E967FAD2E97CE018196E5
:10BD20000E94CC47CE0181960E9474398091500DBB
:10BD300083FF76C16EE77DE087EA9FE00F94CC0B2E
:10BD4000D401ED91FC916081718187EA9FE00F94AD
:10BD5000660B87EA9FE00F94160A62E370E080E0CA
:10BD600090E00E948CE88EE398E090934D0D8093D4
:10BD70004C0D81E090E090934F0D80934E0D83E049
:10BD80000E94A4EB81110BC02091500D3091510DF8
:10BD900050E040E065EA76E0C2010E94A2DE109227
:10BDA000B70A1092B60AC4010E9462581816190602
:10BDB0001CF4C4010E94665981E090E09093B70A98
:10BDC0008093B60A6EE67DE087EA9FE00F94CC0B85
:10BDD000D401ED91FC916081718187EA9FE00F941D
:10BDE000660B87EA9FE00F94160A62E370E080E03A
:10BDF00090E00E948CE883E190E090934D0D809359
:10BE00004C0D84E090E090934F0D80934E0D83E0B5
:10BE10000E94A4EB182F811115C161E67DE087EA2D
:10BE20009FE00F94CC0B00E51DE088E5E82E8DE047
:10BE3000F82EF801619171918F014AE050E087EA94
:10BE40009FE00F941D0B6FE57DE087EA9FE00F9464
:10BE5000CC0BE016F10669F787EA9FE00F94160A0B
:10BE60000091500D1091510D01151105D1F0B8013F
:10BE7000012E000C880B990B0F94123D2DEE3EE91C
:10BE80004CE35EE30F94713D22E538EB42E152E46E
:10BE90000F94FE3E9B01AC0169EC77E0C2010E9469
:10BEA00079E36091520D7091530D072E000C880BB1
:10BEB000990B0F94123D2DEE3EE94CE35EE30F9497
:10BEC000713D22E538EB42E152E40F94FE3E6B01F6
:10BED0007C01AC019B016AE976E0C2010E9479E332
:10BEE0006091560D7091570D161617060CF0A1C0F3
:10BEF000072E000C880B990B0F94123D20E030E0C8
:10BF000040E251E40F946B3F9B01AC0169EA76E09B
:10BF1000C2010E9479E320E030E040E252E4C70130
:10BF2000B6010F9413401816B4F4012BA1F00E942F
:10BF300003D8882369F08091C910811109C0D40108
:10BF4000ED91FC91608171818DEA96E00E9436EB63
:10BF5000C4010E94665980E091E00F94DD348C01A9
:10BF6000892BD9F01CA21BA21EA21DA28FEF9FEF4E
:10BF700098A78FA38BEE92E09AA389A31AA619A67D
:10BF80001CA70BA780E091E098AB8FA71EA61DA66B
:10BF9000B201CE0181960F94DF100E9403D888234E
:10BFA00049F08091C910811105C0B801CE010196F8
:10BFB0000E9436EBC8010F9479354114510409F4FD
:10BFC000EBCCC2010E944DE3E7CC6CE97DE087EA4F
:10BFD0009FE00F94CC0BD401ED91FC9160817181B5
:10BFE00087EA9FE00F94660B64E97DE087EA9FE0B3
:10BFF0000F94CC0B812F90E0B0E0A0E089A39AA32E
:10C00000ABA3BCA380E190E09EA38DA3BE016F5DB6
:10C010007F4F87EA9FE00E94E83A0F94160A86CE87
:10C0200020E030E0A90165EA76E0C2010E94A2DECC
:10C03000C9CE20E030E0A90169EA76E0C2010E94A1
:10C04000A2DE69CF6FE47DE087EA9FE00F94CC0B1E
:10C05000D401ED91FC916081718187EA9FE00F949A
:10C06000660B67E47DE087EA9FE00F94CC0B812F9D
:10C0700090E0B0E0A0E089A39AA3ABA3BCA380E1C9
:10C0800090E09EA38DA3BE016F5D7F4F87EA9FE086
:10C090000E94E83A0F94160A5ECFDC01ED91FC9104
:10C0A0000284F385E02D1995892B09F456CBF40110
:10C0B00081859285DC01ED91FC910480F581E02D74
:10C0C000B30119953C0177CA2F923F924F925F922C
:10C0D0006F927F928F929F92AF92BF92CF92DF9298
:10C0E000EF92FF920F931F93CF93DF93CDB7DEB7FD
:10C0F000CE57D1090FB6F894DEBF0FBECDBFDC011D
:10C1000014962D913C911597232B11F40C94A46A4D
:10C110003B014C01AA969FAF8EAFAA978CE794E0A3
:10C12000A8969FAF8EAFA897AE96BFAFAEAFAE97B3
:10C1300084E694E0AC969FAF8EAFAC97FD01828110
:10C140009B01225031092230310508F017C6803496
:10C1500009F4F7C208F04AC0843008F085C2809123
:10C16000FF098F5F8093FF09A3016FEFC4010E9455
:10C170006520D40112960C911297069501701396C2
:10C180001C9113978AEC810F803108F043C06AEB51
:10C1900076E08D919C910E94E5D77C010097D1F1CA
:10C1A000FC0180858F708530A9F58091E60F18130A
:10C1B00024C08091E70F803401F58091E80F9091C1
:10C1C000E90F5C01990FCC08DD0860E0C7010E940F
:10C1D00097D8FC0181859285A385B485A816B906F8
:10C1E000CA06DB060CF065C0512C3EC0823409F44F
:10C1F000A8C208F439C28058AFCF1093E60F80E48C
:10C200008093E70F812F0E945AE79093E90F809364
:10C21000E80FD7CF212F30E0F901EB50F44D849196
:10C22000F901EB5AF34D1491F901E556F34DF490F1
:10C23000FF2009F43BC081110E94B2E5EF2DF0E030
:10C24000EE0FFF1FE954F04DA591B491EC911E2320
:10C2500031E020E009F430E0832F922F55245394ED
:10C260000817190609F0C0CFF3E06F16710409F43E
:10C2700088C0D4011496ED91FC91E181EF70E150FA
:10C28000EC3008F07EC0F0E08827E65BFE498F4F77
:10C290000D94CC3E6B61E762A161D761E762F0610A
:10C2A000E762246251626A62AC62CE6290E080E032
:10C2B000D5CF61E0C7010E9497D855245394FC0163
:10C2C00081859285A385B4858A159B05AC05BD053E
:10C2D0000CF0CACF89CF0E947EEA9B01AC014427B3
:10C2E0005527D4011496ED91FC916281738190E001
:10C2F00080E0AA24AA94BA2CC12CD12C18EEE12EED
:10C3000013E0F12E00E010E00F9456278823C9F1C6
:10C31000F401008111816AEE75E0C8010E94E5D741
:10C32000892B41F46FEE75E0C8010E94E5D7892B97
:10C3300009F40EC142E050E063E0C4010E946520B0
:10C3400020C00E947EEA9B01AC0144275527D401FE
:10C350001496ED91FC916281738190E080E0AA24B3
:10C36000AA94BA2CC12CD12C1CE2E12EFF24F39408
:10C3700000E010E00F94562742E050E064E08111A5
:10C3800084C0D4011496ED91FC91808183FB9927A0
:10C3900090F9951509F4D2C1982F907E09F439C10E
:10C3A000982F907E90528F71892B808358C10E9464
:10C3B0007EEA9B01AC0144275527D4011496ED91E8
:10C3C000FC916281738190E080E0AA24AA94BA2C47
:10C3D000C12CD12C16E9E12EF12C00E010E0CACFDF
:10C3E0000E947EEA9B01AC0144275527D401149694
:10C3F000ED91FC916281738190E080E0AA24AA947F
:10C40000BA2CC12CD12C18EEE12E13E0F12E00E055
:10C4100010E00F945627882309F4B3CFF40100816C
:10C42000118165EF75E0C8010E94E5D7892B41F4C1
:10C430006BEF75E0C8010E94E5D7892B09F488C02D
:10C4400042E050E068E079CF0E947EEA9B01AC01B7
:10C4500044275527D4011496ED91FC916281738194
:10C4600090E080E0AA24AA94BA2CC12CD12C1CE222
:10C47000E12EFF24F39400E010E00F94562742E0F1
:10C4800050E069E0882309F47CCFC4010E94652054
:10C490000E947EEAD4011496ED91FC91738362832D
:10C4A00070CF0E947EEA9B01AC0144275527D4013E
:10C4B0001496ED91FC916281738190E080E0AA2452
:10C4C000AA94BA2CC12CD12C16E9E12EF12C00E053
:10C4D00010E0D3CF0E947EEA9B01AC014427552790
:10C4E000D4011496ED91FC916281738190E080E01B
:10C4F000AA24AA94BA2CC12CD12C18EEE12E13E058
:10C50000F12E00E010E00F945627882309F439CF6C
:10C51000F4010081118162E076E0C8010E94E5D754
:10C52000892B39F468E076E0C8010E94E5D7892BB1
:10C5300021F042E050E06BE000CF64EE75E0C8010E
:10C540000E94E5D742E050E066E0892B09F4F5CE81
:10C5500042E050E06DE0F1CE0E947EEA9B01AC012A
:10C5600044275527D4011496ED91FC916281738183
:10C5700090E080E0AA24AA94BA2CC12CD12C1CE211
:10C58000E12EFF24F39400E010E00F945627882357
:10C5900009F4F7CE42E050E06CE077CF0E947EEAEB
:10C5A0009B01AC0144275527D4011496ED91FC91D1
:10C5B0006281738190E080E0AA24AA94BA2CC12CF5
:10C5C000D12C16E9E12EF12C00E010E0DECF0E9424
:10C5D0007EEA9B01AC0144275527D4011496ED91C6
:10C5E000FC916281738190E080E0AA24AA94BA2C25
:10C5F000C12CD12C18E5E12E12E0F12E00E010E064
:10C600000F945627882309F4BCCE42E050E060E046
:10C6100094CE0E947EEAD4011496ED91FC91159778
:10C6200073836283E181EF70552009F445C0E230E5
:10C63000F1F050F4EE23E9F1D4011496ED91FC9160
:10C64000808150FA83F9B1CEE53089F0A3016AE028
:10C65000E73091F7C4010E9465208111EDCF8091F0
:10C66000FF0981508093FF0990E080E06FC7F401DB
:10C67000008111816EED75E0C8010E94E5D7892B1C
:10C68000A9F465EF75E0C8010E94E5D7892B71F424
:10C690006BEF75E0C8010E94E5D7892B39F466EC91
:10C6A00075E0C8010E94E5D7892B19F0A30166E067
:10C6B000D1CFA30161E0CECFE150ED3008F0BCCF87
:10C6C000F0E08827E959FC498F4F0D94CC3E746304
:10C6D0001C63776377631C637A631C639B639B6350
:10C6E0009B639B639B637763A30162E0B3CFA3016A
:10C6F00065E0B0CF0D911C916EED75E0C8010E9410
:10C70000E5D7892BA9F465EF75E0C8010E94E5D74C
:10C71000892B71F46BEF75E0C8010E94E5D7892B76
:10C7200039F466EC75E0C8010E94E5D7892B19F051
:10C73000A30167E08FCFA30160E08CCF8F7180648D
:10C7400034CEB3E06B16710409F48ECF6AEB76E059
:10C75000F401808191810E94E5D78C01D401139668
:10C760008C919091E60F8913E5C09091E70F90347A
:10C7700009F0E0C08091E80F9091E90F3C010115AC
:10C78000110509F404C1F80120852F70253009F046
:10C79000FEC0C8010E9429D9AF968FAFAF978430F1
:10C7A00008F4D4C063E0C8010E9497D8DC01199650
:10C7B0008D919C912AE0F22EF89E1001F99E300C8A
:10C7C000112462E0C8010E9497D8FC0181859285FE
:10C7D000F89E5001F99EB00C112465010B2C000C41
:10C7E000EE08FF08EF96CCAEDDAEEEAEFFAEEF97F3
:10C7F00061E0C8010E9497D82C0160E0C8010E9446
:10C8000097D8DC011996CD90DD90ED90FC901C97A7
:10C81000E396CCAEDDAEEEAEFFAEE3979301072C10
:10C82000000C440B550B2C193D094E095F09B10151
:10C83000032C000C880B990BEF96CCACDDACEEAC66
:10C84000FFACEF976C197D098E099F090F94453E47
:10C85000D20119962D913D914D915C911C97E396D3
:10C86000CCACDDACEEACFFACE3972C193D094E0926
:10C870005F09E3962CAF3DAF4EAF5FAFE3970F94E8
:10C88000773EEF96CCACDDACEEACFFACEF97C20ED2
:10C89000D31EE41EF51EAF962FADAF97253009F4D9
:10C8A00065C081E090E0A101032C000C660B770BC2
:10C8B0004C155D056E057F050CF461C0B701A6013E
:10C8C00065010B2C000CEE08FF084C155D056E058C
:10C8D0007F050CF459C06A017B01AF96BFADAF97DD
:10C8E000B23009F065C06301770CEE08FF0860E024
:10C8F000C8010E9497D8FC0181859285A385B485E3
:10C90000C816D906EA06FB060CF43AC661E0C8016F
:10C910000E9497D8FC0181859285A385B4858C15EA
:10C920009D05AE05BF050CF09FCE81E090E0A0E034
:10C93000B0E029C68093E60F90E49093E70F0E9441
:10C940005AE79093E90F8093E80F18CF8AE0869D0D
:10C950006001879DD00C11240D2C000CEE08FF08FF
:10C96000B12CA12C212C88E2382E9BCF64E0C80189
:10C970000E9497D8DC0119968D919C9194CF6624E2
:10C980006A94B3E07B2E9CCF712C612CA6CF2AE059
:10C99000289F6001299FD00C11240D2C000CEE085B
:10C9A000FF08B12CA12C212CA8E23A2E81E090E0C6
:10C9B000D4011496ED91FC9162817381A301461B11
:10C9C000570B57FF03C0519541955109841795079F
:10C9D0000CF4C0C08081982F9295969597709630F0
:10C9E00008F0BBC09F5F9295990F907E8F71892B45
:10C9F000B3C0F20161857285DB018C91811154C64F
:10CA00000115110509F457C0D80118968C91189793
:10CA10008F70843009F04FC019966D917C91CE01D2
:10CA200001960E94E838CE0101960E946F2D88235E
:10CA3000F1F12114310409F460C04114510431F0C2
:10CA4000F20180858F70843009F44CC025961CAEAD
:10CA50001DAE1EAE1FAE259729961CAE1DAE1EAE96
:10CA60001FAE299723961FAD23971F7023961FAFE4
:10CA7000239781E022968FAF2297A12CCC24C394D8
:10CA8000F12CE12C01E024962FAD249725963FADA3
:10CA9000259740E027965FAD279728966FAD28979A
:10CAA00029967FAD2997CE0101960E94CC47CE01F1
:10CAB00001960E947439D4011496ED91FC91338251
:10CAC0002282D2CD6114710429F0F30180858F7028
:10CAD000843019F060EF77E0E7C561857285FB016E
:10CAE00080818CCF61857285FB0180818823F9F27A
:10CAF000CE0101960E9434DFDACF6114710431F067
:10CB0000D30118968C918F708430F1F025961CAE6D
:10CB10001DAE1EAE1FAE259729961CAE1DAE1EAED5
:10CB20001FAE299723961FAD23971F7023961FAF23
:10CB3000239782E022968FAF2297A12CCC24C39416
:10CB4000F12CE12C02E09FCFF30161857285DB01BE
:10CB50008C91CCCF80818F7180838081803A98F0D6
:10CB6000C501BB0CAA0BBB0B8C159D05AE05BF0503
:10CB700051F0C101330CAA0BBB0B8C159D05AE0502
:10CB8000BF0509F071CD6615770509F46DCDA29644
:10CB90001CAE1DAE1EAE1FAEA297A0968FADA09785
:10CBA0008F708066A0968FAFA097A2968CAD9DAD3A
:10CBB000AEADBFADA29768968CAF9DAFAEAFBFAF25
:10CBC0006897AAE0B0E0A70196010F94963E6C9694
:10CBD0006CAF7DAF8EAF9FAF6C9760E179E087EA75
:10CBE0009FE00F94CC0B4AE050E0F401638187EAA8
:10CBF0009FE00F94330A6EE079E087EA9FE00F949C
:10CC0000CC0BCE018C5A9F4F0E941A286EEB76E017
:10CC1000D4018D919C910E94E5D7B12CA12CD12CEF
:10CC2000C12C6596EFAC65976696FFAC66976796E4
:10CC30000FAD679768961FAD689769962FAD699796
:10CC40006A963FAD6A976B964FAD6B976C965FADEA
:10CC50006C976FEF0F94C02BF401008111816FE08E
:10CC600076E0C8010E94E5D77C0164E176E0C80166
:10CC70000E94E5D78C010097F1F1DC0118968C91A8
:10CC800018978F708430B9F519966D917C9140E4B6
:10CC900050E0CE0101960F9467436FE270E0CE0141
:10CCA00001960F942E43892B51F4F801218532858A
:10CCB00043E050E060E4CE0101960F94792800E053
:10CCC00020E032E040E150E0BE016F5B7F4FCE01DB
:10CCD0008C5A9F4F0E94F9250E9403D8882359F04F
:10CCE0008091C910811107C0BE016F5B7F4FCE01DB
:10CCF00001960E941BEBE114F104C9F1D7011896CB
:10CD00008C9118978F70843091F519966D917C9164
:10CD1000CE0101960E94E838CE0101960E946F2D47
:10CD2000882309F1A12CCC24C394F12CE12C659625
:10CD30000FAD659766961FAD669767962FAD67979F
:10CD400068963FAD689769964FAD69976A965FADF3
:10CD50006A976B966FAD6B976C967FAD6C97CE01B3
:10CD600001960E94CC47CE0101960E947439D401ED
:10CD70001496ED91FC917382628276CC863009F430
:10CD800056C070F4843009F45AC0853009F06CCC78
:10CD900061E070E0CE018A599F4F0E9402C064CCCE
:10CDA000883009F4E1C2803109F05ECC0E947EEA4D
:10CDB0002B013C01C4010E94B618A12CB12C6501C5
:10CDC00010E3E12E15E7F12E00E010E0A30192013F
:10CDD0000F945627882309F447CC64E176E0D40108
:10CDE0008D919C910E94E5D78C01009709F497C220
:10CDF000FC0180858F70843009F091C20E947EEA28
:10CE00002AE0AE014F5F5F4F0F94BA370E9403D8FC
:10CE1000882309F484C28091C910811180C2BE01A7
:10CE20006F5F7F4FD80119968D919C9176C261E01A
:10CE300070E0CE0186599F4F0E94B8C115CC0E9468
:10CE40007EEA2B013C01C4010E94B618A12CB12C32
:10CE5000650118E9E12E1AE3F12E00E010E0A301CC
:10CE600092010F945627882309F4FECBF4018381A5
:10CE700027968FAF279796E128969FAF2897282F60
:10CE800030E0F901EB5AF34DE4912996EFAF299781
:10CE9000F901E556F34DE4912A96EFAF2A9740E861
:10CEA0005EE360E070E062964CAF5DAF6EAF7FAF67
:10CEB000629762E00E9447E60E947EEA605D7740EA
:10CEC000810991092E966CAF7DAF8EAF9FAF2E97E3
:10CED00087E364968FAF6497CE018F5B9F4F0E946C
:10CEE000A7ED882349F028968FAD28978C3009F458
:10CEF0006FC048F48B3011F1412C512C60EC662E40
:10CF00006FE7762E47C085518230B0F724961FAD6B
:10CF10002497612F70E0762F662766277F77259606
:10CF20008FAD2597682B90E080E00F94103D2DEC9D
:10CF30003CEC4CEC5DE30F94713D68C024966FAD02
:10CF4000249770E090E080E00F94103D6B017C012D
:10CF500025961FAD259717FF0AC0AC019B0160E025
:10CF600070E080E89FEB0F94FE3E6B017C011F7028
:10CF7000612F70E090E080E00F94123D2DEC3CECCE
:10CF80004CEC5DE30F94713DA70196010F94FF3EB9
:10CF90002B013C01CE018F5B9F4F0E94A7ED8823A0
:10CFA00009F4D7C128968FAD28978B3030F08D309B
:10CFB000B0F18551823008F4BAC1312C212C30EC0B
:10CFC000AF963FAFAF974FE7E0964FAFE0974DC0BA
:10CFD00024961FAD2497612F70E090E080E00F94BD
:10CFE000103D6B017C0125966FAD25976F7070E049
:10CFF00090E080E00F94123D2DEC3CEC4CEC5DE3B6
:10D000000F94713DA70196010F94FF3E2B013C0147
:10D0100017FFC0CF77FA709477F87094BBCF239640
:10D020006FAD239770E090E080E00F94123D2DECFF
:10D030003CEC4CEC5DE30F94713D6B017C0122965E
:10D040006FAD229770E090E080E00F94123D9B015D
:10D05000AC01C701B6010F94FF3E362E272EAF96C6
:10D060008FAFAF97E0969FAFE0976AE379E087EAEA
:10D070009FE00F94CC0B4AE050E0D40113966C91E2
:10D0800087EA9FE00F94330A6AE279E087EA9FE03B
:10D090000F94CC0BB301A20187EA9FE00E940FDD41
:10D0A00063E279E087EA9FE00F94CC0B432D522D89
:10D0B000AF966FADAF97E0967FADE09787EA9FE0C0
:10D0C0000E940FDD61E279E087EA9FE00F94CC0BCC
:10D0D00087EA9FE00F94160AF401008111816EEA3D
:10D0E00078E0C8010E94E5D7E5969FAF8EAFE5973F
:10D0F00062EC76E0C8010E94E5D7E7969FAF8EAF5D
:10D10000E797A3019201C301B2010F94734081110B
:10D110001FC019821A821B821C828A818F708067CD
:10D12000F82E8A83242D4D825E826F827886B12C00
:10D13000A12CD12CC12CE9800B811C813E814F8117
:10D1400058856FEFE5968EAD9FADE5970F94C02B98
:10D15000232D322DAF964FADAF97E0965FADE097A0
:10D16000632D722DAF968FADAF97E0969FADE09790
:10D170000F947340811127C019821A821B821C826E
:10D180008A818F708067F82E8A83232D832D922DBC
:10D19000AF96AFADAF97E096BFADE0978D839E831E
:10D1A000AF83B887B12CA12CD12CC12CE9800B8185
:10D1B0001C813E814F8158856FEFE7968EAD9FAD04
:10D1C000E7970F94C02B64E176E0D4018D919C9198
:10D1D0000E94E5D77C01009709F4A1C0FC0180857D
:10D1E0008F70843009F09BC020E030E0A901C301BA
:10D1F000B2010F940B3D882309F491C020E030E088
:10D20000A901632D722DAF968FADAF97E0969FADBC
:10D21000E0970F940B3D882309F481C0A30192018C
:10D22000C301B2010F940B3D811179C0232D322D22
:10D23000AF964FADAF97E0965FADE097632D722D3F
:10D24000AF968FADAF97E0969FADE0970F940B3DF3
:10D25000811165C01A821982FE0133968EE3DF01C7
:10D260001D928A95E9F7F7016185728540E450E0E7
:10D270008E010F5F1F4FC8010F9467436FE270E08C
:10D28000C8010F942E43892B51F4D70119962D9183
:10D290003C9143E050E060E4C8010F94792861EECE
:10D2A00078E0C8010F942343B301A201CE018C5A48
:10D2B0009F4F0F94A1290E9403D8882351F0809199
:10D2C000C910811106C0BE016C5A7F4FC8010E946F
:10D2D00036EBF80101900020E9F73197E01BF10BE4
:10D2E000EC0FFD1F88E48083432D522DAF966FAD68
:10D2F000AF97E0967FADE097CE018C5A9F4F0F9489
:10D30000A1290E9403D8882351F08091C91081116E
:10D3100006C0BE016C5A7F4FC8010E9436EB0E94C6
:10D320007EEAAB01BC01C4010E948F189DC92396FF
:10D330006EAD7FAD239776276727762790E080E054
:10D340000F94103D2DEC3CEC4CEC5DE30F94713DE3
:10D3500084CE312C212CF0ECAF96FFAFAF972FE7A6
:10D36000E0962FAFE09781CE0E947EEA2B013C0130
:10D37000C4010E94B618A12CB12C650118E9E12E58
:10D380001AE3F12E00E010E0A30192010F9456275A
:10D39000882309F469C9D4011496ED91FC9115977D
:10D3A000818113961C91811157C0163008F03FC03F
:10D3B0008CE0E0E5F2E0DE01119601900D928A9595
:10D3C000E1F7E12FF0E0EE0FFF1FCC24C394D12C46
:10D3D000CC0EDD1EEC0DFD1D60E080810E9447E655
:10D3E00066E079E183E01330C9F070F46EE079E132
:10D3F00081E0113099F06AE079E182E0123071F059
:10D4000062E179E180E00AC062E079E184E0143011
:10D4100029F06EEF78E185E0153091F70E94DFDEAC
:10D42000D4011496ED91FC9181E081831DC962E9DC
:10D4300079E087EA9FE00F94CC0B4AE050E0F401DA
:10D44000638187EA9FE00F94330A65E679E087EA13
:10D450009FE00F94CC0B08C924E0129FF001112427
:10D46000E050F64FC080D180E280F38061E679E041
:10D4700087EA9FE00F94CC0B4AE050E0D40113966A
:10D480006C9187EA9FE00F94330A6DE479E087EAB4
:10D490009FE00F94CC0B2AE030E0B701A60187EAA9
:10D4A0009FE00F94D50A64E176E0F40180819181D8
:10D4B0000E94E5D78C01009709F443C0DC0118965F
:10D4C0008C9118978F708430E1F519966D917C914D
:10D4D00040E450E0CE0101960F9467436FE270E0A4
:10D4E000CE0101960F942E43892B51F4F80121852A
:10D4F000328543E050E060E4CE0101960F94792834
:10D50000FF92EF92DF92CF9280E296E09F938F930B
:10D510008E010F5B1F4F1F930F930F94BE430E940A
:10D5200003D80FB6F894DEBF0FBECDBF882309F431
:10D53000F6CE8091C9108111F2CEB801CE010196CC
:10D54000ECCE6EE379E083CF8FEF9FEFC258DF4FD1
:10D550000FB6F894DEBF0FBECDBFDF91CF911F9104
:10D560000F91FF90EF90DF90CF90BF90AF909F9082
:10D570008F907F906F905F904F903F902F90089585
:10D5800080E090E0DC01F40124813581F9014281E1
:10D590005381052E000C660B770B481759076A0755
:10D5A0007B0709F461C81C01D4016D907C906FE089
:10D5B00076E0C3010E94E5D78C0164E176E0C30107
:10D5C0000E94E5D77C010115110519F4892B09F496
:10D5D00072CA69ED75E0C3010E94E5D72C0164EDC4
:10D5E00075E0C3010E94E5D73C0166E179E087EA76
:10D5F0009FE00F94CC0B4AE050E0F401638187EA8E
:10D600009FE00F94330A64E179E087EA9FE00F948A
:10D61000CC0B4AE050E0B10187EA9FE00F941D0B6C
:10D6200087EA9FE00F94160AE114F10409F4E8C9AF
:10D63000D70118968C9118978F70843009F0E0C943
:10D6400019966D917C9140E450E0CE0101960F94C3
:10D6500067430E9403D8882309F4D2C98091C91076
:10D660008111CEC96FE270E0CE0101960F942E4376
:10D67000892B51F4F7012185328543E050E060E4C5
:10D68000CE0101960F9479282114310409F41ACAA5
:10D690004114510439F0D20118968C918F70843066
:10D6A00009F4A7C965EE77E0CE0101960E941BEB55
:10D6B000A7C96F927F928F929F92AF92BF92CF92A3
:10D6C000DF92EF92FF920F931F93CF93DF93CDB72B
:10D6D000DEB7A5970FB6F894DEBF0FBECDBF809121
:10D6E000B10A9091B20A892B09F419C68091DF1012
:10D6F000811115C68091DF108F5F8093DF106DEE72
:10D700007BE186EF9EE00F94CC0B86EF9EE00F94BA
:10D71000160A0091B10A1091B20A66EC76E0C801CF
:10D720000E94E5D79093E6108093E5106CEC76E0CC
:10D73000C8010E94E5D79093C8108093C71064E891
:10D7400076E0C8010E94E5D79093E2108093E11043
:10D7500063ED76E0C8010E94E5D79093AC0A809310
:10D76000AB0A0E94F11D68ED76E08091B10A9091BC
:10D77000B20A0E94E5D79093AA0A8093A90A00975B
:10D7800009F4B2C00E9429D9082F10E00115110533
:10D7900009F4AAC0000F111F000F111F8091A70AE2
:10D7A0009091A80A892B09F08EC0780101381105E3
:10D7B0001CF040E8E42EF12CC7010F94DD34909367
:10D7C000A80A8093A70AE092A60A1092DA10109293
:10D7D000D9101092A50A1092A40A1092D810109293
:10D7E000DC101092DB10C70101960F94DD3490938A
:10D7F000DE108093DD109093D7108093D6108E0D9D
:10D800009F1D9093D1108093D0100E947EEA609368
:10D81000D2107093D3108093D4109093D51090E0D1
:10D8200080E0E091DD10F091DE10E80FF91F10822A
:10D830000196E816F906ACF782E090E09093DA10D2
:10D840008093D9108091A40A9091A50A009741F085
:10D8500061E00E9447E660E08091A40A0E9419E618
:10D8600080E98093C9001092C8001092CD0083E037
:10D870008093CC008EE08093CA00F0924302E09245
:10D8800042022091DD103091DE1080914202909191
:10D890004302820F931F9093D1108093D010232BBB
:10D8A00009F460C06DE77BE187EA9FE00F94CC0B41
:10D8B000B70187EA9FE00E94FBDC86E39CE190933E
:10D8C000CF108093CE1063ED7BE186EF9EE00F9446
:10D8D000CC0B4AE050E0B80186EF9EE00F941D0BA0
:10D8E00086EF9EE00F94160A6EED76E08091B10A05
:10D8F0009091B20A0E94E5D78C01009709F472C09A
:10D900000E9429D9882309F46DC06FEF680FC80100
:10D910000E9497D8DC011996ED90FC909091CC1064
:10D92000992359F0809170008E7F8093700010923F
:10D93000CC1010923E0210923D0282E180933C0294
:10D9400091110F94FE21C7010F94262201E010E0EF
:10D95000E016F10674F060E0C8010F945A220F5FE0
:10D960001F4FF6CF66E67BE187EA9FE00F94F00B4E
:10D97000A4CF68E57BE187EA9FE00F94CC0B0F947E
:10D98000FA29AB01BC012AE030E087EA9FE00F945E
:10D99000310A87EA9FE00F94160A67EB7BE186EF76
:10D9A0009EE00F94CC0B4AE050E0B70186EF9EE07A
:10D9B0000F941D0B86EF9EE00F94160A61EB7BE13E
:10D9C00087EA9FE00F94CC0B0F94FA29AB01BC01BE
:10D9D0002AE030E087EA9FE00F94310A87EA9FE06F
:10D9E0000F94160A0091B10A1091B20A62EE76E025
:10D9F000C8010E94E5D79093B50A8093B40A69EEF6
:10DA000076E0C8010E94E5D79093E8108093E71074
:10DA1000892BA1F08091E910811110C08091CA106A
:10DA20009091CB10892B09F47CC081E08093E910A0
:10DA300061EA7BE186EF9EE00F94CC0B1092B00A76
:10DA40001092AF0AE091E510F091E610309709F4DA
:10DA500002C3C680D7800091E5101091E610011531
:10DA6000110509F4F1C2C114D10409F4EDC2F601A3
:10DA700080858F70853099F7C6010E9429D9823040
:10DA800070F3B601CE0101960E94D23ACE01019602
:10DA90000E946F2D8823E1F18A859B85009709F408
:10DAA00044C2DC01ED91FC910284F385E02D1995CF
:10DAB000892B49F08A859B85DC01ED91FC910084DE
:10DAC000F185E02D19958A859B85DC01ED91FC910E
:10DAD0000680F781E02D1995892BD1F0CE010196B2
:10DAE0000E94E535882341F040E051E060E070E0BD
:10DAF000CE0101960E949F308D819E81892B41F03D
:10DB000040E052E060E070E0CE0101960E949F305C
:10DB1000D6011296CD90DC90CE0101960E94743908
:10DB20009ACF62E37BE187EA9FE00F94CC0B87EA10
:10DB30009FE00F94160A8FE090E00F94DD348C0183
:10DB400088E1F801818312821082168615860E9470
:10DB50002EE21093CB100093CA10012B69F463E2FC
:10DB60007BE180E09FE00F94CC0B80E09FE00F947E
:10DB7000160A1092E91062CF0E942EE28091CA101C
:10DB80009091CB100F9488228CEF9CE00F942D2461
:10DB9000811193C064E07BE186EF9EE00F94F00B6F
:10DBA0008091CA109091CB100F94CC25E091CA10AF
:10DBB000F091CB1081E080838091CA109091CB10BE
:10DBC0000F94DA2560EF7AE1811102C06BED7AE102
:10DBD00087EA9FE00F94F00B8091E7109091E81096
:10DBE000892B39F28091B80A9091B90A892B09F0F2
:10DBF000EEC083E190E00F94DD348C018091CA1077
:10DC00009091CB1025E033E0D80152963C932E93AF
:10DC1000519716969C938E93159714961C92149771
:10DC20001C9289E011968C93119781E012968C9347
:10DC3000129713968C931093B90A0093B80A0E9416
:10DC40007EEA6B017C01B0E1CB0EB7E2DB1EE11C8A
:10DC5000F11CD8011596ED91FC9116978FEF8387F3
:10DC600014861382148215821682178210861186FA
:10DC7000128614961C92BB24B394BE01625E7F4F41
:10DC8000F801858196810F94B42618160CF09AC07D
:10DC90000E947EEA6C157D058E059F0508F092C0F6
:10DCA000DE015E9698E080E0915039F1ED91E82731
:10DCB000F0E0E657F14D8491F7CF0F94E127809182
:10DCC000CA109091CB100F9488228CEF9CE00F9497
:10DCD0002D2481110BC06EEB7AE186EF9EE00F944C
:10DCE000CC0B86EF9EE00F94160A76CF62EA7AE1BB
:10DCF00080E09FE00F94F00B3CCF9DA19813BDCF27
:10DD0000D8018C91811138C015968D919C910F94FA
:10DD1000DA25BE01625E7F4FF801858196810F94FE
:10DD2000AD2540E064EBD80115968D919C910F9440
:10DD30008725F80185809680C4010F940B25C401C6
:10DD40000F94882267E88CEF9CE00F94DD0460E874
:10DD50008CEF9CE00F94DD040E942AE2C4010F9432
:10DD60000B25A82ED80115968D919C910F94DA253C
:10DD7000A5FC02C0F801B082AE014F5F5F4FBE014B
:10DD8000625E7F4FC8010F941B26D8011196AC909C
:10DD90008E8D803109F4D8C2BE01625E7F4FC8010A
:10DDA0000F948A268A1508F0B4C0F8018181D80141
:10DDB00011968C93119714968C9114978F5F1496EB
:10DDC0008C935BCFE091B80AF091B90A1282E0918E
:10DDD000E710F091E810E680F7803FE7D32E8091BE
:10DDE000E7109091E810892B09F41FCEE114F1049B
:10DDF00009F41BCEBE01625E7F4FF70180819181E5
:10DE00000F94862B882309F410CE6BE87AE187EA19
:10DE10009FE00F94CC0BD7016D917C9187EA9FE036
:10DE20000F94660B87EA9FE00F94160A0091B80AD8
:10DE30001091B90AAE014F5F5F4FBE01625E7F4F26
:10DE4000C8010F947026882309F45EC08E8D80313E
:10DE500009F45AC0DD82F801858196810F94DA2594
:10DE6000BE01625E7F4FD80115968D919C910F94F3
:10DE7000AD2540E06EE4F801858196810F948725F9
:10DE800040E06B81D80115968D919C910F94872568
:10DE900040E06C81F801858196810F9487258E8DF5
:10DEA000803141F040E06D81D80115968D919C91B3
:10DEB0000F948725F801858196810F94DA25BE019C
:10DEC000625E7F4FD80115968D919C910F94AD2580
:10DED000F801408168E4858196810F94872564E18B
:10DEE00070E080E090E00E948CE8D8018C9188235B
:10DEF00031F06AE070E080E090E00E948CE8F80188
:10DF0000858196810F94DA25D7011296ED90FC90C9
:10DF100066CF8E8D803111F48CE049CFBE01625EF8
:10DF20007F4FC8010F948A2642CF70E060E0CE0197
:10DF300001960E94612E8C01912C812C97FF06C0C6
:10DF400011950195110988248394912CCE01019695
:10DF50000E94E535E82EF12C8985853091F08630D8
:10DF600009F0D6CDB02E61E0802F0E9447E661E037
:10DF7000892809F443C0EA94EF2809F043C060E01F
:10DF800041C0EF2829F462E0CE0101960E947C1B7B
:10DF900040E051E060E070E0CE0101960E949F30C9
:10DFA0008D819E81892B41F040E052E060E070E07D
:10DFB000CE0101960E949F3061E0802F0E9447E6CB
:10DFC00060E0802F0E9419E669E97BE187EA9FE023
:10DFD0000F94CC0B4AE050E0B80187EA9FE00F9421
:10DFE0001D0B64E97BE187EA9FE00F94CC0B62E9AB
:10DFF0007BE187EA9FE00F94CC0B8ACDEA94EF286F
:10E0000009F0BDCFE62EF12C8B2D0E9419E66DE8AC
:10E010007BE187EA9FE00F94CC0B4AE050E0B80127
:10E0200087EA9FE00F941D0B6BE87BE187EA9FE096
:10E030000F94CC0B4AE050E0B70187EA9FE00F94C1
:10E040001D0B69E87BE1D5CFF8018681978190931C
:10E05000B00A8093AF0A87EA9FE00F94160A67E739
:10E060007AE186EF9EE00F94CC0B86EF9EE00F9452
:10E07000160AE091E110F091E210309709F4ADC07A
:10E080008091DF108F5F8093DF10068117815E0122
:10E09000FEE1AF0EB11C84E6682E84E0782E9CE78A
:10E0A000892E94E0992E0115110509F491C0D8012B
:10E0B00018968C918F70863009F068C01F8F0E8F74
:10E0C00070E060E0C5010E9417408AA19BA1892BE6
:10E0D00009F45CC08091B10A9091B20A892B09F4CD
:10E0E00055C0EE8CFF8CF70180858F70863099F5D6
:10E0F0006EEB76E0C7010E94E5D70097F1F0DC01F6
:10E1000018962C9118972F702530B9F41696CD904B
:10E11000DC90C114D104F9F0DA82C982B701CE01D2
:10E1200001960E941740ED81FE81108211821282B9
:10E130001382F601C280D380ECCFFA82E98270E0CC
:10E1400060E0CE0101960E94174062E070E0CE01CF
:10E1500001960E946460EAA1FBA1108211821282E2
:10E16000138288A1843068F462E0823008F060E0B5
:10E1700089A10E9447E6EAA1FBA18181807F81837A
:10E1800005C08630E1F038F4853081F0D801129670
:10E190000D911C9188CF803439F060E08234B1F762
:10E1A00089A10E9447E6F2CF62E0FACFBC82AB823F
:10E1B0009A828982CE0101960E94FAC3E7CFBC827F
:10E1C000AB827A826982CE0101960E9449C3DECF7A
:10E1D0008091DF1081508093DF106AE67AE186EF4C
:10E1E0009EE00F94CC0B62E67AE186EF9EE00F94FE
:10E1F000CC0B81E02091E5103091E610232B09F43F
:10E2000080E00E94A91969E57AE186EF9EE00F940B
:10E21000CC0B81E02091E1103091E210232B09F426
:10E2200080E00E94A9196AE47AE186EF9EE00F94EB
:10E23000CC0B6FE37AE186EF9EE00F94CC0B81E08C
:10E240002091B40A3091B50A232B09F480E00E9492
:10E25000A91968E37AE186EF9EE00F94CC0B81E088
:10E260002091AB0A3091AC0A232B09F480E00E9484
:10E27000A9196FE27AE186EF9EE00F94CC0B81E062
:10E280002091E7103091E810232B09F480E00E94E0
:10E29000A91966E27AE186EF9EE00F94CC0B80919B
:10E2A000BA0A0E94A91986EF9EE00F94160A61E24D
:10E2B0007AE186EF9EE00F94CC0B0F94FA29AB0124
:10E2C000BC012AE030E086EF9EE00F94310A86EF31
:10E2D0009EE00F94160A81E08093AE0A85EC9EE0E2
:10E2E0000F945719882351F085EC9EE00F940F206E
:10E2F00084E090E09093E4108093E3108091E31029
:10E300009091E410079731F484E090E09093E4104A
:10E310008093E3108091DF1081508093DF10A596E9
:10E320000FB6F894DEBF0FBECDBFDF91CF911F9126
:10E330000F91FF90EF90DF90CF90BF90AF909F90A4
:10E340008F907F906F900895BCE0BA1508F42DCDA2
:10E35000E3CDAF92BF92CF92DF92EF92FF920F93F5
:10E360001F93CF93DF93CDB7DEB7C554D1090FB656
:10E37000F894DEBF0FBECDBF8091FB099091FC09E0
:10E38000A091FD09B091FE09892B8A2B8B2B09F4F2
:10E39000CCC00E947EEA9B01AC016091FB097091A8
:10E3A000FC098091FD099091FE09A12CB12C650119
:10E3B0001CE2E12EFF24F39400E010E00F945627B6
:10E3C000882309F4B2C01092FB091092FC09109244
:10E3D000FD091092FE098091A60A90E09595879517
:10E3E0009595879510E000E0E1E0F0E08017910757
:10E3F00009F49BC09F01002E02C0220F331F0A9414
:10E40000E2F7C090F709D090F809E090F909F09090
:10E41000FA09A901032E000C660B770B4C215D2134
:10E420006E217F21452B462B472B09F4DCC0409100
:10E43000F7095091F8096091F9097091FA0920954E
:10E440003095C901330FAA0BBB0B84239523A62358
:10E45000B7238093F7099093F809A093F909B09333
:10E46000FA098091A90A9091AA0A009709F45DC05F
:10E47000FC0120852F70253009F057C0602F0E94C5
:10E4800097D8FC0190859F70943009F04EC061854B
:10E4900072856115710509F448C0E091A70AF091F1
:10E4A000A80A000F111F000F111FE00FF11F1381A9
:10E4B0000281F180E080CE0101960E94E838E110EF
:10E4C00046C0F11044C0011142C0111140C01EA24B
:10E4D0001FA218A619A61AA61BA61CA61DA68FA1C8
:10E4E0008F708FA362E0CE0186960E9443202E8F0C
:10E4F0003F8F48A359A36AA37BA38CA39DA361E08C
:10E50000CE014E960E941C20A12CCC24C394F12C49
:10E51000E12C89019A01AB01BC01CE0101960E9458
:10E52000CC47CE0101960E947439CB5BDF4F0FB60A
:10E53000F894DEBF0FBECDBFDF91CF911F910F9139
:10E54000FF90EF90DF90CF90BF90AF9008951EA204
:10E550001FA218A619A68FA18F7080658FA3ECA6A5
:10E56000FBA60AA71DA78AA59BA5ACA5BDA54EA184
:10E570005FA168A579A54E8F5F8F68A379A38AA351
:10E580009BA3ACA3BDA362E0CE014E960E941C20CB
:10E59000A12CCC24C394F12CE12C89019A01AB016C
:10E5A000BC01CE0101960E94CC471EA21FA218A654
:10E5B00019A61AA61BA61CA61DA68FA18F708FA335
:10E5C00061E0CE0186960E9443202E8F3F8F48A3A4
:10E5D00059A36AA37BA38CA39DA361E0CE014E96B1
:10E5E0000E941C2096CF0F5F1F4F00CF4F925F926B
:10E5F0006F927F92AF92BF92CF92DF92EF92FF9293
:10E600000F931F93CF93DF93CDB7DEB76D970FB600
:10E61000F894DEBF0FBECDBF2091B10A3091B20A8F
:10E62000FF24F394232B09F420C1811149C0FF2456
:10E63000F39466E672E187EA9FE00F94CC0B87EAD9
:10E640009FE00F94160A8091360A8F5F8093360AF6
:10E65000E091E510F091E610309709F48DC0068145
:10E6600017810115110509F491C0D80118968C91F4
:10E670008F70853009F5C8010E9429D98823E1F0FF
:10E68000F80160817181CE0101960E94E838CE01C7
:10E6900001960E946F2D882359F08A859B850097EB
:10E6A00039F0DC01ED91FC910084F185E02D1995A4
:10E6B000CE0101960E947439F80102811381D1CFF5
:10E6C0006FE972E187EA9FE00F94CC0B87EA9FE045
:10E6D0000F94160A0E947EEA2B013C018091DF1004
:10E6E000882381F10E947EEA9B01AC01A12CB12C10
:10E6F000650110E1E12E17E2F12E00E010E0C30108
:10E70000B2010F94562781111DC00F9419108091EA
:10E71000E910811128C00E94A9718091E3109091A5
:10E72000E410059741F08091E5109091E610892B57
:10E7300011F00E9444CF0E9410D082E090E00E942D
:10E740004CC8CCCF8091DF10882309F470CF6CE7E0
:10E7500072E180E09FE00F94CC0B80E09FE00F948B
:10E76000160AF12C66CF8091E7109091E810892B62
:10E7700091F20E94F6C4CFCF66E572E187EA9FE08E
:10E780000F94CC0B87EA9FE00F94160A1092B00A00
:10E790001092AF0A6EE472E187EA9FE00F94CC0B0F
:10E7A00087EA9FE00F94160A64E670E080E090E04C
:10E7B0000E948CE81092BA0A1092AE0A66E372E1E7
:10E7C00087EA9FE00F94CC0B0F94FA29AB01BC01B0
:10E7D0002AE030E087EA9FE00F94310A8091B10A85
:10E7E0009091B20A009711F00E944DE31092B20A84
:10E7F0001092B10A1092E2101092E1101092E610FD
:10E800001092E5101092C8101092C7101092AC0A26
:10E810001092AB0A1092C6101092C5101092AA0A5C
:10E820001092A90A1092E8101092E7101092B50AFF
:10E830001092B40A61E372E187EA9FE00F94CC0B77
:10E840000F94FA29AB01BC012AE030E087EA9FE08F
:10E850000F94310A87EA9FE00F94160A1092AD0ACE
:10E860008091360A81508093360A8F2D6D960FB6AF
:10E87000F894DEBF0FBECDBFDF91CF911F910F91F6
:10E88000FF90EF90DF90CF90BF90AF907F906F9010
:10E890005F904F9008954F925F926F927F928F9208
:10E8A0009F92AF92BF92CF92DF92EF92FF920F931F
:10E8B0001F93CF93DF93CDB7DEB7C659D1090FB6FB
:10E8C000F894DEBF0FBECDBF8E010F5B1F4FD80186
:10E8D0001D921C92FE01ED5BFF4F8EE1DF011D9248
:10E8E0008A95E9F78091D20E9091D30E892B09F485
:10E8F000FEC10E9439D9882309F4F9C1A091D20E32
:10E90000B091D30E52961C921E92519754961C921F
:10E910001E92539784E890E01D969C938E931C97CB
:10E920001E961C921E9782E755968C935597ED91F3
:10E93000FC9111970088F189E02D60E270E0CD0133
:10E9400019954FE150E0B8018091D20E9091D30E0D
:10E950000E948ED97C018091D20E9091D30EDC0161
:10E96000ED91FC910488F589E02D1995E114F104ED
:10E9700009F4BDC1F801EE0DFF1D10828091DF0E7C
:10E980001F928F938091DE0E1F928F938091DD0EE8
:10E990001F928F938091DC0E1F928F938091DB0EDC
:10E9A0001F928F938091DA0E1F928F938CEE96E0D8
:10E9B0009F938F931F9280E48F93FE0131966F0196
:10E9C000FF93EF930F9481436DEB7EE186EF9EE022
:10E9D0000F94CC0BB80186EF9EE00F94660BB60146
:10E9E00086EF9EE00F94660B86EF9EE00F94160A6A
:10E9F0007E01F1E6EF0EF11CD70113961C921E92D8
:10EA0000129788EE93E0A0E0B0E0F701848395834D
:10EA1000A683B78384E0848782E195E09183808335
:10EA200016861586108B0787128A118A80E590E07A
:10EA3000948B838B178A61EE7DE187EA9FE00F94C8
:10EA4000CC0B64ED7EE0CE0187589F4F0F94A30757
:10EA5000BE0167587F4F87EA9FE00F94BE0B87EA9D
:10EA60009FE00F94160ACE0187589F4F0F949B0783
:10EA70006BE177E0CE0185579F4F0F94AC076BE1B8
:10EA800077E0CE0187589F4F0F94AC07BE016758BF
:10EA90007F4FCE018D579F4F0F94A3074091D80E03
:10EAA0005091D90E6091D40E7091D50ECE018D5734
:10EAB0009F4F0F94C7060FB6F894DEBF0FBECDBFB1
:10EAC000811105C0CE018D579F4F0F942C07C15760
:10EAD000DF4F48815981CF58D040C557DF4F6881FB
:10EAE0007981CB58D040CE018D579F4F0F94C706E8
:10EAF000811105C0CE018D579F4F0F942C07BE0189
:10EB00006D577F4FCE018F569F4F0F94A307CE01B5
:10EB10008D579F4F0F949B07CE0187589F4F0F949F
:10EB20009B07CE0185579F4F0F949B078DE197E080
:10EB3000CD57DF4F99838883C358D040C957DF4FE3
:10EB400019821882C758D040C757DF4F19821882E0
:10EB5000C958D040CF56DF4F88819981C159D040E4
:10EB6000CB57DF4F99838883C558D04067EB7EE150
:10EB700087EA9FE00F94CC0B0F94FA29AB01BC01FC
:10EB80002AE030E087EA9FE00F94310A87EA9FE0AD
:10EB90000F94160A64E670E080E090E00E948CE832
:10EBA00086E091E4D7011E969C938E931D9761E5B4
:10EBB00072E085EF92E00F9420388C01892B09F4E4
:10EBC000EEC083E090E00F94DD34F80195878487F0
:10EBD000DC011196FC92EE9212961C92C7010F94E2
:10EBE0005719882319F0C7010F940F20F701618985
:10EBF0007289A388B4886115710509F48FC0CE01AC
:10EC000087589F4F0F94110CA501BE0167587F4F85
:10EC1000C7010F94BF20181619060CF0BDC0D7010C
:10EC20001F96BC901F975096AC90DF92CF928CE3CA
:10EC30009EE19F938F931F930F930F94A738DF92BA
:10EC4000CF9287E39EE19F938F931F930F930F942F
:10EC5000A738D8011C96ED91FC9181E08283DF9268
:10EC6000CF9284E39EE19F938F931F930F930F9412
:10EC7000A738D8011C96ED91FC911282AF92BF92F9
:10EC80008EEF9DE19F938F931F930F930F94A7385F
:10EC90000FB6F894DEBF0FBECDBFB12C85EFC82EE6
:10ECA0008DE1D82EBB2D24E0B202F001112483E8BF
:10ECB00090E08C0F9D1FE80FF91F808191810097D4
:10ECC000A1F12281338121153105C9F33F932F939F
:10ECD0009F938F93DF92CF921F930F930F94A73838
:10ECE000B3940FB6F894DEBF0FBECDBFDBCF40E2CA
:10ECF00050E06FEE7EE1C8010F944D3761ED7EE18B
:10ED000086EF9EE00F94CC0BB80186EF9EE00F9447
:10ED1000660B86EF9EE00F94160A30CE67857089E9
:10ED2000A501C7010F940A1D76CF89E39EE19F9349
:10ED30008F931F930F930F94A738F701168A158AA4
:10ED4000D8011C96ED91FC91C080D1800F900F905E
:10ED50000F900F9033E3A32EB12CD601ED91FC91CF
:10ED60000084F185E02DC601199541975CF4B1E06E
:10ED7000AB1AB10839F064E170E080E090E00E94E5
:10ED80008CE8EBCFD601ED91FC910084F185E02D6C
:10ED9000C6011995419734F4C8010F94FB1210E095
:10EDA00000E065C06AE879E0CE0185579F4F0F9477
:10EDB000AC07912CA12CD601ED91FC910688F78926
:10EDC000E02DC6011995882309F446C0BDE0AB12B9
:10EDD00001C0A92CD601ED91FC910688F789E02DA0
:10EDE000C60119958111DEC0D601ED91FC91008418
:10EDF000F185E02DC6011995892B09F4E5C0D601EE
:10EE0000ED91FC910284F385E02DC6011995B82E91
:10EE1000BAE08B1709F4DAC0EDE08E1709F4D6C01A
:10EE2000FFEF8F1709F4D0C0EA968FAFEA97EB9601
:10EE30001FAEEB9741E050E0BE0167587F4FCE0117
:10EE400085579F4F0F94C7069A2CAB2CB4CFBAE0CE
:10EE5000BB12FACFAB12F8CFCC24C394D12CCE0185
:10EE600085579F4F0F949B07CD2809F498CFD70162
:10EE70005596ED90FC9069EA7EE187EA9FE00F9459
:10EE8000CC0B4AE050E0B70187EA9FE00F941D0BDE
:10EE900087EA9FE00F94160A64E670E080E090E055
:10EEA0000E948CE80115110509F469C1B8ECEB1654
:10EEB000F10409F040C16DE97EE186EF9EE00F9418
:10EEC000CC0B64EF71E080E090E00E948CE8ED965E
:10EED0001FAE1EAEED97EF961FAE1EAEEF978FEFF3
:10EEE0009FEFC158DF4F99838883CF57D04084E983
:10EEF00094E0EB969FAF8EAFEB97CF57DF4F198320
:10EF00000883C158D040F89481E00E94F672CE0187
:10EF100087589F4F0E94B6E39093B20A8093B10A3C
:10EF20007894C8010F94FB128091B10A9091B20AB3
:10EF3000892B09F0EEC06AE879E0CE0185579F4F32
:10EF40000F94AC07CE0185579F4F0E9479F2CE01F6
:10EF500085579F4F0F949B0766E87EE180E09FE016
:10EF60000F94CC0BF12CE12CCE018F569F4F0F94B8
:10EF70009B07C701CA56DF4F0FB6F894DEBF0FBE1E
:10EF8000CDBFDF91CF911F910F91FF90EF90DF9058
:10EF9000CF90BF90AF909F908F907F906F905F9039
:10EFA0004F900895D601ED91FC910084F185E02DFC
:10EFB000C6011995892B09F017CF64E670E080E04F
:10EFC00090E00E948CE806CFBB24BA946BE277E015
:10EFD0008AE09FE00F94660BBE0165577F4F8AE081
:10EFE0009FE00F94BE0B8AE09FE00F94160AEB9609
:10EFF0001FAE1EAEEB97ED961FAE1EAEED97EF96D1
:10F000001FAE1EAEEF976CEE7DE1CE0187589F4F8D
:10F010000F943E07C157DF4F28813981CF58D04028
:10F02000EF968EAD9FADEF97912C2817390748F0DA
:10F03000BE0167587F4FCE0185579F4F0E9454E510
:10F04000982ECE0187589F4F0F949B07992079F1F6
:10F05000C157DF4F28813981CF58D04049E050E077
:10F06000BE0165577F4FCE0187589F4F0F94BD0754
:10F07000EB968EAD9FADEB97412C512C3201009752
:10F0800019F00F94C8362B014201CE0187589F4FCB
:10F090000F949B074114510429F0D70156965C92B6
:10F0A0004E925597B4018AE09FE00E94FBDCF70185
:10F0B0008584968481149104D1F0C157DF4F8881F3
:10F0C0009981CF58D040892B91F0BE0165577F4F71
:10F0D000CE0187589F4F0F94A307CE0187589F4FAB
:10F0E000F4011995CE0187589F4F0F949B0750E06C
:10F0F00040E06AE879E0CE0185579F4F0F9463079F
:10F10000FFEFBF12A4CEC8010F94FB12D12CC12C6B
:10F11000A6CE0E94596B8091AE0A882329F00E94E6
:10F120001EDC67FF0E9401C86FE77EE186EF9EE06C
:10F130000F94CC0B19CFE0E3EE16E1E0FE0651F49C
:10F140006BE67EE186EF9EE00F94CC0BC8010F9436
:10F15000FB120ACF63E57EE180E09FE00F94CC0BC9
:10F16000C8010F94FB124AE050E0B70180E09FE035
:10F170000F941D0B80E09FE00F94160AF5CE60E41B
:10F180007EE187EA9FE00F94CC0BEE24EA94FE2CFC
:10F19000EBCE0F931F93CF93DF93EB0102970CF409
:10F1A000A1C00A811B816EEF7CE1C8010F94F83683
:10F1B000892B61F40E941EDC677F0E9478DC88EC5A
:10F1C00090E0DF91CF911F910F91089567E07DE16D
:10F1D000C8010F94F836892B21F40E941EDC686068
:10F1E000ECCF65ED7CE186EF9EE00F94CC0B0E94A6
:10F1F0001EDC63FB662760F981E0682770E04AE067
:10F2000050E086EF9EE00F941D0B86EF9EE00F947A
:10F21000160A8091D20E9091D30E892B09F452C018
:10F220000A811B810E9439D9882309F44BC0F80157
:10F2300001900020E9F73197E01BF10BB09708F03F
:10F2400041C0A091D20EB091D30E52961C921E9244
:10F25000519754961C921E92539784E890E01D9605
:10F260009C938E931C971E961C921E9782E7559630
:10F270008C935597ED91FC9111970088F189E02DC1
:10F2800060E270E0CD011995B8018091D20E9091A5
:10F29000D30E0F94660B8091D20E9091D30EDC01A9
:10F2A000ED91FC910190F081E02D60E01995809145
:10F2B000D20E9091D30EDC01ED91FC910488F5897A
:10F2C000E02D19956A817B8186EF9EE00F94660B95
:10F2D0006EEC7CE186EF9EE00F94CC0B86EF9EE017
:10F2E0000F94160A8091E3109091E41002977CF13C
:10F2F0000E944B74883C910539F424E030E030934F
:10F30000E4102093E3105DCF8F3F9807C9F463EBBF
:10F310007CE187EA9FE00F94CC0B87EA9FE00F9493
:10F32000160A1092AD0A83E090E09093E410809367
:10F33000E31085EC9EE00F940F2089EC90E041CF24
:10F340002091AE0A2111D9CF2FE030E0D8CF66EA64
:10F350007CE180E09FE00F94CC0B80E09FE00F9475
:10F36000160A84EF91E02DCF4F925F926F927F92B9
:10F370008F929F92AF92BF92CF92DF92EF92FF92C5
:10F380000F931F93CF93DF93CDB7DEB7C357D14011
:10F390000FB6F894DEBF0FBECDBF2091E3103091C1
:10F3A000E410F9013B96EB31F10508F06EC68827B1
:10F3B000E352F6488F4F0D94CC3ECF88C2884580EB
:10F3C0004580458045804580458045804580458015
:10F3D000F8799D81A481B081F681AC85BC88458097
:10F3E0004580458045804580F0884C8974896789CF
:10F3F0008AE895E0C259DE4F99838883CE56D14082
:10F40000C059DE4F188219821A821B82C057D14020
:10F41000C859DE4F99838883C856D140C659DE4FFC
:10F42000188219821A821B82CA56D140CE59DE4FE9
:10F4300099838883C256D140CC59DE4F18821982F5
:10F440001A821B82C456D140CE5BDE4F99838883DB
:10F45000C254D140CC5BDE4F188219821A821B82C3
:10F46000C454D14063E574E186EF9EE00F94CC0B69
:10F4700086EF9EE00F94160A8091D20E9091D30EE3
:10F480008E010F571F4F892B09F471C00E9439D983
:10F49000882309F46CC0A091D20EB091D30E52967D
:10F4A0001C921E92519754961C921E92539784E878
:10F4B00090E01D969C938E931C971E961C921E970F
:10F4C00082E755968C935597ED91FC9111970088A2
:10F4D000F189E02D60E170E0CD01199544E050E044
:10F4E000BE016F5F7F4F8091D20E9091D30E0F942B
:10F4F000980989819A81AB81BC81C059DE4F88838C
:10F500009983AA83BB83C057D1408091D20E90913A
:10F51000D30EDC01ED91FC910488F589E02D19955D
:10F52000C059DE4F8881C057D140882301F18F3FF9
:10F53000A9F4CF58DE4F8881C157D1408F3F71F475
:10F54000CE58DE4F8881C257D1408F3F39F4CD5815
:10F55000DE4F8881C357D1408F3F49F00E941EDCA7
:10F5600070FF8FC180919E0A833008F08AC167E4E2
:10F5700074E186EF9EE00F94CC0B0FB6F894A8953B
:10F5800080916000886180936000109260000FBEDF
:10F590008091950A81112AC010927D0A10927C0AEE
:10F5A00088EE93E0A0E0B0E080937E0A90937F0A1B
:10F5B000A093800AB093810A82E695E090937B0A3B
:10F5C00080937A0A8AE895E09093890A8093880A62
:10F5D00010928A0A10928B0A10928C0A10928D0A4D
:10F5E00084E08093920A81E08093950A87E39AE011
:10F5F0009093FB0C8093FA0C0E94EBE880E590E07E
:10F600000E94D4E346E050E06AED7EE089E090E0BD
:10F610000F9408148AE895E09A8389831B821C82E0
:10F620001D821E82CE0103960F94BA140F94CF143C
:10F630008091FA0C9091FB0CFC0112A213A214A26F
:10F6400015A2DC0116A217A210A611A612A613A6D7
:10F6500014A615A640EE5EE260E070E046AB57AB44
:10F6600060AF71AF40EA5FE060E070E042AF53AF7F
:10F6700064AF75AF189626E0FD01322F11923A95CE
:10F68000E9F7AC01425F5F4F34E1FA0111923A951C
:10F69000E9F7EAEDFEE001900D922A95E1F7FC0111
:10F6A000EE5BFF4F10820F948B1E7C01019709F0D7
:10F6B00046C080E590E00E94D4E36091FA0C70911E
:10F6C000FB0C625F7F4FCE0101960F94110CCE01AF
:10F6D00003960F94BA146091FA0C7091FB0C6A5E59
:10F6E0007F4FCE0101960F94110CCE0103960F941B
:10F6F000C8146091FA0C7091FB0C6E5E7F4FCE01C6
:10F7000001960F94110CCE0103960F94C1140F941F
:10F71000CF146091FA0C7091FB0C625E7F4FCE01AA
:10F7200001960F94110C8B819C81AD81BE818093D9
:10F73000F60C9093F70CA093F80CB093F90C88E1B9
:10F7400099E20FB6F894A895809360000FBE90934D
:10F750006000A895EF2809F429C36EE973E186EFEC
:10F760009EE00F94CC0BCE0101960E94D7E38B81D3
:10F770009C81AD81BE81C059DE4F88839983AA8365
:10F78000BB83C057D1403AE8E32E35E0F32EFA822E
:10F79000E982CE0101960F940D2986EF9EE00F9429
:10F7A000160ACE0182599E4F0E947ADA8091F60C99
:10F7B0009091F70CA091F80CB091F90C8B839C837D
:10F7C000AD83BE83C659DE4F88839983AA83BB83EA
:10F7D000CA56D140CE0188599E4F0E944CDBFA8216
:10F7E000E9821B821C821D821E8280E590E00E94BD
:10F7F000D4E344E050E0BE016D5F7F4F81E090E0D4
:10F800000F94D8130F94CF148B819C81AD81BE814E
:10F81000CC59DE4F88839983AA83BB83C456D140D9
:10F82000CE018E599E4F0E94B5DBFA82E9821B827F
:10F830001C821D821E8280E590E00E94D4E344E099
:10F8400050E0BE016D5F7F4F85E090E00F94D813CC
:10F850000F94CF148B819C81AD81BE81CC5BDE4F38
:10F8600088839983AA83BB83C454D140CE018E5B25
:10F870009E4F0E94E3DA81E00E94DCDC10929E0A37
:10F8800016C261E374E186EF9EE00F94CC0B8AE828
:10F8900095E09A838983C059DE4F88819981AA8136
:10F8A000BB81C057D1408B839C83AD83BE83CE0187
:10F8B00001960F940D298091D20E9091D30E892B31
:10F8C00009F45FC20E9439D9882309F45AC2A09171
:10F8D000D20EB091D30E52961C921E92519754960E
:10F8E0001C921E92539784E890E01D969C938E93F1
:10F8F0001C971E961C921E9782E755968C935597DF
:10F90000ED91FC9111970088F189E02D64E170E0A0
:10F91000CD01199544E050E0BE016F5F7F4F8091AB
:10F92000D20E9091D30E0F94980989819A81AB8160
:10F93000BC81C659DE4F88839983AA83BB83CA568C
:10F94000D1408091D20E9091D30EDC01ED91FC91CB
:10F950000488F589E02D1995C659DE4F8881CA566D
:10F96000D140882309F40DC28F3FB1F4C559DE4F51
:10F970008881CB56D1408F3F79F4C459DE4F8881BE
:10F98000CC56D1408F3F41F4C359DE4F8881CD56CC
:10F99000D1408F3F09F4F5C16BE274E186EF9EE040
:10F9A0000F94CC0B8AE895E09A838983C659DE4F81
:10F9B00088819981AA81BB81CA56D1408B839C835F
:10F9C000AD83BE83CE0101960F940D298091D20E96
:10F9D0009091D30E892B09F4ADC10E9439D98823A7
:10F9E00009F4A8C1A091D20EB091D30E52961C92E8
:10F9F0001E92519754961C921E92539784E890E061
:10FA00001D969C938E931C971E961C921E9782E7C0
:10FA100055968C935597ED91FC9111970088F1893B
:10FA2000E02D68E170E0CD01199544E050E0BE01A1
:10FA30006F5F7F4F8091D20E9091D30E0F949809F3
:10FA400089819A81AB81BC81CC59DE4F88839983AF
:10FA5000AA83BB83C456D1408091D20E9091D30E1D
:10FA6000DC01ED91FC910488F589E02D1995CC59C4
:10FA7000DE4F8881C456D140882309F45BC18F3F93
:10FA8000B1F4CB59DE4F8881C556D1408F3F79F410
:10FA9000CA59DE4F8881C656D1408F3F41F4C959BB
:10FAA000DE4F8881C756D1408F3F09F443C166E2DB
:10FAB00074E186EF9EE00F94CC0B8AE895E09A8380
:10FAC0008983CC59DE4F88819981AA81BB81C45634
:10FAD000D1408B839C83AD83BE83CE0101960F946E
:10FAE0000D298091D20E9091D30E892B09F4E2C09A
:10FAF0000E9439D9882309F4DDC0A091D20EB091BB
:10FB0000D30E52961C921E92519754961C921E929E
:10FB1000539784E890E01D969C938E931C971E96B5
:10FB20001C921E9782E755968C935597ED91FC9108
:10FB300011970088F189E02D6CE170E0CD011995F5
:10FB400044E050E0BE016F5F7F4F8091D20E9091F4
:10FB5000D30E0F94980989819A81AB81BC81CC5BCB
:10FB6000DE4F88839983AA83BB83C454D14080919C
:10FB7000D20E9091D30EDC01ED91FC910488F589B1
:10FB8000E02D1995CC5BDE4F8881C454D140882389
:10FB900009F490C08F3FB1F4CB5BDE4F8881C55430
:10FBA000D1408F3F79F4CA5BDE4F8881C654D14083
:10FBB0008F3F41F4C95BDE4F8881C754D1408F3FEE
:10FBC00009F478C06FE174E186EF9EE00F94CC0BEE
:10FBD0004AE8E42E45E0F42EFA82E982CC5BDE4F5F
:10FBE00088819981AA81BB81C454D1408B839C8335
:10FBF000AD83BE83CE0101960F940D29FA82E9826E
:10FC0000CC5BDE4F88819981AA81BB81C454D140ED
:10FC10008B839C83AD83BE83F801F182E082CC5953
:10FC2000DE4F88819981AA81BB81C456D1408283ED
:10FC30009383A483B583CE53DF4FF982E882C25CFD
:10FC4000D040C659DE4F88819981AA81BB81CA56AE
:10FC5000D140CC53DF4F88839983AA83BB83C45C94
:10FC6000D040CE5FDE4FF982E882C250D140C05909
:10FC7000DE4F88819981AA81BB81C057D140CC5F7A
:10FC8000DE4F88839983AA83BB83C450D1409E01F1
:10FC90002F5F3F4FA801BE016E537F4FCE018E5F95
:10FCA0009E4F0E946DE986EF9EE00F94160A82E057
:10FCB00090E08FC08AE895E09A838983CC59DE4F23
:10FCC000488159816A817B81C456D1404B835C83D2
:10FCD0006D837E83D8018D939C93C659DE4F4881F6
:10FCE00059816A817B81CA56D140F801428353838E
:10FCF00064837583CE53DF4F99838883C25CD04081
:10FD0000C059DE4F88819981AA81BB81C057D140FB
:10FD1000CC53DF4F88839983AA83BB83C45CD040D4
:10FD2000AE014F5F5F4FB801CE018E539F4F0E94CF
:10FD3000AAE9B9CF8AE895E09A838983C659DE4F4C
:10FD4000488159816A817B81CA56D1404B835C834B
:10FD50006D837E83D8018D939C93C059DE4F88813B
:10FD60009981AA81BB81C057D140F80182839383D6
:10FD7000A483B583BE016F5F7F4FC8010E94FCE979
:10FD800092CF8AE895E09A838983C059DE4F8881B3
:10FD90009981AA81BB81C057D1408B839C83AD835D
:10FDA000BE83CE0101960E9447EA7DCF6DED73E1DF
:10FDB00080E09FE00F94CC0B6EEA73E180E09FE05F
:10FDC0000F94CC0B80919E0A8F5F80939E0A86EFE2
:10FDD0009FEF9093E4108093E31089E0ECE5F2E06C
:10FDE000D80101900D928A95E1F787E1F8013996E3
:10FDF000DF011D928A95E9F78EED9EE0009731F0C4
:10FE0000A801485F5F4F62E00F94B827CE018E5380
:10FE10009F4F0E94D7E30E947EEA683B7B408105AA
:10FE2000910538F464E670E080E090E00E948CE890
:10FE3000F2CFCC53DF4F88819981AA81BB81C45C0A
:10FE4000D04080936C0E90936D0EA0936E0EB09385
:10FE50006F0EC8010E9419E5892BC9F0E090680E69
:10FE6000F090690ED701ED91FC91C088D18868E2CD
:10FE700072E0CE0101960F94110C49EE54E1BE01DF
:10FE80006F5F7F4FC701F6011995811130C26DE791
:10FE900073E180E09FE00F94CC0B80E09FE00F9433
:10FEA000160A2CE7A22E2EE0B22E7501D12CC12C01
:10FEB000D7018D919C91892B49F1960143E050E047
:10FEC00060E070E0CB010E9484F3D701ED91FC91DA
:10FED00080859185009711F00F947935D701ED91C8
:10FEE000FC9186819781009711F00F947935D701A5
:10FEF000ED91FC91848195810F947935F701808192
:10FF000091810F947935D7011D921C92BFEFCB1AC6
:10FF1000DB0AE2E0EE0EF11CF8E0CF16D10441F668
:10FF200086E0ECE7F2E09E012F5F3F4F4901D901E7
:10FF300001900D928A95E1F7FE0137968AE1DF0183
:10FF40001D928A95E9F78AED9EE0009731F0AE01A7
:10FF50004A5F5F4F66E00F94B8276EE277E0C80112
:10FF60000F942343D12CC12CF501819191915F0114
:10FF7000892B09F0C5C18AE090E00F94DD347C0143
:10FF8000009709F4BDC1DC0119961C921E921897C6
:10FF900015961C921E921497F80101900020E9F723
:10FFA000CF010197801B910B0F94DD345C01D701C9
:10FFB00015969C938E931497892B11F40C94F489C5
:10FFC000F40101900020E9F7CF0101978819990900
:10FFD0000F94DD34D70119969C938E931897009750
:10FFE00011F40C94F189B4010F94424380E590E040
:10FFF000F7019183808313821282B801C5010F94A7
:020000021000EC
:100000004243F50101900020E9F73197AE16BF0693
:1000100020F4319781818E32C9F75F0122E0A20E70
:10002000B11CD5010D900020E9F7CD018A199B097B
:100030000B960F94DD344C01F7019783868300976C
:1000400041F0B5010F94424365E377E0C4010F949A
:100050002343F601EE0FFF1FE458F14FF182E082D7
:10006000960142E050E060E070E0CB010E9484F332
:10007000019709F44EC161E477E080E09FE00F94BE
:10008000660B80E09FE00F94160A0FB6F894A895CF
:1000900080916000886180936000109260000FBEC4
:1000A0008091E3109091E41002970CF4F9C08091D4
:1000B0009E0A8111F5C00091FA0C1091FB0C0115FC
:1000C000110509F4EDC00E947EEA4B015C01780144
:1000D000FEE3EF0EF11CF70180819181A281B381D3
:1000E000A5019401281B390B4A0B5B0BCA01B9010E
:1000F000683E33E0730781059105B0F128EE33E0E7
:1001000040E050E00F94553E861A970AA80AB90AB3
:10011000D7018D929D92AD92BC921397F80186A55E
:1001200097A5A0A9B1A969017A01CC0CDD1CEE1C30
:10013000FF1C8C159D05AE05BF0510F00C94A3891E
:1001400016A617A610AA11AAF80182A993A9A4A914
:10015000B5A98C159D05AE05BF0510F00C94AD89B1
:1001600012AA13AA14AA15AAF80186A597A5A0A9F0
:10017000B1A9892B8A2B8B2B11F00C94B789EE5BDC
:10018000FF4F8081833011F00C94B78984E0808325
:10019000C8010F948B1E01967C01F80182A993A9D6
:1001A000A4A9B5A9892B8A2B8B2BA1F4EE5BFF4F59
:1001B0008081833011F081110DC01082F8013E96CC
:1001C00084E1DF011D928A95E9F7C8010F948B1E27
:1001D00003967C01B2E0EB16F10429F0E4E0EE16A0
:1001E000F10409F046C080E590E00E94D4E36091FC
:1001F000FA0C7091FB0C625F7F4FCE0101960F9459
:10020000110CCE0103960F94BA146091FA0C709100
:10021000FB0C6A5E7F4FCE0101960F94110CCE014C
:1002200003960F94C8146091FA0C7091FB0C6E5EEB
:100230007F4FCE0101960F94110CCE0103960F94BF
:10024000C1140F94CF146091FA0C7091FB0C625E94
:100250007F4FCE0101960F94110C8B819C81AD8153
:10026000BE818093F60C9093F70CA093F80CB0939A
:10027000F90CF3E0EF16F10411F40C94DA8914F0A0
:100280000C94BB8931E0E316F10411F40C94D78986
:1002900061E676E142E0E416F10411F40C94DF89A2
:1002A00088E199E20FB6F894A895809360000FBE9C
:1002B000909360002091E3103091E410C901CD5873
:1002C000DE4F0FB6F894DEBF0FBECDBFDF91CF91EA
:1002D0001F910F91FF90EF90DF90CF90BF90AF9064
:1002E0009F908F907F906F905F904F90089565E6FC
:1002F00073E186EF9EE00F94CC0B86EF9EE0CFCDAE
:10030000FFEFCF1ADF0A28E0C216D10409F02CCE85
:10031000B2CE64E573E186EF9EE00F94CC0BB8019A
:1003200086EF9EE00F94660B6DE473E186EF9EE02E
:100330000F94CC0B86EF9EE0A6CE82E090E09093E7
:10034000E4108093E310A1CE8091A30A811105C02F
:100350000E94F11D81E08093A30A83E090E0EFCF3B
:100360008091DF108111AACF0E941EDC63FD2EC098
:100370008091AD0A811127C00E944B74883C910581
:1003800019F484E090E0DBCF8091AE0A882359F025
:1003900062E377E186EF9EE00F94CC0B86EF9EE060
:1003A0000F94160AEECFCE0101960E94D7E38B81FF
:1003B0009C81AD81BE81892B8A2B8B2B09F435C2A0
:1003C0008FE090E0BCCF62E277E1E4CF8091AE0AAB
:1003D000882349F084E090E09093E4108093E31048
:1003E00068EE76E1A3CF8FE090E0F6CFA8958091FC
:1003F000AB0A9091AC0A009721F00E9429D9823073
:1004000068F465ED76E186EF9EE00F94CC0B86EF05
:100410009EE00F94160A87E090E091CFCE59DE4F10
:100420001882C256D140FE01EE5FFE4F119211922A
:100430008EE0DF011D928A95E9F70E9403D8882398
:1004400019F085E090E07BCFE090AB0AF090AC0A29
:10045000E114F10441F0C7010E9429D9082F10E0EE
:10046000023011055CF46FE575E180E09FE00F94C8
:10047000CC0B80E09FE00F94160AA2CF70E060E002
:10048000C7010E94521B009709F49CC09093C610AC
:100490008093C51062E575E186EF9EE00F94CC0B6A
:1004A0006091C5107091C61086EF9EE00F94660BA8
:1004B00086EF9EE00F94160A8091C5109091C610A9
:1004C0000E9419E5892B09F080C062E677E080E0A0
:1004D0009FE00F94660B80E09FE00F94160AE09077
:1004E000AB0AF090AC0A61E070E0C7010E94521BB9
:1004F0005C010230110509F47FC062E0C7010E946F
:1005000097D8FC01C184D2840330110509F47DC061
:1005100063E070E0C7010E94521B7C018091D20E03
:100520009091D30E892B09F475C00E9439D9882384
:1005300009F470C0A091D20EB091D30E52961C92C5
:100540001E92519754961C921E92539784E890E005
:100550001D969C938E931C971E961C921E9782E765
:1005600055968C935597ED91FC9111970088F189E0
:10057000E02D60E470E0CD0119954FE050E0BE0140
:100580006E5F7E4F8091D20E9091D30E0E948ED9D5
:100590004C018091D20E9091D30EDC01ED91FC9133
:1005A0000488F589E02D19958114910499F1E2E010
:1005B000F1E0EC0FFD1FE80DF91D10828E010E5FBA
:1005C0001E4F3EC087E594E061CF6EE375E186EF94
:1005D0009EE00F94CC0B6091C5107091C61086EF11
:1005E0009EE00F94660B67E375E186EF9EE00F9443
:1005F000CC0B86EF9EE071CF8BE5C82E87E0D82E1E
:100600009E012E593E4F790189CFAE014E595E4F62
:100610007A0184CF053011058CF264E070E080919E
:10062000AB0A9091AC0A0E94521B8C0167E175E104
:1006300086EF9EE00F94CC0B86EF9EE00F94160A97
:10064000B092420DA092410DD092440DC092430D44
:1006500082E899E390933A0D8093390D40E150E0A0
:100660006AE075E1CE018E539F4F0F944D3730E015
:1006700020E041E050E060E2CE018F579F4F0F94A1
:10068000792840E250E066E171E2CE018F579F4F3A
:100690000F942F376AEE74E186EF9EE00F94CC0B37
:1006A000B50186EF9EE00F94660B68EE74E186EF6D
:1006B0009EE00F94CC0B4AE050E0B60186EF9EE03E
:1006C0000F941D0B61EE74E186EF9EE00F94CC0B4E
:1006D000B70186EF9EE00F94660B6CED74E186EF38
:1006E0009EE00F94CC0BF7018081811104C010E0D3
:1006F00000E0F12CE12CA090C510B090C6100E9433
:1007000003D88111B5C18091240D9091250DDC0194
:10071000ED91FC910688F789E02D1995882309F45D
:1007200087C081E090E090932F0D80932E0D87E09D
:10073000ECE9F2E0DE01119601900D928A95E1F765
:10074000FE01319685E090E02191A091260DB091B7
:10075000270DA80FB91F2C9301968C309105A1F796
:1007600086E3E114F10429F086EB0115110509F087
:1007700086EFC090260DD090270DF60184878091DA
:100780002B0D858780912A0D86878090280D90906B
:10079000290DB401C5010F9460374196881699065A
:1007A00008F07DC08091240D9091250DDC01ED9124
:1007B000FC910488F589E02D199565EA74E180E0E3
:1007C0009FE00F94CC0B6091470D7091480D4AE06B
:1007D00050E080E09FE00F941D0B6DE874E180E035
:1007E0009FE00F94CC0B80E09FE00F94160A0E94CC
:1007F0007EEA60939F0A7093A00A8093A10A909367
:10080000A20A80919D0A8F5F80939D0A83330CF426
:10081000A0C160E674E180E09FE00F94CC0B80E023
:100820009FE00F94160A10929D0A86EF9FEF87CDE6
:100830006091410D7091420D8091240D9091250D94
:10084000DC01ED91FC914091430D5091440D6115F7
:10085000710571F00088F189E02D1995019709F46F
:1008600060CF8EEF9FEF9093480D8093470DA5CFFB
:100870000684F785E02D2AE835E03A832983409005
:100880003D0D50903E0D60903F0D7090400D4B829D
:100890005C826D827E82BE016F5F7F4FDECF4FE054
:1008A00050E0B601C5010E943BD86C01A090280D14
:1008B000B090290DB501CE018F579F4F0F9460372F
:1008C0008C0D9D1D0296A816B90608F46BCF609199
:1008D000260D7091270DA601CE018F579F4F0E94C4
:1008E0003BD86C01A090280DB090290DB501CE0128
:1008F0008E539F4F0F9460378C0D9D1D0296A81646
:10090000B90608F44FCF6091260D7091270DA6010E
:10091000CE018E539F4F0E943BD86C01E114F1042D
:10092000B9F1A090280DB090290DB501C7010F9421
:10093000603796012E5F3F4F820F931FA816B906AE
:1009400008F430CF6091260D7091270DA601C701E4
:100950000E943BD86C0101151105D1F0E090280DE3
:10096000F090290DB701C8010F94603796012E5FF2
:100970003F4F820F931FE816F90608F413CF6091DA
:10098000260D7091270DA601C8010E943BD86C016D
:10099000A601455051096091260D7091270D80E107
:1009A0000E948AEA0E947EEA6093300D7093310DB6
:1009B0008093320D9093330D6093340D7093350D09
:1009C0008093360D9093370D8091240D9091250DD5
:1009D000DC01ED91FC910084F185E02D1995892BC6
:1009E00021F50E947EEA0091340D1091350D209181
:1009F000360D3091370D6B017C01C01AD10AE20A25
:100A0000F30A20912C0D30912D0DA8EEB3E00F9438
:100A1000A93EC616D706E806F906B0F28CEF9FEF9E
:100A20009093480D8093470DBDCECE018E5B9E4FB7
:100A30000E94F6EE643071058105910509F0B2CE91
:100A4000E091260DF091270D838190E08111E8CF90
:100A50000E947EEA6093340D7093350D8093360DBD
:100A60009093370D1092380D1092480D1092470D4B
:100A700010929D0A6EEC74E186EF9EE00F94CC0B11
:100A80006091C5107091C61086EF9EE00F94660BC2
:100A900086EF9EE00F94160A81E08093AD0A30E065
:100AA00020E043E050E061E4CE0101960F94792804
:100AB0006CE777E0CE0101960F942343CE010196B7
:100AC0000E9451EB30E020E042E050E061E4CE01D2
:100AD00001960F94792860E877E0CE0101960F9493
:100AE0002343BE016F5F7F4F87EA9FE00F941A0A8E
:100AF000CE0101960E9451EB30E020E041E050E051
:100B000061E4CE0101960F94792860E877E0CE0188
:100B100001960F942343BE016F5F7F4F87EA9FE0EA
:100B20000F941A0ACE0101960E9451EB85E090E0E5
:100B30009093E4108093E3100E947EEA60939F0AF2
:100B40007093A00A8093A10A9093A20A61EB74E1CA
:100B5000EDCB8CE090E0F3CB0E947EEA9B01AC01F0
:100B600060919F0A7091A00A8091A10A9091A20AB7
:100B7000A12CB12C650110E4E12E1FE1F12E00E063
:100B800010E00F945627882309F47FCA30E020E054
:100B900043E050E061E4CE018F579F4F0F947928D6
:100BA0006CE777E0CE018F579F4F0F94234300915E
:100BB000280D1091290DB801CE018F579F4F0F942A
:100BC000603709960817190790F10E9403D8882307
:100BD00071F180912E0D90912F0D019609F441C174
:100BE00090932F0D80932E0DE091260DF091270DFF
:100BF00080912F0D8583E091260DF091270D809136
:100C00002E0D86836091260D7091270D47E050E0F0
:100C1000CE018F579F4F0E943BD8AC0145505109E0
:100C20006091260D7091270D82EA0E948AEAFE01EA
:100C3000EE5FFE4F119211921EE3DF01212F1D92F4
:100C40002A95E9F71A821982FE0133968EE7DF01B1
:100C50001D928A95E9F730E020E041E050E060E441
:100C6000CE018E5F9E4F0F9479284FE350E066E1EE
:100C700071E2CE018E5F9E4F0F942F374FE750E009
:100C800060E171E2CE0101960F944D37BE016F5FB6
:100C90007F4FCE018E5F9E4F0E941BEB30E020E025
:100CA00041E050E060E4CE018E5F9E4F0F947928C2
:100CB0004FE350E06CE276E1CE018E5F9E4F0F94E1
:100CC0002F374FE750E062E276E1CE0101960F94B4
:100CD0004D374FE750E06FE076E1CE0101960F947B
:100CE0002F37BE016F5F7F4FCE018E5F9E4F0E94F8
:100CF0001BEB30E020E041E050E060E4CE018E5F8D
:100D00009E4F0F9479284FE350E06DE271E2CE01DF
:100D10008E5F9E4F0F942F374FE750E06FEF75E1D6
:100D2000CE0101960F944D37BE016F5F7F4FCE010C
:100D30008E5F9E4F0E941BEB30E020E041E050E0D0
:100D400060E4CE018E5F9E4F0F9479284FE350E010
:100D500068EF75E1CE018E5F9E4F0F942F374FE7FE
:100D600050E062EF75E1CE0101960F944D37BE0160
:100D70006F5F7F4FCE018E5F9E4F0E941BEB809175
:100D8000DF108F5F8093DF10A091E510B091E61027
:100D9000109709F4DEC18091A3029091A402AE01E4
:100DA0004E5B5E4FFA01819391932EE111922A9549
:100DB000E9F79E012E533F4FF901819391931192D0
:100DC0001A95E9F716960D911C91F12CE12C809162
:100DD000E5109091E610892B09F42FC1011511053A
:100DE00009F42BC1D80118968C918F70853009F0C9
:100DF000FEC0C8010E9429D9882309F4F8C0D8018F
:100E0000ED91FC91DF010D900020E9F7EE1AFF0A49
:100E1000EA0EFB1E60E0C8010E9497D8FC018185A4
:100E20009285A385B48582319105A105B10550F560
:100E3000FC018827E15EF8478F4F0D94CC3EFC877C
:100E40000F880F88FC87FC873487FC87FC87FC872A
:100E5000FC87428742874287428742874287428790
:100E60000F8881E090E0BCCE4FE150E06CEE75E180
:100E7000CE018E5B9E4F0F944D37CE53DF4F1882BD
:100E8000C25CD04030E020E041E050E060E4CE01C0
:100E90008E5F9E4F0F947928D8016D917C914FE31E
:100EA00050E0CE018E5F9E4F0F94494362E877E099
:100EB000CE018E5F9E4F0F94234340E450E06AECD6
:100EC00075E1CE018E5F9E4F0F942F3765EC75E173
:100ED000CE018E5F9E4F0E94E0F130E020E041E0C5
:100EE00050E060E4CE018E5F9E4F0F947928F801A8
:100EF000608171814FE350E0CE018E5F9E4F0F9471
:100F0000494362E877E0CE018E5F9E4F0F94234302
:100F100040E450E06DEB75E1CE018E5F9E4F0F9483
:100F20002F376CE975E1CE018E5F9E4F0E94E0F194
:100F300030E020E041E050E060E4CE018E5F9E4F63
:100F40000F947928D8016D917C914FE350E0CE0148
:100F50008E5F9E4F0F94494368E877E0CE018E5F25
:100F60009E4F0F9423434FE350E06AEC75E1CE01AE
:100F70008E5F9E4F0F942F37BE016E5B7E4FCE016A
:100F80008E5F9E4F0E941BEBCE53DF4F8881C25C69
:100F9000D040882361F130E020E041E050E060E49F
:100FA000CE018E5F9E4F0F947928F8016081718188
:100FB0004FE350E0CE018E5F9E4F0F94494368E8A7
:100FC00077E0CE018E5F9E4F0F9423434FE350E0B6
:100FD0006DEB75E1CE018E5F9E4F0F942F37BE01F2
:100FE0006E537F4FCE018E5F9E4F0E941BEBD80148
:100FF00012960D911C91EBCE4FE150E064EE75E13D
:10100000CE018E5B9E4F0F944D374FE350E06EED57
:1010100075E1CE018E539F4F0F944D3733CF4FE183
:1010200050E068ED75E1CE018E5B9E4F0F944D3719
:101030004FE350E064ED75E1ECCF30E020E041E0BB
:1010400050E060E4CE018E5F9E4F0F9479284FE30D
:1010500050E065E975E1CE018E5F9E4F0F942F370A
:101060000E9403D88823F1F16091260D7091270D1D
:1010700045E050E0CE018E5F9E4F0E943BD88C0130
:10108000B6E0EB1AF108A701480F591F6091260D31
:101090007091270D81E30E945DD8A091240DB0913D
:1010A000250DA801480F591F4550510925E030E092
:1010B000281B390B6091260D7091270D620F731F4D
:1010C000ED91FC9111970280F381E02DCD011995EE
:1010D0000E947EEA6093300D7093310D8093320D43
:1010E0009093330DE091E510F091E61006811781A1
:1010F0008091E5109091E610892B59F101151105A9
:1011000041F1F80180858F708530F1F4C8010E94AB
:1011100029D98823C9F0D8016D917C91FB010190F8
:101120000020E9F73197AF01461B570B80E29DE0A5
:101130000F940C05F80182819381892B29F06CE2D0
:1011400080E29DE00F942C05D80112960D911C9120
:10115000CFCF8091DF1081508093DF1086E090E048
:101160009093E4108093E3106EEB76E186EF9EE0BF
:101170000F94CC0B0C9445800E9403D881110C94E1
:101180004580FFC80E947EEA60939F0A7093A00A80
:101190008093A10A9093A20A85EF9FEFD0C80E9486
:1011A0007EEA9B01AC0160919F0A7091A00A809138
:1011B000A10A9091A20AA12CB12C650118E8E12E98
:1011C00013E1F12E00E010E00F945627882311F46C
:1011D0000C9445801092E4101092E3100C9445801A
:1011E0000E9403D8882309F44AC0E091260DF091AB
:1011F000270D80EE8083E091260DF091270D11825E
:101200008091240D9091250D6091260D7091270DF0
:10121000DC01ED91FC910280F381E02D42E050E091
:1012200019958FEF9FEF9093480D8093470D809114
:10123000240D9091250DDC01ED91FC910680F78144
:10124000E02D19958091240D9091250DDC01ED91F3
:10125000FC910488F589E02D19950E947EEA60933F
:10126000300D7093310D8093320D9093330D609358
:10127000340D7093350D8093360D9093370D0E9489
:101280007EEA60939F0A7093A00A8093A10A9093CC
:10129000A20A8DE090E053C80E947EEA9B01AC0157
:1012A00060919F0A7091A00A8091A10A9091A20A70
:1012B000A12CB12C650110E1E12E17E2F12E00E026
:1012C00010E00F94562781115CC80C9445800E9451
:1012D0007EEA60939F0A7093A00A8093A10A90937C
:1012E000A20A8EE090E02BC88091DF10811105C02A
:1012F0000E94FACD892B09F044C80E947EEA9B0126
:10130000AC0160919F0A7091A00A8091A10A90910E
:10131000A20AA12CB12C650110E3E12E15E7F12EF4
:1013200000E010E00F945627882311F40C944580B8
:101330006BE976E180E09FE00F94CC0BF0E0E0E019
:1013400019950C944580821B930BA40BB50B86A7B3
:1013500097A7A0ABB1AB0C94A480821B930BA40BFA
:10136000B50B82AB93ABA4ABB5AB0C94B480F12CB2
:10137000E12C0C94CD8054E0E516F104F1F062E923
:1013800076E185E0E816F10411F00C94508180E0DC
:101390009FE00F94CC0B80E09FE00F94160A86EF3D
:1013A0009FEF9093E4108093E3100C9450816EE7CC
:1013B00076E1EDCF6EE476E1EACF62E376E186EFA7
:1013C0009EE00F94CC0BCE0101960E94D7E3CE0194
:1013D00001960F940D2986EF9EE00F94160A0C9447
:1013E0005081C5010F947935D70116968D919C9146
:1013F000009711F00F947935F7018085918500975A
:1014000011F00F947935C7010F9479350C943B8016
:1014100090E080E00895DC01ED91FC910284F38579
:10142000E02D1994DF92EF92FF920F931F93CF93C9
:10143000DF93EC010C891D890115110559F01D8AF6
:101440001C8AC801DF91CF911F910F91FF90EF90FF
:10145000DF900895EC85FD858E859F85DF01A80FBF
:10146000B91F2C91243209F055C011962C912B37BD
:1014700009F050C00296E80FF91FF12CE12CDF01B2
:10148000D190DD2009F446C08DE7D816E9F08FEF42
:10149000E81AF80AF4CF198A188A2C853D85211597
:1014A000310579F08E859F85280F391FF90120813C
:1014B000222321F001969F878E873EC01D861C86C1
:1014C000C0CF0FEF1FEFBDCFE114F10419F11C9253
:1014D0008E859F8502966C857D85680F791FE881D2
:1014E000F9810684F785E02DCE011995998B888BBB
:1014F0001B8A1A8AEC85FD858E859F85E80FF91F6A
:10150000EE0DFF1DD2828E859F850396E80EF91E93
:10151000FF86EE86288939892115310509F4BDCF6A
:101520008A899B89280F391FF9012081222309F418
:10153000B2CF01969B8B8A8B022F220F110B81CF8A
:10154000DC011C96ED91FC911D971E968D919C914E
:10155000E80FF91F8081082E000C990B0895DC011B
:1015600015968D919C91009739F0DC01ED91FC91DD
:101570000680F781E02D19940895FC0183859485F8
:101580009C0144E0359527954A95E1F756E09595FD
:1015900087955A95E1F72817390719F081E090E00F
:1015A000089582E090E0089583E090E00895DC01E2
:1015B0001296ED91FC9113973097B9F016968D9194
:1015C0009C918430910541F08530910541F003975D
:1015D00049F482E090E0089581E090E0089581E18F
:1015E00090E00895808590E0089590E080E008956F
:1015F00085E090E0089590E080E008958EE090E02E
:101600000895DC011296ED91FC9113973097B9F093
:1016100016968D919C918430910541F0853091050D
:1016200041F0039749F482E090E0089581E090E072
:10163000089581E190E00895808590E0089590E01C
:1016400080E0089584E190E00895DC01ED91FC9143
:101650000484F585E02D60E0199581E090E008951F
:10166000DC011496ED91FC9180E0309711F085A19A
:10167000817090E008954F925F926F927F92AF9247
:10168000BF92DF92EF92FF920F931F93CF93DF935E
:1016900000D000D0CDB7DEB77C01D62E8091BA0A3B
:1016A000882309F4BEC0D70114969C91809144020E
:1016B000891708F4B6C080912D0B90912E0BBAE0DB
:1016C0006B13F0C08352954FFC011082D70118961E
:1016D0000D911C910115110509F49FC0F801618558
:1016E00072856115710591F445805680678070841C
:1016F0008091EA0C9091EB0CA091EC0CB091ED0C68
:10170000481659066A067B0609F487C0D8011B965D
:101710004D915C911C974115510509F47EC0F7016C
:10172000248153968C91539790E0322F377002C0EA
:10173000959587953A95E2F780FF6FC0A22EB12C60
:10174000C501887F9370892B39F451968D919C91B6
:10175000887F9370A82AB92AD8018D919C91DC01C9
:10176000ED91FC916115710509F486C00688F78931
:10177000E02D1995019709F050C06CE3F8018081C4
:1017800091810F94CE0AA50170E060E02AE0D801B3
:101790008D919C910F94CA09F801228180819181D9
:1017A00065ED7BE2222311F063ED7BE20F94CC0B1D
:1017B000D8011D966D917C911E978D919C910F94EF
:1017C000660B60E2F801808191810F94CE0AD80106
:1017D0001F966D917C9150978D919C910F94660B03
:1017E000F80122818081918168EC7BE2222311F053
:1017F00062EC7BE20F94CC0B6DED7AE0D8018D9119
:101800009C910F94660BF80180819181DC01ED9130
:10181000FC91008CF18DE02D199510922E0B1092F9
:101820002D0BD70115968D919C911697009771F00D
:1018300014963C9120914502231740F0DC01ED9174
:10184000FC910190F081E02D6D2D199581E090E0E3
:1018500026960FB6F894DEBF0FBECDBFDF91CF91B5
:101860001F910F91FF90EF90DF90BF90AF907F900E
:101870006F905F904F9008950488F589E02D2AE8D5
:1018800035E03A832983D80115964D905D906D908F
:101890007C9018974B825C826D827E82BE016F5F66
:1018A0007F4F67CF8F3491050CF0BBCFBDE06B1736
:1018B00009F4B7CF9C012F5F3F4F30932E0B20933D
:1018C0002D0B8352954FFC016083ABCFCF93DF93F9
:1018D000EC0167EF78E287EA9FE00F94CC0B87EA90
:1018E0009FE00F94160AE881F9810484F585E02DC4
:1018F00060E0CE01199581E090E0DF91CF910895ED
:10190000CF93DF93EC0160E875E287EA9FE00F94E4
:10191000CC0BEA81FB810190F081E02D6081718127
:1019200087EA9FE00F94660B87EA9FE00F94160A00
:10193000E881F9810484F585E02D60E0CE011995F8
:1019400081E090E0DF91CF9108950D9479350D9469
:1019500079350D9479350D9479350D9479350D944B
:1019600079350D9479350D9479350D9479350D943B
:1019700079352F923F924F925F926F927F928F9222
:101980009F92AF92BF92CF92DF92EF92FF920F930E
:101990001F93CF93DF93CDB7DEB7AA970FB6F89416
:1019A000DEBF0FBECDBF5C010E8F1F8F28A339A3F2
:1019B0004AA35BA36CA37DA31C8A1B8ADC01189637
:1019C0008D919C9101979E8B8D8BE114F104D1F048
:1019D000CE0145969F938F9302979F938F938EE8A6
:1019E00097E09F938F93FF92EF920F94EE430FB681
:1019F000F894DEBF0FBECDBF019721F48B899C897F
:101A00009E8B8D8B6B897C894AE050E087EA9FE052
:101A10000F941D0B67E57BE287EA9FE00F94CC0BE8
:101A20006D897E894AE050E087EA9FE00F941D0BA4
:101A300061E57BE287EA9FE00F94CC0BFE8DFAA76D
:101A40004AE050E06F2F87EA9FE00F94330A87EA5D
:101A50009FE00F94160A19861A861B861C861D861F
:101A60001E861F86188A8A858F7080648A87D501B2
:101A700018968D919C912D893E89281739071CF065
:101A800001979E8B8D8B8B899C8997FF02C01C8A46
:101A90001B8A8B889C885401312C212C8D899E892E
:101AA0008A159B050CF46AC1BAA5B13091F1B23028
:101AB00009F453C1EE24EA94FE2C0E8D1F8D28A14B
:101AC00039A14AA15BA16CA17DA1CE0109960E941A
:101AD000884229833A834B835C836D837E838F8323
:101AE00098878091D50A9091D60AFC012281338192
:101AF000A216B30608F088C06F852E8530E050E04E
:101B000040E0542F432F322F2227462B6D85262B62
:101B100033C1E090D50AF090D60AF7018281938113
:101B2000A816B90608F070C0968553850185128500
:101B30004084A92FB0E06484712C658570E0940125
:101B4000220D331D951372C0A901440F551F240F98
:101B5000351F200F311FA20FB31F9C91F301E20F1D
:101B6000F31F1081260F371FD9010C91442009F46F
:101B700052C0512C712C612C692F70E0762F662792
:101B8000072E000C880B990BA30192010F94553E70
:101B9000C901772766276EA37FA388A799A7612F1E
:101BA00070E0762F6627072E000C880B990BA30197
:101BB00092010F94553E542F432F322F22278EA18E
:101BC0009FA1A8A5B9A5822B932BA42BB52B8EA3DF
:101BD0009FA3A8A7B9A7602F70E0762F6627072ECE
:101BE000000C880B990BA30192010F94553E6EA136
:101BF0007FA188A599A5262B372B482B592B232B62
:101C0000242B252B09F4A0C0FFEFAF1ABF0A2FEF3A
